:020000040000FA
:0400000007EF00F016
:100008007582D5ED46F0E7EF4CF066C0D9FF67C0C2
:10001800DAFFDE6ADD6A68C00BF0DFEC49F00BC07E
:10002800B6F00CC0B7F00001B7BF0B0CD890B635CE
:10003800D96EB735DA6E8C0ED926010EDA22DECFEC
:10004800D0F0DDCFD1F0D051D11101E10C0C66C058
:10005800D9FF67C0DAFFD0C0DEFFD1C0DDFFD0C056
:10006800D9FFD1C0DAFFDF5012E020EE01F0D05105
:10007800D926D151DA22DF50AAEC5AF00001C26F1A
:10008800C2B105D06950D8A4C2A5000C0A0CD0C0D2
:10009800D9FFD1C0DAFFDF6A20EE01F0D051D926AE
:1000A800D151DA22B6C0DFFF20EE01F0D051D926B7
:1000B800D151DA22DF505DEC45F00001C26FC2B1C8
:1000C800030C695002E0C2B50A0CC96BCA6BCB6B52
:1000D800CC6BD0C044F0D1C045F0466A476A486A44
:1000E800496A9DEC3EF00001CF6FCF0501E0D4D006
:1000F800CD6BCE6BCE5105E1040ECD5D01E390D002
:1001080001D08ED0CDC080F0CEC081F0803B813B45
:10011800F00E811780510F0B8113F00E8017D0C09D
:1001280082F0D1C083F08051822781518323EC0E65
:100138008225C36F010E8321C46F20EE04F0C351E2
:10014800D926C451DA22DF5005E1A86BA96BAA6B46
:10015800AB6B55D020EE09F0C351D926C451DA2231
:10016800DF50816F806B20EE0AF0C351D926C4514D
:10017800DA22DF50826F82C083F0846B856B866BD6
:1001880084C086F083C085F0846B836B20EE0BF00F
:10019800C351D926C451DA22DF50876F87C088F04F
:1001A800896B8A6B8B6B88C08BF08A6B896B886BC9
:1001B800835188118C6F845189118D6F85518A11F3
:1001C8008E6F86518B118F6F80518C11906F81517A
:1001D8008D11916F000E8E11926F000E8F11936F1B
:1001E80020EE08F0C351D926C451DA22DF5090110D
:1001F800A86F9151A96F9251AA6F9351AB6FCD51CE
:10020800040DF350980FD96EDA6AA8C0DEFFA9C0B2
:10021800DEFFAAC0DEFFABC0DEFFCD4BCE2B6AD718
:10022800CD6BCE6BCD51CE1103E0CD07D8A0CE0754
:10023800CD51040DF350980FD96EDA6ADECFC9F0AC
:10024800DECFCAF0DECFCBF0DECFCCF0C951CA1179
:10025800CB11CC1105E1000EAD6F020EAC6F11D0C1
:10026800D0C044F0D1C045F0C9C046F0CAC047F07C
:10027800CBC048F0CCC049F09DEC3EF00001AC6F1B
:10028800AD6BACC0CFF0CF5107E0CD4BCE2BCE51EC
:1002980003E1040ECD5DCCE3030ECF1901E1010C9F
:1002A800CF5101E00D0C20EE3AF0D051D926D151B2
:1002B800DA22DF50816F806B20EE39F0D051D926D9
:1002C800D151DA22DF508013020E8119801101E02A
:1002D8000D0C20EE45F0D051D926D151DA22DF504D
:1002E800816F806B20EE44F0D051D926D151DA22AB
:1002F800DF50801380C0C5F081C0C6F0C76BC86BE3
:10030800C551C611C711C81155E120EE53F0D0519F
:10031800D926D151DA22DF50816F806B20EE54F05C
:10032800D051D926D151DA22DF50826F82C083F0B2
:10033800846B856B866B84C086F083C085F0846B84
:10034800836B20EE55F0D051D926D151DA22DF50F7
:10035800876F87C088F0896B8A6B8B6B88C08BF03E
:100368008A6B896B886B835188118C6F84518911D2
:100378008D6F85518A118E6F86518B118F6F8051C9
:100388008C11906F81518D11916F000E8E11926FAB
:10039800000E8F11936F20EE52F0D051D926D15113
:1003A800DA22DF509011C56F9151C66F9251C76F15
:1003B8009351C86F20EE16F0D051D926D151DA22C8
:1003C800C5C0DEFFC6C0DEFFC7C0DEFFC8C0DEFF97
:1003D80020EE3EF0D051D926D151DA2210EE03F0AA
:1003E800D051E126D151E222DFCFE7FF20EE03F022
:1003F800D051D926D151DA22DE040AE020EE03F0EA
:10040800D051D926D151DA22020EDE1801E00D0CA6
:10041800C5C00BF0C6C00CF0C7C00DF0C8C00EF0C8
:1004280020EE03F0D051D926D151DA22DF500F6ED9
:10043800106A116A126ABEEC52F00BC0C5F00CC00B
:10044800C6F00DC0C7F00EC0C8F020EE3BF0D0518A
:10045800D926D151DA2210EE02F0D051E126D1513D
:10046800E222DFCFE7FF20EE02F0D051D926D151AA
:10047800DA22DF50D8B40D0C20EE02F0D051D92684
:10048800D151DA22DF50806F20EE02F0D051D92608
:10049800D151DA22DF50816F8105801501E00D0C02
:1004A80020EE40F0D051D926D151DA22DF50816FA9
:1004B800806B20EE3FF0D051D926D151DA22DF509F
:1004C800801320EE08F0D051D926D151DA2280C00D
:1004D800DEFF81C0DDFF20EE08F0D051D926D151D2
:1004E800DA22DF50806F0F0E801701E00D0C20EE2E
:1004F80042F0D051D926D151DA22DF50816F806B7A
:1005080020EE41F0D051D926D151DA22DF508013A4
:1005180080C0BAF081C0BBF0BC6BBD6BBA51BB11D7
:10052800BC11BD1155E120EE4FF0D051D926D15163
:10053800DA22DF50816F806B20EE50F0D051D9263F
:10054800D151DA22DF50826F82C083F0846B856BD1
:10055800866B84C086F083C085F0846B836B20EE45
:1005680051F0D051D926D151DA22DF50876F87C098
:1005780088F0896B8A6B8B6B88C08BF08A6B896B70
:10058800886B835188118C6F845189118D6F8551C7
:100598008A118E6F86518B118F6F80518C11906FDD
:1005A80081518D11916F000E8E11926F000E8F1177
:1005B800936F20EE4EF0D051D926D151DA22DF5078
:1005C8009011BA6F9151BB6F9251BC6F9351BD6F2F
:1005D80020EE3CF0D051D926D151DA22DF50806F7D
:1005E80020EE3DF0D051D926D151DA22DF50816F6B
:1005F8008051B86F81C0B9F0B851B91101E10D0C43
:1006080020EE08F0D051D926D151DA22DECF80F081
:10061800DDCF81F0040E826FD89081338033822F32
:10062800FBD7B8518025836FB9518121846F856BC1
:10063800D8B0852B866BC5518325B26FC6518421EE
:10064800B36FC7518521B46FC8518621B56FB251B8
:10065800BA5DB351BB59B451BC59B551BD5901E24A
:100668000D0CB251BA5D0B6EB351BB590C6EB4513F
:10067800BC590D6EB551BD590E6E20EE02F0D05129
:10068800D926D151DA22DF500F6E106A116A126A28
:10069800BCEC53F00BC0BEF00CC0BFF00DC0C0F0F6
:1006A8000EC0C1F00001BE51BF11C011C11101E15E
:1006B8000D0C010ECF6FC151C01105E1F60EBE5DE4
:1006C8000F0EBF5902E3020ECF6FC151C01105E1F1
:1006D800F60EBE5DFF0EBF5902E3030ECF6F020E8A
:1006E800BE25806F000EBF21816F000EC021826F72
:1006F800000EC121836F20EE12F0D051D926D151BE
:10070800DA2280C0DEFF81C0DEFF82C0DEFF83C048
:10071800DEFF20EE1AF0D051D926D151DA22C9C015
:10072800DEFFCAC0DEFFCBC0DEFFCCC0DEFFB851A3
:10073800C925806FB951CA21816F000ECB21826F04
:10074800000ECC21836F20EE1EF0D051D926D15156
:10075800DA2280C0DEFF81C0DEFF82C0DEFF83C0F8
:10076800DEFFB251C925806FB351CA21816FB451E0
:10077800CB21826FB551CC21836F20EE26F0D0516A
:10078800D926D151DA2280C0DEFF81C0DEFF82C0C7
:10079800DEFF83C0DEFF030ECF1901E08CD020EE10
:1007A80008F0D051D926D151DA22DE50DE1001E00E
:1007B8000D0C20EE5BF0D051D926D151DA22DF5052
:1007C800816F806B20EE5CF0D051D926D151DA22AE
:1007D800DF50826F82C083F0846B856B866B84C028
:1007E80086F083C085F0846B836B20EE5DF0D0517A
:1007F800D926D151DA22DF50876F87C088F0896BFC
:100808008A6B8B6B88C08BF08A6B896B886B835182
:1008180088118C6F845189118D6F85518A118E6F63
:1008280086518B118F6F80518C11906F81518D1172
:10083800916F000E8E11926F000E8F11936F20EE44
:100848005AF0D051D926D151DA22DF509011946F45
:100858009151956F9251966F9351976F20EE22F0B8
:10086800D051D926D151DA2294C0DEFF95C0DEFFDF
:1008780096C0DEFF97C0DEFF20EE12F0D051D926D9
:10088800D151DA22DECF80F0DECF81F0DECF82F0E8
:10089800DECF83F0020ED8908037813782378337D6
:1008A800E82EF9D780C0AEF081C0AFF082C0B0F0BA
:1008B80083C0B1F0B7D020EE08F0D051D926D1517D
:1008C800DA22DE50DE1001E10D0C20EE1EF0D051D0
:1008D800D926D151DA22DECF80F0DECF81F0DECF0B
:1008E80082F0DECF83F0C5518025846FC651812107
:1008F800856FC7518221866FC8518321876F20EE8B
:1009080022F0D051D926D151DA2284C0DEFF85C029
:10091800DEFF86C0DEFF87C0DEFF020ECF196BE068
:1009280020EE12F0D051D926D151DA22DECF80F054
:10093800DECF81F0DECF82F0DECF83F0010E8015AE
:10094800846F856B866B876B20EE12F0D051D926A9
:10095800D151DA22DECF88F0DECF89F0DECF8AF0FF
:10096800DECF8BF0030E8803F3CF8CF0F4CF8DF03D
:100978008E6B8F6B8903F3508D27F4508E23000EF6
:100988008F238803F3508D27F4508E23000E8F2376
:10099800030E8A03F3508E27F4508F23000E890329
:1009A800F3508E27F4508F23000E8803F3508E27C0
:1009B800F4508F23030E8B03F3508F27000E8A0306
:1009C800F3508F27000E8903F3508F27000E8803FA
:1009D800F3508F27D8908F338E338D338C338451D7
:1009E8008C25AE6F85518D21AF6F86518E21B06FEA
:1009F80087518F2116D020EE12F0D051D926D1512F
:100A0800DA22DECF80F0DECF81F0DECF82F0DECFDB
:100A180083F0D8908035AE6F8135AF6F8235B06F77
:100A28008335B16FFF0EAE25806F010EAF21816F48
:100A3800000EB021826F000EB121836F0A0E05D01F
:100A4800D8908333823381338033E82EF9D720EE70
:100A580016F0D051D926D151DA228051DE5C81516D
:100A6800DE588251DE588351DE5801E20D0C20EE2B
:100A78000EF0D051D926D151DA22DE68DE68DE6860
:100A8800DD68DD52DD5210EE0AF0D051E126D15179
:100A9800E222DECFE6FFDECFE6FFDECFE6FFDECFE7
:100AA800E6FF20EE05F0D051D926D151DA22800E8A
:100AB800DF6E030ECF1901E0D3D120EE5FF0D051E5
:100AC800D926D151DA22DF50816F806B20EE5EF09B
:100AD800D051D926D151DA22DF50801380058111F7
:100AE80001E0BED1D0C039F0D1C03AF0C9293B6E7F
:100AF800000ECA213C6E000ECB213D6E000ECC21AB
:100B08003E6EC3EC50F0000901E0AAD1000120EECE
:100B180005F0D051D926D151DA22DF6A22EE2DF024
:100B2800D051D926D151DA22DF50816F806B22EE65
:100B38002CF0D051D926D151DA22DF508013550E2E
:100B4800801903E1AA0E8119D8A48AD120EE2FF0CA
:100B5800D051D926D151DA22DF50816F806B20EE37
:100B680030F0D051D926D151DA22DF50826F82C0BD
:100B780083F0846B856B866B84C086F083C085F0B8
:100B8800846B836B20EE31F0D051D926D151DA2213
:100B9800DF50876F87C088F0896B8A6B8B6B88C042
:100BA8008BF08A6B896B886B835188118C6F8451A9
:100BB80089118D6F85518A118E6F86518B118F6FB8
:100BC80080518C11906F81518D11916F000E8E1193
:100BD800926F000E8F11936F20EE2EF0D051D92610
:100BE800D151DA22DF509011946F9151956F925143
:100BF800966F9351976F520E941909E1520E9519F9
:100C080006E1610E961903E1410E9719D8A428D17F
:100C180022EE13F0D051D926D151DA22DF50816F5C
:100C2800806B22EE14F0D051D926D151DA22DF5050
:100C3800826F82C083F0846B856B866B84C086F07C
:100C480083C085F0846B836B22EE15F0D051D926D2
:100C5800D151DA22DF50876F87C088F0896B8A6BA1
:100C68008B6B88C08BF08A6B896B886B835188117A
:100C78008C6F845189118D6F85518A118E6F8651C1
:100C88008B118F6F80518C11906F81518D11916FE5
:100C9800000E8E11926F000E8F11936F22EE12F0DC
:100CA800D051D926D151DA22DF509011946F915149
:100CB800956F9251966F9351976F720E941909E13F
:100CC800720E951906E1410E961903E1610E971906
:100CD800D8A4C6D022EE17F0D051D926D151DA22A5
:100CE800DF50816F806B22EE18F0D051D926D15198
:100CF800DA22DF50826F82C083F0846B856B866B4B
:100D080084C086F083C085F0846B836B22EE19F073
:100D1800D051D926D151DA22DF50876F87C088F0A9
:100D2800896B8A6B8B6B88C08BF08A6B896B886B3D
:100D3800835188118C6F845189118D6F85518A1167
:100D48008E6F86518B118F6F80518C11906F8151EE
:100D58008D11916F000E8E11926F000E8F11936F8F
:100D680022EE16F0D051D926D151DA22DF50901157
:100D7800946F9151956F9251966F9351976F20EEA2
:100D88000EF0D051D926D151DA2294C0DEFF95C099
:100D9800DEFF96C0DEFF97C0DEFF22EE1BF0D051CB
:100DA800D926D151DA22DF50816F806B22EE1CF0F8
:100DB800D051D926D151DA22DF50826F82C083F018
:100DC800846B856B866B84C086F083C085F0846BEA
:100DD800836B22EE1DF0D051D926D151DA22DF5093
:100DE800876F87C088F0896B8A6B8B6B88C08BF0A4
:100DF8008A6B896B886B835188118C6F8451891138
:100E08008D6F85518A118E6F86518B118F6F80512E
:100E18008C11906F81518D11916F000E8E11926F10
:100E2800000E8F11936F22EE1AF0D051D926D151AE
:100E3800DA22DF509011946F9151956F9251966F0D
:100E48009351976F20EE0AF0D051D926D151DA226A
:100E580094C0DEFF95C0DEFF96C0DEFF97C0DEFFC0
:100E6800D0C0D9FFD1C0DAFFCFC0DFFF01018A4B64
:100E78008B2B000120EE06F0D051D926D151DA2271
:100E88008AC1DEFF8BC1DDFF000C0C6A0B6A5CECCB
:100E98005AF00F0B0101FD6F966B070E966E010E4F
:100EA800FE6FA06B0F0EC16E926893689468948E63
:100EB800929092928982020EFC6FADEC59F0929456
:100EC800898492988998929E899E95689368D10E94
:100ED8000001806FF40E816FA60E826FFF0E836F84
:100EE800D20E846FFE0E856F2B0E866FFF0E876FF6
:100EF8007DEC5AF043EC5AF017D0780E0001806F61
:100F0800FE0E816F82CF82F0836B7DEC5AF0150E56
:100F18000001FA6F4B0EF96FBE0EE82EFED7F92FBF
:100F2800FCD7FA2FFAD700F082B2E7D7F8EC4AF0EC
:100F38000101FD6F2A0E0001806FFB0E816FFDC15C
:100F480082F0836B7DEC5AF00400150E0001FA6FF5
:100F58004B0EF96FBE0EE82EFED7F92FFCD7FA2FED
:100F6800FAD700F0F286F180F288F19CF28E57EC05
:100F780056F08992899457EC4DF057EC4DF0000EDD
:100F88000B6E340E27EC57F04F0E0F6EFF0E106EDF
:100F980043EC53F0A60E0F6EFF0E106E43EC53F0A9
:100FA800000E0B6E390E27EC57F0898004008CEC8C
:100FB80035F0AFEC42F0F7EC53F0000E0B6E800EFC
:100FC80027EC57F00101FD510F0D740EF3240F6E3D
:100FD8000C0EF420106E43EC53F0725001E1EAD08D
:100FE8004A0E0001806FFD0E816F7DEC5AF014EC03
:100FF80055F00FC0E3F110C0E4F111C0E5F112C0E3
:10100800E6F10101E351E411E511E61117E1880E5B
:101018000001806FFB0E816FE3C182F0E4C183F0B1
:10102800E5C184F0E6C185F07DEC5AF00A0E0E6E3B
:10103800000E0F6A106A116AD5EC56F00101E76BD1
:10104800E86BE8BF05D0E85119E1040EE75D16E248
:10105800DB0E0001806FFF0E816FE30E0101E725B3
:10106800D96E010EE821DA6EDF500001826F836BC2
:101078007DEC5AF00101E74BE82BE3D7490E00015C
:10108800806FFC0E816F7DEC5AF02F0E0001806F8F
:10109800FA0E816F7DEC5AF022EE00F000EECAF0F5
:1010A8001F0EDBCFEBFFE806FCE2D30E0001EA6F70
:1010B800FF0EEB6FC7EC36F0CAC078F1CBC079F100
:1010C800CCC07AF1CDC07BF10101785179117A1148
:1010D8007B1170E0150E0001806FFA0E816F78C1E8
:1010E80082F079C183F07AC184F07BC185F07DEC10
:1010F8005AF0000E0001A36F020EA46F78C1FAF037
:1011080079C1FBF07AC1FCF0F96B000EF925A56FE7
:10111800010EFA21A66F000EFB21A76F000EFC211D
:10112800A86F2CEC12F0000E626E020E636E740E45
:10113800646E0A0E656E676A080E666EE00E686E6B
:10114800010E696E16EC15F00101E96BEA6BEABF56
:1011580005D0EA5119E1080EE95D16E2D70E000143
:10116800806FFF0E816F740E0101E925D96E0A0E9A
:10117800EA21DA6EDF500001826F836B7DEC5AF052
:101188000101E94BEA2BE3D72AEE74F0DF50D86F60
:10119800D96BDA6BDB6B400E0001806FFE0E816F3E
:1011A800D8C182F0D9C183F0DAC184F0DBC185F0FF
:1011B8007DEC5AF00101A0AF13D09468899289821E
:1011C800150E0001FA6F4B0EF96FBE0EE82EFED712
:1011D800F92FFCD7FA2FFAD700F0ABEC43F0EED793
:1011E800FE5104E0020E9A6F2D0E0BD05A0E00012C
:1011F800806FFD0E816F7DEC5AF0010E01019A6F30
:10120800040E996FDC6BDD6BEE6B899E000EED6F43
:10121800010EEC6FEDBF05D0ED5162E1040EEC5DFF
:101228005FE20F0EEC03F3CFF9F0F4CFFAF0ED0321
:10123800F3500001FA27640EF9250B6E0D0EFA2102
:101248000C6EAFEC57F00C5003E1030E0B5C44E35B
:10125800B90E0001806FFD0E816F0F0E0101EC03C6
:10126800F3CFF9F0F4CFFAF0ED03F3500001FA27C9
:10127800640EF925826F0D0EFA21836F7DEC5AF00A
:10128800ECC1F9F0EDC1FAF0050ED8900001F9377C
:10129800FA37E82EFAD7000EF925D26F020EFA2196
:1012A800D36F0F0E0101EC03F3CFFBF0F4CFFCF08A
:1012B800ED03F3500001FC27640EFB25D46F0D0EDF
:1012C800FC21D56F030ED66FCBEC17F00101DE6F52
:1012D800DF6BDE51FEEC56F00101EC4BED2B9AD79B
:1012E800899E000E0B6EC00E27EC57F0EAEC59F001
:1012F800000E0B6EC00E27EC57F0940E0F6EFF0E0B
:10130800106E43EC53F01FD181A89394B6EC5AF0B9
:101318000B500C1001E1EED0EEC1E2F1EB0E0B6EBA
:10132800010E0C6E35EC52F00101EE6FEBB9EE9F39
:10133800350EEE1907E1490E0001806FFC0E816F32
:101348007DEC5AF0340E0001806FFF0E816FEEC104
:1013580082F0836B010E80A0000E846F856B7DEC9C
:101368005AF00101EBA935D0600EEE1932E15F0E9B
:10137800E2192FE1AA0E0001806FF80E816FEEC10D
:1013880082F0836BE2C184F0856B010E81A2000EAE
:10139800866F876B010E81A4000E886F896B7DECC8
:1013A8005AF00101FC832AEE74F09AC1DFFF2AEE9D
:1013B80075F099C1DFFF8984496A020E486E8EEC88
:1013C8003DF08994FC93716A1BEC5AF00101EE6BB5
:1013D800BAD0FE5144E0EB51100B0001A86F000E8B
:1013E800A96F0101EE5145EC3AF0A8C0EFF1A9C090
:1013F800F0F1080E0101EF19F01101E100F0070EFC
:101408000101EF19F01102E180EC53F00101EF0541
:10141800F01102E1C4EC4DF0020EEF19F01102E1F7
:10142800AFEC40F0030EEF19F01106E18BEC1CF065
:10143800E1C0DCF1E2C0DDF1050E0101EF19F011A8
:1014480006E112EC30F0EAC0DCF1EBC0DDF1090E88
:101458000101EF19F01177E173EC50F074D0EB5102
:10146800100B486E000E496EEE512FEC27F048C065
:10147800EFF149C0F0F1070E0101EF19F01102E197
:1014880031EC54F0020EEF19F01102E179EC55F04D
:10149800EF05F01102E11EEC39F0030EEF19F0111F
:1014A80002E198EC44F0040EEF19F01102E14BEC64
:1014B80058F0050EEF19F01102E1F5EC37F0060EC1
:1014C8000101EF19F01102E168EC5AF0080EEF196A
:1014D800F01102E1DDEC2CF0090EEF19F01102E138
:1014E8007FEC3CF00A0E0101EF19F0112CE1FBEC46
:1014F8004BF029D0F8EC4AF00101966F975123E0A0
:10150800FD51961920E0898E000E0B6EC00E27EC57
:1015180057F0EAEC59F0000E0B6EC00E27EC57F0AE
:10152800F60E0F6EFE0E106E43EC53F096C1FDF1F1
:10153800380E0001806FFC0E816FFDC182F0836B55
:101548007DEC5AF032D082B230D0050E0101DC19A0
:10155800DD112BE0D9D6780E0001806FFE0E816F69
:1015680082CF82F0836B7DEC5AF0150E0001FA6F82
:101578004B0EF96FBE0EE82EFED7F92FFCD7FA2FC7
:10158800FAD700F00400000E0B6EC00E27EC57F0DF
:10159800EAEC59F0000E0B6EC00E27EC57F0570E10
:1015A8000F6EFF0E106E43EC53F082B2D4D7150EB7
:1015B8000001FA6F4B0EF96FBE0EE82EFED7F92F19
:1015C800FCD7FA2FFAD700F0000EAAEC5AF0010166
:1015D800956F4C0E0001806FFC0E816F95C182F0F3
:1015E800836B7DEC5AF0150E0001FA6F4B0EF96F04
:1015F800BE0EE82EFED7F92FFCD7FA2FFAD700F047
:10160800899489920001D26BD36B4B0ED46FFC0E78
:10161800D56FD66B11EC51F0C9D4646E636A37D3B9
:10162800645016E10001FD5113E0E40E806FFB0EDB
:10163800816FCFCF82F0836BCECF84F0856B7DEC4A
:101648005AF0636A0101856B0A0EC5D0899090D360
:10165800020E641814E10001FD5111E05A0E806F6A
:10166800FB0E816FCFCF82F0836BCECF84F0856B7A
:101678007DEC5AF0636A0101856B140EACD01F0E25
:1016880064643FD0300E64603CD00001FD5139E005
:101698006450E00F736EE60E806FF80E816FCFCF47
:1016A80082F0836BCECF84F0856B73C086F0876B36
:1016B8007DEC5AF0636A7350200D0A0EF324D96E3C
:1016C800020EF420DA6EDE50DE10DE10DE1003E0CB
:1016D800030E736443D0010E6B6E7350140D130E1A
:1016E800F324D96E010EF420DA6E7350140D130E24
:1016F800F324E16E010EF420E26EE7500409DF6E78
:101708002DD03F0E64642ED0500E64602BD00001A3
:10171800FD5128E07350140D000EF324D96E010E0C
:10172800F420DA6E6450C00FDF6E300E806FF80E52
:10173800816FCFCF82F0836BCECF84F0856B7350EF
:10174800140D000EF324D96E010EF420DA6EDF506A
:10175800866F876B7DEC5AF0636A6B6A0101846B54
:10176800856B74D7310E641808E10001FD5105E05E
:101778000C0E0101856F1D0E74D2340E641814E12D
:101788000001FD5111E00F0E806FFC0E816FCFCF6D
:1017980082F0836BCECF84F0856B7DEC5AF001012B
:1017A800846B856B636A52D7350E641816E10001A5
:1017B800FD5113E0E10E806FF90E816FCFCF82F0FB
:1017C800836BCECF84F0856B7DEC5AF0636A0D0E87
:1017D8000101856FAC0E846F39D7370E641809E1A3
:1017E8000001FD5106E089800E0E0101856F750E1E
:1017F80038D20D0E641818E10001FD5115E0636A36
:10180800020E0101856FBC0E846F8990AB0E00013A
:10181800806FF90E816FCFCF82F0836BCECF84F0CB
:10182800856B7DEC5AF0A4D2100E641808E1000113
:10183800FD5105E0030E0101856FE90E12D2180E65
:10184800641808E10001FD5105E0070E0101856FEC
:10185800090E07D23B0E641808E10001FD5105E0AE
:101868000E0E0101856F7E0EFCD13E0E641808E154
:101878000001FD5105E00F0E0101856F3D0EF1D10C
:10188800590E0001806FF90E816FCFCF82F0836B04
:10189800CECF84F0856B64C086F0876B7DEC5AF000
:1018A80067D27350140D010EF324D96E010EF42083
:1018B800DA6E64C0DFFF030E0101856FEA0ED1D135
:1018C8007350140D020EF324D96E010EF420DA6E53
:1018D80064C0DFFF030E0101856FEB0EC2D17350A8
:1018E800140D030EF324D96E010EF420DA6E64C0D1
:1018F800DFFF030E0101856FEC0EB3D17350140D99
:10190800040EF324D96E010EF420DA6E64C0DFFFF2
:10191800030E0101856FED0EA4D17350140D050E51
:10192800F324D96E010EF420DA6E64C0DFFF030ED3
:101938000101856FEE0E95D17350140D060EF32438
:10194800D96E010EF420DA6E64C0DFFF7350140DF7
:10195800060EF324D96E010EF420DA6EDF50486EBD
:1019680048C049F04A6A4B6A4C6A4BC04CF04AC0BE
:101978004BF049C04AF0496A7350140D050EF32420
:10198800D96E010EF420DA6EDF504D6E4DC04EF068
:101998004F6A506A516A4FC051F04EC050F04F6ABA
:1019A8004E6A7350140D040EF324D96E010EF42000
:1019B800DA6EDF50526E52C053F0546A556A566A56
:1019C80053C056F0556A546A536A7350140D030E87
:1019D800F324D96E010EF420DA6EDF505324576ECB
:1019E800000E5420586E000E5520596E000E5620D9
:1019F8005A6E4E5057245B6E4F5058205C6E5050B4
:101A080059205D6E51505A205E6E49505B245F6EBE
:101A18004A505C20606E4B505D20616E4C505E20D9
:101A2800626E7350140D070EF324D96E010EF42064
:101A3800DA6E5FC0DEFF60C0DEFF61C0DEFF62C03D
:101A4800DEFF4E0E0001806FF70E816FCFCF82F060
:101A5800836BCECF84F0856B7350140D070EF3247F
:101A6800D96E010EF420DA6EDECF86F0DECF87F075
:101A7800DECF88F0DECF89F07DEC5AF00101846B6F
:101A8800856B76D17350140D120EF324D96E010EA6
:101A9800F420DA6E64C0DFFF070E0101856F0A0EBD
:101AA800E0D07350140D110EF324D96E010EF420FA
:101AB800DA6E64C0DFFF070E0101856F0B0ED1D00F
:101AC8007350140D100EF324D96E010EF420DA6E43
:101AD80064C0DFFF070E0101856F0C0EC2D0735082
:101AE800140D0F0EF324D96E010EF420DA6E64C0C3
:101AF800DFFFF00E0001806FF70E816FCFCF82F00D
:101B0800836BCECF84F0856B7350140D0F0EF324C6
:101B1800D96E010EF420DA6EDECF86F0DECF87F0C4
:101B2800DECF88F0DECF89F07DEC5AF0A7D701012F
:101B3800846B856BD00E0001806FF70E816FCFCF5D
:101B480082F0836BCECF84F0856B64C086F0876BA0
:101B58007DEC5AF06B6A7AD564C06CF10F0E010106
:101B6800856F3E0E7ED064C06DF10F0E0101856F4A
:101B78003F0E77D064C06EF10F0E0101856F400EE5
:101B880070D064C06FF10F0E0101856F410E69D0EE
:101B980064C070F10F0E0101856F420E62D064C0FF
:101BA80071F10F0E0101856F430E5BD064C072F1B5
:101BB8000F0E0101856F440E54D064C073F1660E98
:101BC8000001806FF40E816FCFCF82F0836BCECF90
:101BD80084F0856B6CC186F0876B6DC188F0896B6A
:101BE8006EC18AF08B6B6FC18CF08D6B70C18EF0FB
:101BF8008F6B71C190F0916B72C192F0936B73C14E
:101C080094F0956B7DEC5AF039D70F0E0001806F78
:101C1800FC0E816FCFCF82F0836BCECF84F0856BC3
:101C28007DEC5AF02BD70C0E0101856F1E0E19D0D2
:101C38004F0E0001806FF80E816FCFCF82F0836B5B
:101C4800CECF84F0856B7DEC5AF00C0E0101856FC8
:101C58001C0E846F0A0E636EF9D40E0E0101856F97
:101C6800760E846F85D0900E0001806FF90E816F1B
:101C7800CFCF82F0836BCECF84F0856B7DEC5AF0AA
:101C88000101846B856B090E636E898071D084C1F4
:101C980048F085C149F0495011E0030A13E0040AED
:101CA80025E00B0A31E0010A35E0030A39E0010AB0
:101CB80040E0130A58E03B0A59E05AD0485001E185
:101CC800AFD456D04850E90A01E1EBD5030A01E147
:101CD800F7D5010A01E103D6070A01E10FD6010A87
:101CE80001E11BD6030A01E127D642D04850090A70
:101CF80001E1C8D6030A01E1D4D6010A01E1E0D620
:101D0800070A01E1ECD634D048501D0A8CE0030ADA
:101D18008FE02ED04850480A01E177D7E40A28D04E
:101D28004850750A9AE0030A9EE0080A01E1FFD6C6
:101D38001FD048503D0A01E10FD7030A01E113D72C
:101D4800010A01E117D77F0A01E11BD7010A01E166
:101D58001FD7030A01E123D7010A01E127D7070AA0
:101D680001E12BD705D048502A0A02D048500F0A63
:101D780063501200A5C0B7F0A6C0B8F0A951D96E3B
:101D8800DA6ADE6ADD6AA3C00CF0A4C00DF0EEECDE
:101D980051F00001B66FB65102E0B651120020EEC4
:101DA80005F0A351D926A451DA22DF5008E020EE2D
:101DB80005F0A351D926A451DA22DF50120020EEF3
:101DC80004F0A351D926A451DA22DFA2070C20EE91
:101DD80006F0A351D926A451DA2210EE06F0A35139
:101DE800E126A451E222E6CFAEF0E6CFAFF0E6CF8F
:101DF800B0F0E6CFB1F0A751AE25B26FA851AF2130
:101E0800B36F000EB021B46F000EB121B56FDE5074
:101E1800B25DDE50B359DE50B459DE50B55901E316
:101E2800E1D2A76BA86BDED220EE06F0A351D9262B
:101E3800A451DA22FF0EDE14AA6F010EDE14AB6F76
:101E4800000EDE14AC6F000EDE14AD6FAA51AB119C
:101E5800AC11AD1101E032D220EE06F0A351D92623
:101E6800A451DA22DECFAAF0DECFABF0DECFACF0A1
:101E7800DECFADF00A0E05D0D890AD33AC33AB331E
:101E8800AA33E82EF9D7A3C0D9FFA4C0DAFF10EE11
:101E980002F0DE50E126DD50E222E750AE6FAE05DB
:101EA800AA15B96FB95101E099D020EE06F0A351F7
:101EB800D926A451DA22DE50DE10DE10DE1022E12F
:101EC80020EE0EF0A351D926A451DA22DECFC0F0BD
:101ED800DECFC1F0DECFC2F0DECFC3F0C051C111FA
:101EE800C211C3112FE1A3C0D9FFA4C0DAFFDECF0E
:101EF8008CF0DDCF8DF08E6B8F6B906B916BE2EC7D
:101F080032F018D0A3C0D9FFA4C0DAFFDECF8CF01E
:101F1800DDCF8DF020EE12F0A351D926A451DA229C
:101F2800DECF8EF0DECF8FF0DECF90F0DECF91F0F7
:101F3800E2EC32F08CC0C0F08DC0C1F08EC0C2F0AF
:101F48008FC0C3F0C051C111C211C31101E14ED2FB
:101F5800C005C111C211C31109E120EE05F0A3515A
:101F6800D926A451DA22020EDF6E020CC0290FE135
:101F7800C1290DE1C2290BE1C32909E120EE05F0D1
:101F8800A351D926A451DA22010EDF6E010C20EEEE
:101F980012F0A351D926A451DA22C0C0DEFFC1C075
:101FA800DEFFC2C0DEFFC3C0DEFF20EE0EF0A3518D
:101FB800D926A451DA22DE50DE10DE10DE100EE142
:101FC80020EE0EF0A351D926A451DA22C0C0DEFFBC
:101FD800C1C0DEFFC2C0DEFFC3C0DEFF20EE16F0C8
:101FE800A351D926A451DA22A3C0E1FFA4C0E2FF7D
:101FF80000EE2AF0E650E926E550EA22DE50EE1817
:1020080016E1DE50EE1813E1DE50EE1810E1DE5056
:10201800EE180DE1A3C0D9FFA4C0DAFFDECF24F08B
:10202800DDCF25F07AEC47F0000901E083D1A3C0A9
:10203800D9FFA4C0DAFFDECF0BF0DDCF0CF0000132
:1020480020EE12F0A351D926A451DA22DECF0DF0EA
:10205800DECF0EF0DECF0FF0DECF10F071EC4AF0DD
:102068000BC0BCF00CC0BDF00DC0BEF00EC0BFF080
:102078000001BC51BD11BE11BF1101E16ED7B951AC
:10208800BC27000EBD23BE23BF23A7C0AAF0A8C04B
:10209800ABF0090EAC6FD890AB33AA33AC2FFBD79B
:1020A800AAC0BAF0ABC0BBF0BA51BB1101E1C3D0B2
:1020B800B951BA25AA6F000EBB21AB6FA3C0D9FFD7
:1020C800A4C0DAFF10EE02F0DE50E126DD50E22275
:1020D800E750AC6FAD6BAA51AC5DAB51AD5912E294
:1020E800A3C0D9FFA4C0DAFF10EE02F0DE50E1264B
:1020F800DD50E222E750AA6FB951AA5DBA6FBB6BF7
:10210800D8A0BB07B7C01AF0B8C01BF0BCC01CF001
:10211800BDC01DF0BEC01EF0BFC01FF0BAC020F089
:10212800BBC021F0A3C0D9FFA4C0DAFF10EE01F0B4
:10213800DE50E126DD50E222E75075EC4CF0000954
:1021480001E0F8D00001BA51AA6FBB51AB6FAC6B7C
:10215800AD6BA3C0D9FFA4C0DAFF10EE2AF0DE50A1
:10216800E126DD50E222E6CFAEF0E6CFAFF0E6CFD3
:10217800B0F0E6CFB1F0BC51AE5DB26FBD51AF5912
:10218800B36FBE51B059B46FBF51B159B56FAA51B1
:10219800B25DAB51B359AC51B459AD51B5593CE2EC
:1021A800A3C0D9FFA4C0DAFFDECFAAF0DDCFABF021
:1021B8002E0EAA250B6E000EAB210C6EA3C0D9FF04
:1021C800A4C0DAFF10EE2AF0DE50E126DD50E2224C
:1021D800E6CFACF0E5CFADF0BC51AC5FBD51AD5B27
:1021E800090ED890AC37AD37E82EFBD7AC51B725E0
:1021F8000D6EAD51B8210E6E020E106E0F6AF0EC26
:1022080057F0A3C0D9FFA4C0DAFF10EE04F0DE50E7
:10221800E126DD50E222E76ABAC0AAF0BBC0ABF003
:10222800090ED890AA37AB37E82EFBD7AAC0C4F05E
:10223800ABC0C5F0BBD020EE0AF0A351D926A451FB
:10224800DA2210EE06F0A351E126A451E222DE5074
:10225800E65CDE50E658DE50E658DE50E6581FE3EE
:10226800A3C0D9FFA4C0DAFFDECF24F0DDCF25F06C
:102278007AEC47F0000901E05DD0A3C0D9FFA4C003
:10228800DAFF10EE2AF0DE50E126DD50E222BCC073
:10229800E6FFBDC0E6FFBEC0E6FFBFC0E6FF000127
:1022A80020EE16F0A351D926A451DA22BCC0DEFFD5
:1022B800BDC0DEFFBEC0DEFFBFC0DEFFAA69010EE3
:1022C800AB6F20EE06F0A351D926A451DA22DECF57
:1022D800ACF0DDCFADF0AA51AC17AB51AD17AC5196
:1022E8000008C46FAD51D8A0E82A0208C56FC451D0
:1022F800A75DC551A85904E2A7C0C4F0A8C0C5F09D
:10230800A3C0D9FFA4C0DAFFDECF39F0DDCF3AF0A1
:1023180020EE16F0A351D926A451DA22DECF3BF0E5
:10232800DECF3CF0DECF3DF0DECF3EF0C3EC50F028
:10233800000902E0000122D60001AA69010EAB6F74
:1023480020EE06F0A351D926A451DA22DECFACF054
:10235800DDCFADF0AA51AC17AB51AD17A3C0D9FF73
:10236800A4C0DAFFDECFAEF0DDCFAFF0AC51AE27C0
:10237800AD51AF232E0EAE250B6E000EAF210C6EA5
:10238800B7C00DF0B8C00EF0C4C00FF0C5C010F053
:10239800F0EC57F0A3C0D9FFA4C0DAFF10EE04F0A8
:1023A800DE50E126DD50E222010EE76EC451B72768
:1023B800C551B82320EE06F0A351D926A451DA223C
:1023C800C451DE26C551DE22000EDE22DE22A951CE
:1023D800D96EDA6AC451DE26C551DD22C451A75F21
:1023E800C551A85BA751A81101E01ED520EE06F043
:1023F800A351D926A451DA2210EE0AF0A351E126FE
:10240800A451E222DE50E65CDE50E658DE50E65883
:10241800DE50E65814E220EE06F0A351D926A45166
:10242800DA2210EE0AF0A351E126A451E222DECF0F
:10243800E6FFDECFE6FFDECFE6FFDECFE6FF20EEEB
:1024480004F0A351D926A451DA22000EDB8A000C2D
:10245800A3C00CF0A4C00DF0EEEC51F00001BD6F6C
:10246800BD5102E0BD51120020EE05F0A351D9265E
:10247800A451DA22DF5008E020EE05F0A351D92656
:10248800A451DA22DF50120020EE0AF0A351D92617
:10249800A451DA22A551DE5CA651DE58A751DE58B8
:1024A800A851DE5816E220EE04F0A351D926A45113
:1024B800DA22DFB20ED020EE0AF0A351D926A451B9
:1024C800DA22DECFA5F0DECFA6F0DECFA7F0DECF92
:1024D800A8F020EE06F0A351D926A451DA22DECFC7
:1024E800B9F0DECFBAF0DECFBBF0DECFBCF0BE6B0A
:1024F800BF6BC06BC16B20EE06F0A351D926A45167
:10250800DA22BEC0DEFFBFC0DEFFC0C0DEFFC1C032
:10251800DEFFA551A611A711A81101E119D2A3C088
:10252800D9FFA4C0DAFF10EE02F0DE50E126DD503C
:10253800E222E750A96FA9C0AAF0AB6BAC6BAD6BF8
:10254800090ED890AA37AB37AC37AD37E82EF9D794
:10255800AAC0C2F0ABC0C3F0ACC0C4F0ADC0C5F0F7
:10256800B951BA11BB11BC1101E196D0FF0EA525D6
:102578000B6EFF0EA6210C6EFF0EA7210D6EFF0E2F
:10258800A8210E6EC2C00FF0C3C010F0C4C011F075
:10259800C5C012F0BCEC53F00BC0A9F00CC0AAF0F7
:1025A8000DC0ABF00EC0ACF0FF0E0001B9250B6EEC
:1025B800FF0EBA210C6EFF0EBB210D6EFF0EBC2163
:1025C8000E6EC2C00FF0C3C010F0C4C011F0C5C079
:1025D80012F0BCEC53F00B500001A95D0C50AA5945
:1025E8000D50AB590E50AC5957E3FF0EC225A96FD9
:1025F800FF0EC321AA6FFF0EC421AB6FFF0EC521CA
:10260800AC6FA91DAD6FAA1DAE6FAB1DAF6FAC1D32
:10261800B06FFF0EB925B16FFF0EBA21B26FFF0E72
:10262800BB21B36FFF0EBC21B46FAD51B115B56FAF
:10263800AE51B215B66FAF51B315B76FB051B415EF
:10264800B86F20EE06F0A351D926A451DA22B5C0FE
:10265800DEFFB6C0DEFFB7C0DEFFB8C0DEFF20EE8B
:1026680006F0A351D926A451DA22DE50A55FDE5028
:10267800A65BDE50A75BDD50A85B20EE12F0A351ED
:10268800D926A451DA22DECFC6F0DECFC7F0DECFDE
:10269800C8F0DECFC9F064D020EE0EF0A351D926E1
:1026A800A451DA22DECFC6F0DECFC7F0DECFC8F005
:1026B800DECFC9F0C651C711C811C91143E1A3C083
:1026C800D9FFA4C0DAFFDECF8CF0DDCF8DF08E6BA2
:1026D8008F6B906B916BE2EC32F08CC0C6F08DC0C2
:1026E800C7F08EC0C8F08FC0C9F0C605C711C811A1
:1026F800C91109E120EE05F0A351D926A451DA2227
:10270800020EDF6E020CC6290FE1C7290DE1C829A8
:102718000BE1C92909E120EE05F0A351D926A451FE
:10272800DA22010EDF6E010C20EE0EF0A351D9263D
:10273800A451DA22C6C0DEFFC7C0DEFFC8C0DEFF74
:10274800C9C0DEFF20EE12F0A351D926A451DA2227
:10275800C6C0DEFFC7C0DEFFC8C0DEFFC9C0DEFFDF
:10276800C651C711C811C91101E095D0F1D020EEAA
:1027780004F0A351D926A451DA22DFA228D0A3C09D
:10278800D9FFA4C0DAFFDECF8CF0DDCF8DF0C6C054
:102798008EF0C7C08FF0C8C090F0C9C091F0E2ECCD
:1027A80032F08CC0C6F08DC0C7F08EC0C8F08FC0A4
:1027B800C9F0C651C711C811C91123E1C2C0A5F09B
:1027C800C3C0A6F0C4C0A7F0C5C0A8F06ED0A3C00F
:1027D800D9FFA4C0DAFFDECF44F0DDCF45F0C6C094
:1027E80046F0C7C047F0C8C048F0C9C049F0E7EC98
:1027F8001EF044C0C6F045C0C7F046C0C8F047C088
:10280800C9F00001C62907E1C72905E1C82903E184
:10281800C92901E180D7C951C811C71104E1020EC5
:10282800C65D01E267D7A3C0D9FFA4C0DAFF10EEE6
:1028380012F0DE50E126DD50E222E650C65DE65099
:10284800C759E650C859E650C95901E353D720EE95
:1028580012F0A351D926A451DA22C6C0DEFFC7C0A0
:10286800DEFFC8C0DEFFC9C0DEFF20EE06F0A351C0
:10287800D926A451DA22C251DE26C351DE22C45120
:10288800DE22C551DE22C251A55FC351A65BC451E9
:10289800A75BC551A85BA551C25DA651C359A751F5
:1028A800C459A851C55901E262D720EE06F0A351D8
:1028B800D926A451DA22A551DE26A651DE22A75137
:1028C800DE22A851DE22A551A96F010EA615AA6F16
:1028D800AB6BAC6BA911AB11AC113AE0A3C0D9FF3B
:1028E800A4C0DAFFDECF0BF0DDCF0CF0C6C00DF0D0
:1028F800C7C00EF0C8C00FF0C9C010F071EC4AF0A4
:102908000BC0BEF00CC0BFF00DC0C0F00EC0C1F0CF
:102918000001BE51BF11C011C11101E1EBD6A5C024
:10292800A9F0A6C0AAF0A7C0ABF0A8C0ACF00A0EE8
:1029380005D0D890AC33AB33AA33A933E82EF9D7F6
:10294800A951BE27AA51BF23AB51C023AC51C12303
:1029580020EE06F0A351D926A451DA22FF0EDE1488
:10296800A96F010EDE14AA6F000EDE14AB6F000E05
:10297800DE14AC6FA951AA11AB11AC1120E020EE06
:1029880016F0A351D926A451DA22BE51DE1809E166
:10299800BF51DE1806E1C051DE1803E1C151DE184F
:1029A8000EE020EE16F0A351D926A451DA22BEC0BB
:1029B800DEFFBFC0DEFFC0C0DEFFC1C0DEFF20EE0D
:1029C80006F0A351D926A451DA2210EE0AF0A35139
:1029D800E126A451E222DE50E65CDE50E658DE50E5
:1029E800E658DE50E65801E33DD520EE06F0A35147
:1029F800D926A451DA2210EE0AF0A351E126A451F7
:102A0800E222DECFE6FFDECFE6FFDECFE6FFDECF57
:102A1800E6FF20EE04F0A351D926A451DA22000ED5
:102A2800DB8A20D564C0A1F065C0A2F068C0D9FFD8
:102A380069C0DAFFDE6ADD6A62C00CF063C00DF0BF
:102A4800EEEC51F000019C6F9C5102E09C51120089
:102A580020EE05F06250D9266350DA22DF5008E0F4
:102A680020EE05F06250D9266350DA22DF501200BA
:102A780020EE04F06250D9266350DA22DFA0070C5A
:102A880020EE06F06250D9266350DA22DECF8CF0B1
:102A9800DECF8DF0DECF8EF0DECF8FF020EE0AF0A5
:102AA8006250D9266350DA22DECF90F0DECF91F063
:102AB800DECF92F0DECF93F08C51905D986F8D5100
:102AC8009159996F8E5192599A6F8F5193599B6F63
:102AD80066508C6F67508D6F8E6B8F6B8C51985DC5
:102AE8008D5199598E519A598F519B5901E34AD268
:102AF80098C066F099C067F045D220EE06F06250A3
:102B0800D9266350DA22FF0EDE148C6F010EDE1414
:102B18008D6F000EDE148E6F000EDE148F6F8C51D9
:102B28008D118E118F1101E0A5D120EE06F06250B3
:102B3800D9266350DA22DECF8CF0DECF8DF0DECFDF
:102B48008EF0DECF8FF00A0E05D0D8908F338E33FB
:102B58008D338C33E82EF9D762C0D9FF63C0DAFF12
:102B680010EE02F0DE50E126DD50E222E750906FD1
:102B780090058C15A36FA3516AE120EE06F0625010
:102B8800D9266350DA22DE50DE10DE10DE100FE1A7
:102B980020EE0EF06250D9266350DA22DECF9DF087
:102BA800DECF9EF0DECF9FF0DECFA0F020D062C057
:102BB800D9FF63C0DAFFDECF44F0DDCF45F020EE69
:102BC80012F06250D9266350DA22DECF46F0DECF0B
:102BD80047F0DECF48F0DECF49F0E7EC1EF044C006
:102BE8009DF045C09EF046C09FF047C0A0F0000190
:102BF800A0519F119E110CE1020E9D5D09E220EE8D
:102C080005F06250D9266350DA22020EDF6E020CFC
:102C18009D290FE19E290DE19F290BE1A02909E1DA
:102C280020EE05F06250D9266350DA22010EDF6EDD
:102C3800010C20EE12F06250D9266350DA229DC0B2
:102C4800DEFF9EC0DEFF9FC0DEFFA0C0DEFF62C0C9
:102C5800D9FF63C0DAFFDECF0BF0DDCF0CF020EE3A
:102C680012F06250D9266350DA22DECF0DF0DECFA3
:102C78000EF0DECF0FF0DECF10F071EC4AF00BC093
:102C8800A4F00CC0A5F00DC0A6F00EC0A7F000017E
:102C9800A451A511A611A71101E1B1D7A351A427E9
:102CA800000EA523A623A72366C08CF067C08DF06D
:102CB800090E8E6FD8908D338C338E2FFBD78CC036
:102CC800A8F08DC0A9F0A851A91101E1C5D0A35160
:102CD800A8258C6F000EA9218D6F62C0D9FF63C033
:102CE800DAFF10EE02F0DE50E126DD50E222E75076
:102CF8008E6F8F6B8C518E5D8D518F5912E262C031
:102D0800D9FF63C0DAFF10EE02F0DE50E126DD5095
:102D1800E222E7508C6FA3518C5DA86FA96BD8A0F5
:102D2800A907A1C01AF0A2C01BF0A4C01CF0A5C03E
:102D38001DF0A6C01EF0A7C01FF0A8C020F0A9C0B3
:102D480021F062C0D9FF63C0DAFF10EE01F0DE5057
:102D5800E126DD50E222E75021EC50F0000901E0C5
:102D68005FD762C0D9FF63C0DAFF10EE04F0DE500F
:102D7800E126DD50E222E7505FE00001A8518C6FA8
:102D8800A9518D6F8E6B8F6B62C0D9FF63C0DAFF5C
:102D980010EE2AF0DE50E126DD50E222E6CF90F078
:102DA800E6CF91F0E6CF92F0E6CF93F0A451905D94
:102DB800946FA5519159956FA6519259966FA75145
:102DC8009359976F8C51945D8D5195598E519659A1
:102DD8008F51975931E262C0D9FF63C0DAFF10EE14
:102DE8002AF0DE50E126DD50E222E6CF8CF0E5CF76
:102DF8008DF0A4518C5FA5518D5B090ED8908C374E
:102E08008D37E82EFBD78C51A1250B6E8D51A22151
:102E18000C6E62C0D9FF63C0DAFFDECF8EF0DDCF63
:102E28008FF02E0E8E250D6E000E8F210E6E020E67
:102E3800106E0F6AF0EC57F0A8C08CF0A9C08DF0A6
:102E4800090ED89000018C378D37E82EFAD78CC040
:102E5800AAF08DC0ABF079D020EE16F06250D926DA
:102E68006350DA22A4C0DEFFA5C0DEFFA6C0DEFFE5
:102E7800A7C0DEFF8C69010E8D6F20EE06F0625050
:102E8800D9266350DA22DECF8EF0DDCF8FF08C5159
:102E98008E178D518F178E510008AA6F8F51D8A0A9
:102EA800E82A0208AB6FAA51665CAB51675804E286
:102EB80066C0AAF067C0ABF062C0D9FF63C0DAFF92
:102EC800DECF39F0DDCF3AF020EE16F06250D92689
:102ED8006350DA22DECF3BF0DECF3CF0DECF3DF0B0
:102EE800DECF3EF0C3EC50F0000901E099D6A1C056
:102EF8000BF0A2C00CF000018C69010E8D6F20EE62
:102F080006F06250D9266350DA22DECF8EF0DDCF8C
:102F18008FF08C518E178D518F1762C0D9FF63C007
:102F2800DAFFDECF90F0DDCF91F08E5190278F51F0
:102F380091232E0E90250D6E000E91210E6EAAC0C3
:102F48000FF0ABC010F0F0EC57F0AA51A127AB512D
:102F5800A22320EE06F06250D9266350DA22AA5145
:102F6800DE26AB51DE22000EDE22DE2268C0D9FF4B
:102F780069C0DAFFAA51DE26AB51DD22AA51665E8E
:102F8800AB51675A6650671001E0B7D5000CD251B3
:102F9800D31101E1090CD2C0D9FFD3C0DAFFDE6A30
:102FA800DD6A8CC1C2F18DC1C3F11F0ED617C20EE6
:102FB800666E010E676ED40E686ED651FE0B696E92
:102FC80009EC00F00101BF6FBF5101E040D2AB0E28
:102FD800D66F010ED76FC20E0001BC6F010EBD6F18
:102FE800D4C0BEF0D5C0BFF01BEC46F00101BF6FE6
:102FF800D4C1C0F1D5C1C1F1BF5105E1C051C11162
:1030080002E1060EBF6FD6C0D7F01C0E0001D7171D
:1030180001E114D10101BF5113E0040EBF1909E108
:10302800C20E0001C06F010EC16F6BEC4FF00101C1
:10303800BF6F0001D687D4C1C0F1D5C1C1F113D08B
:1030480020EE0BF0C051D926C151DA22DF50000121
:10305800D76F110ED71702E0070E03D0D6A503D0FD
:10306800080E0101BF6F0101BF5101E002D100014B
:10307800D6A7FFD00101BB6BBC6B210EBD6F460EFE
:10308800BE6F20EE0EF0C051D926C151DA22DF6A98
:1030980020EE0FF0C051D926C151DA22BCC1DFFFA2
:1030A80020EE10F0C051D926C151DA22BDC1DFFF90
:1030B80020EE11F0C051D926C151DA22BEC1DFFF7E
:1030C80020EE16F0C051D926C151DA22DF6A20EE6F
:1030D80017F0C051D926C151DA22BCC1DFFF20EE5A
:1030E80018F0C051D926C151DA22BDC1DFFF20EE48
:1030F80019F0C051D926C151DA22BEC1DFFF20EE36
:103108000BF0C051D926C151DA22DF6A20EE1CF03B
:10311800C051D926C151DA22DF6A20EE1DF0C05114
:10312800D926C151DA22DF6A20EE1EF0C051D92615
:10313800C151DA22DF6A20EE1FF0C051D926C151F1
:10314800DA22DF6AC2C10BF0C3C10CF0C0C10DF0B6
:10315800C1C10EF0CCEC4FF00BC0B7F10CC0B8F108
:103168000DC0B9F10EC0BAF1C0C10BF0C1C10CF06D
:103178000D6A0E6A0F6A106A8EEC57F0010120EE94
:1031880004F0C251D926C351DA22010EDF6EB751BD
:10319800B811B911BA116DE020EE2AF0C251D92642
:1031A800C351DA22DECFBBF1DECFBCF1DECFBDF1F9
:1031B800DECFBEF1C2C18CF0C3C18DF0B7C18EF0B5
:1031C800B8C18FF0B9C190F0BAC191F049EC49F09B
:1031D8000101BF6FBF514DE1FF0EB7250001D76F49
:1031E800FF0E0101B8210001D86FFF0E0101B921BE
:1031F8000001D96FFF0E0101BA210001DA6F010148
:1032080020EE0AF0C251D926C351DA22D7C0DEFF18
:10321800D8C0DEFFD9C0DEFFDAC0DEFFC2C139F098
:10322800C3C13AF0BBC13BF0BCC13CF0BDC13DF0ED
:10323800BEC13EF0C3EC50F001011AD00101BF51EC
:1032480018E120EE0BF0C051D926C151DA22DFA8CF
:1032580002D0040E0DD00001D6A30BD0010120EE40
:103268000BF0C051D926C151DA22DFA002D0070ED7
:10327800BF6F0101BF5123E10001D6B7D68B010111
:1032880020EE2AF0C251D926C351DA22000110EEED
:103298001AF0D251E126D351E222DECFE6FFDECF8B
:1032A800E6FFDECFE6FFDECFE6FF20EE1EF0D251CE
:1032B800D926D351DA22C0C1DEFFC1C1DDFF010129
:1032C800BF5101E0C4D0000120EE04F0D251D9264C
:1032D800D351DA22D6C0DFFF20EE05F0D251D9262D
:1032E800D351DA22DF6AC2C10BF0C3C10CF0C0C1EE
:1032F8000DF0C1C10EF0CCEC4FF0000120EE0EF045
:10330800D251D926D351DA220BC0DEFF0CC0DEFF22
:103318000DC0DEFF0EC0DEFF010120EE1DF0C05122
:10332800D926C151DA22DF500001D86FD76B0101CD
:1033380020EE1EF0C051D926C151DA22DF5000011B
:10334800D96FD9C0DAF0DB6BDC6BDD6BDBC0DDF08D
:10335800DAC0DCF0DB6BDA6B010120EE1FF0C05144
:10336800D926C151DA22DF500001DE6FDEC0DFF05E
:10337800E06BE16BE26BDFC0E2F0E16BE06BDF6B0F
:10338800DA51DF11E36FDB51E011E46FDC51E11139
:10339800E56FDD51E211E66FD751E311E76FD851C0
:1033A800E411E86F000EE511E96F000EE611EA6F0F
:1033B800010120EE1CF0C051D926C151DA22DF509C
:1033C8000001E711EB6FE851EC6FE951ED6FEA513D
:1033D800EE6F20EE0AF0D251D926D351DA22EBC093
:1033E800DEFFECC0DEFFEDC0DEFFEEC0DEFF20EE4C
:1033F80006F0D251D926D351DA22DE6ADE6ADE6AB5
:10340800DD6A20EE16F0D251D926D351DA22DE6ACF
:10341800DE6ADE6ADD6AD2C0D9FFD3C0DAFFC2C174
:10342800DEFFC3C1DDFFD2C0D9FFD3C0DAFF10EE83
:1034380006F0DE50E126DD50E22220EE02F0D25105
:10344800D926D351DA22E6CFDEFFE5CFDDFF010131
:10345800BF51120049504810471003E1020E465C64
:1034680010E320EE12F04450D9264550DA22DE50FF
:10347800465CDE504758DE504858DE50495801E255
:103488002FD2020E866F41D246C084F047C085F025
:10349800D89085314F6E84314E6E4E5084274F50F0
:1034A800852344C039F045C03AF020EE1EF0445060
:1034B800D9264550DA22DECF4EF0DECF4FF0DECFF0
:1034C80050F0DECF51F084C052F085C053F0090EA1
:1034D800546ED89053325232542EFBD752504E2449
:1034E8003B6E53504F203C6E000E50203D6E000E38
:1034F80051203E6EC3EC50F00001866F865101E00A
:1035080004D24E68010E4F6E84C050F085C051F051
:103518004E5050164F50511644C052F045C053F00B
:1035280050505226515053222E0E5224876F000EAF
:103538005320886F844B852B46B004D04AC080F056
:10354800816B1AD04A504E6E4F6A4E3A4F3AF00E7F
:103558004F164E500F0B4F12F00E4E1687C0D9FF64
:1035680088C0DAFFDF500F0B506E516A4E50501072
:10357800806F4F505110816F87C0D9FF88C0DAFF24
:1035880080C0DFFF20EE04F04450D9264550DA22EF
:10359800010EDF6E44C039F045C03AF020EE1EF04F
:1035A8004450D9264550DA22DECF4EF0DECF4FF018
:1035B800DECF50F0DECF51F084C052F085C053F01A
:1035C800090E546ED89053325232542EFBD75250B3
:1035D8004E243B6E53504F203C6E000E50203D6EE3
:1035E800000E51203E6EC3EC50F00001866F8651EC
:1035F80001E08BD14E68010E4F6E84C050F085C03B
:1036080051F04E5050164F50511644C052F045C01C
:1036180053F050505226515053222E0E5224876F89
:10362800000E5320886F46B00CD04BC04EF00F0EE2
:103638004E1687C0D9FF88C0DAFFDF50F00B4E1056
:1036480012D04AC04EF04BC04FF04CC050F04DC0A5
:1036580051F0050E05D0D890513250324F324E32CB
:10366800E82EF9D74E50826F836B87C0D9FF88C088
:10367800DAFF82C0DFFF2BD144C039F045C03AF0F1
:1036880020EE1EF04450D9264550DA22DECF4EF007
:10369800DECF4FF0DECF50F0DECF51F04750526E04
:1036A8004850536E4950546E556A4E5052243B6EE2
:1036B8004F5053203C6E505054203D6E5150552071
:1036C8003E6EC3EC50F00001866F865101E01DD1BB
:1036D8004E68010E4F6E46C050F047C051F0D8906A
:1036E800503651364E5050164F50511644C052F075
:1036F80045C053F050505226515053222E0E52249A
:10370800876F000E5320886F87C0D9FF88C0DAFF03
:103718004AC0DFFF20EE01F08751D9268851DA220E
:103728004BC0DFFFD4D044C039F045C03AF020EE9A
:103738001EF04450D9264550DA22DECF4EF0DECFB7
:103748004FF0DECF50F0DECF51F046C052F047C008
:1037580053F048C054F049C055F0080E05D0D89031
:103768005532543253325232E82EF9D74E50522441
:103778003B6E4F5053203C6E505054203D6E51507C
:1037880055203E6EC3EC50F00001866F865101E073
:10379800BCD04E68010E4F6E46C050F047C051F085
:1037A800D89050365136D890503651364E50501623
:1037B8004F50511644C052F045C053F05050522655
:1037C800515053222E0E5224876F000E5320886FBB
:1037D80020EE01F08751D9268851DA22DF504F6E4A
:1037E8004E6A20EE02F08751D9268851DA22DF503E
:1037F800506E50C051F0526A536A546A52C054F025
:1038080051C053F0526A516A20EE03F08751D9260D
:103818008851DA22DF50556E55C056F0576A586AFB
:10382800596A56C059F0586A576A566A5150561024
:103838005A6E525057105B6E535058105C6E54506D
:1038480059105D6E4E505A105E6E4F505B105F6E91
:10385800000E5C10606E000E5D10616E87C0D9FFAF
:1038680088C0DAFFDF505E10626E5F50636E605092
:10387800646E6150656E666A676A686AF00E651400
:10388800696E66504A1267504B1268504C12695064
:103898004D1287C0D9FF88C0DAFF4AC0DFFF20EE8B
:1038A80001F08751D9268851DA224BC0DFFF20EE7C
:1038B80002F08751D9268851DA224CC0DFFF20EE6A
:1038C80003F08751D9268851DA224DC0DFFF20EE58
:1038D80004F04450D9264550DA22010EDF6E15D087
:1038E80044C0D9FF45C0DAFFDF504E6E4F6A4F50D3
:1038F80001E0C7D54E50010A01E1C6D5030A01E12E
:10390800BBD6010A01E10FD7BCD5865112008980C8
:103918002D0E0001806FF70E816FCFCF82F0836B81
:10392800CECF84F0856B7350140D070EF324D96E37
:10393800010EF420DA6EDECF86F0DECF87F0DECF20
:1039480088F0DECF89F07350140D070EF324D96E7A
:10395800010EF420DA6EDECF8AF0DECF8BF0DECFF8
:103968008CF0DECF8DF07DEC5AF0B2EC41F0CAC09D
:10397800B3F1CBC0B4F10101B351B4111AE07350E3
:10398800140D130EF324D96E010EF420DA6E735061
:10399800140D130EF324E16E010EF420E26EE750CD
:1039A8000409DF6E55EC59F0B3C1E1F0B4C1E2F09F
:1039B800120072507BE07350140D070EF324D96E79
:1039C800010EF420DA6E78C1E8F079C1E9F07AC125
:1039D800EAF00001E76B000EE725EB6F010EE82126
:1039E800EC6F000EE921ED6F000EEA21EE6FDE505C
:1039F800EB195CE1DE50EC1959E1DE50ED1956E1A6
:103A0800DE50EE1953E114EC55F00FC0B8F110C0B8
:103A1800B9F111C0BAF112C0BBF1000EE8CF74FAC7
:103A28002AEE75F0BBC1DFFFE8CF76FA2AEE77F011
:103A3800BAC1DFFFE8CF78FA2AEE79F0B9C1DFFF23
:103A4800E8CF7AFA2AEE7BF0B8C1DFFF0101FC93D8
:103A5800010E496E486A8EEC3DF0FC935F0E000142
:103A6800806FF50E816FCFCF82F0836BCECF84F05D
:103A7800856B2AEE75F0DF50866F876B2AEE77F03C
:103A8800DF50886F896B2AEE79F0DF508A6F8B6B75
:103A98002AEE7BF0DF508C6F8D6B7DEC5AF06B6AF1
:103AA80089906BC0E1F00001E26B12007350140DB5
:103AB8000F0EF324D96E010EF420DA6EDECFE3F098
:103AC800DECFE4F0DECFE5F0DECFE6F0E4C0E3F0F1
:103AD800E5C0E4F0E6C0E5F00001E66BE3C0AFF155
:103AE800E4C0B0F17350140D0F0EF324D96E010E1B
:103AF800F420DA6EDECFE3F0DDCFE4F0E35101012C
:103B0800B56FB66BFC93AB6BAC6BAD6BAE6BB16B5F
:103B1800B26BA9D0E369E469AFC1E5F0B0C1E6F0E2
:103B2800E351E527E451E6230101B1510001E5190C
:103B38000AE10101B2510001E61905E10101B5519F
:103B4800B61101E1FC837350200D000EF324626E60
:103B5800020EF420636E740E646E0A0E656E010E1A
:103B6800676E666ABC0E686E010E696E16EC15F01B
:103B78000101B76FC60E0001806FF60E816FCFCFBF
:103B880082F0836BCECF84F0856BB7C186F0876BEC
:103B9800BCC188F0BDC189F07DEC5AF00101B75174
:103BA80001E0EDD6BCC148F0BDC149F08EEC3DF056
:103BB800BC51AB27BD51AC23000EAD23AE237350CF
:103BC800140D070EF324D96E010EF420DA6E000EE0
:103BD800DE240001E36F010EDE20E46F000EDE201C
:103BE800E56F000EDE20E66F7350140D070EF32408
:103BF800D96E010EF420DA6EE3C0DEFFE4C0DEFF0A
:103C0800E5C0DEFFE6C0DEFF3D0E806FF90E816F76
:103C1800CFCF82F0836BCECF84F0856B7350140DB9
:103C2800070EF324D96E010EF420DA6EDECF86F08B
:103C3800DECF87F0DECF88F0DECF89F07350140D29
:103C4800070EF324D96E010EF420DA6EDECF8AF067
:103C5800DECF8BF0DECF8CF0DECF8DF07DEC5AF02E
:103C68000101B14BB22BAF51B15DB251800A0001D5
:103C7800E36F0101B051800A0001E35901E24AD71C
:103C88000101B6BF88D0B65103E1B50501E283D082
:103C98007350200D000EF324626E020EF420636E42
:103CA800740E646E0A0E656EB5C166F0B6C167F033
:103CB800BC0E686E010E696E16EC15F00101B76F47
:103CC800D30E0001806FF60E816FB7C182F0836B4F
:103CD800BCC184F0BDC185F07DEC5AF00101B7513B
:103CE80001E04DD6FC83B5C148F0B6C149F08EEC71
:103CF8003DF0BC51AB27BD51AC23000EAD23AE2324
:103D08007350140D070EF324D96E010EF420DA6EE9
:103D1800000EDE240001E36F010EDE20E46F000ECA
:103D2800DE20E56F000EDE20E66F7350140D070EDF
:103D3800F324D96E010EF420DA6EE3C0DEFFE4C08E
:103D4800DEFFE5C0DEFFE6C0DEFF740E806FFC0E0E
:103D5800816F7350140D070EF324D96E010EF420F1
:103D6800DA6EDECF82F0DECF83F0DECF84F0DECFF6
:103D780085F07350140D070EF324D96E010EF4204C
:103D8800DA6EDECF86F0DECF87F0DECF88F0DECFCA
:103D980089F07DEC5AF00101FC93970E0001806FC9
:103DA800FA0E816FCFCF82F0836BCECF84F0856B14
:103DB800ABC186F0ACC187F0ADC188F0AEC189F067
:103DC8007DEC5AF06CD649504810471003E1020EBA
:103DD800465C0FE320EE12F04450D9264550DA2213
:103DE800DE50465CDE504758DE504858DE50495891
:103DF80008E3010E0001846F000E856B866B876BEC
:103E0800EFD100018469856986698769D4D146C084
:103E180088F047C089F0D89089314B6E88314A6E56
:103E28004A5088274B50892344C039F045C03AF09E
:103E380020EE1EF04450D9264550DA22DECF4AF053
:103E4800DECF4BF0DECF4CF0DECF4DF088C04EF029
:103E580089C04FF0090E506ED8904F324E32502E16
:103E6800FBD74E504A243B6E4F504B203C6E000E01
:103E78004C203D6E000E4D203E6EC3EC50F0000904
:103E880001E0AED14A68010E4B6E88C04CF089C083
:103E98004DF04A504C164B504D1644C04EF045C09C
:103EA8004FF04C504E264D504F222E0E4E24D96EB8
:103EB800000E4F20DA6EDF500001826F836B884B53
:103EC800892B44C039F045C03AF020EE1EF044502A
:103ED800D9264550DA22DECF4AF0DECF4BF0DECFCE
:103EE8004CF0DECF4DF088C04EF089C04FF0090E7F
:103EF800506ED8904F324E32502EFBD74E504A2437
:103F08003B6E4F504B203C6E000E4C203D6E000E19
:103F18004D203E6EC3EC50F0000901E061D14A68C3
:103F2800010E4B6E88C04CF089C04DF04A504C16BB
:103F38004B504D1644C04EF045C04FF04C504E26E5
:103F48004D504F222E0E4E24D96E000E4F20DA6EA1
:103F5800DF50516E506A5050000182135150831344
:103F680046B006D08251806F0F0E8315816F0FD037
:103F780082C04AF083C04BF0040E4C6ED8904B328E
:103F88004A324C2EFBD74AC080F04BC081F080C02B
:103F980084F081C085F05BD044C039F045C03AF068
:103FA80020EE1EF04450D9264550DA22DECF4AF0E2
:103FB800DECF4BF0DECF4CF0DECF4DF047504E6EEB
:103FC80048504F6E4950506E516A4A504E243B6ECD
:103FD8004B504F203C6E4C5050203D6E4D50512060
:103FE8003E6EC3EC50F0000901E0FAD04A68010EB9
:103FF8004B6E46C04CF047C04DF0D8904C364D360D
:104008004A504C164B504D1644C04EF045C04FF028
:104018004C504E264D504F222E0E4E2400018A6FD2
:10402800000E4F208B6F20EE01F08A51D9268B515C
:10403800DA22DF504B6E4A6A8AC0D9FF8BC0DAFF9A
:10404800DF504A12000E4AC084F04BC085F0866BE0
:10405800876BC6D044C039F045C03AF020EE1EF058
:104068004450D9264550DA22DECF4AF0DECF4BF055
:10407800DECF4CF0DECF4DF046C04EF047C04FF0DB
:1040880048C050F049C051F0080E05D0D8905132C0
:1040980050324F324E32E82EF9D74A504E243B6EFA
:1040A8004B504F203C6E4C5050203D6E4D5051208F
:1040B8003E6EC3EC50F0000901E092D04A68010E50
:1040C8004B6E46C04CF047C04DF0D8904C364D363C
:1040D800D8904C364D364A504C164B504D1644C06D
:1040E8004EF045C04FF04C504E264D504F222E0EEC
:1040F8004E2400018A6F000E4F208B6F20EE01F0D6
:104108008A51D9268B51DA22DF504B6E4A6A20EE4B
:1041180002F08A51D9268B51DA22DF504C6E4CC0FE
:104128004DF04E6A4F6A506A4EC050F04DC04FF085
:104138004E6A4D6A20EE03F08A51D9268B51DA2255
:10414800DF50516E51C052F0536A546A556A52C0DA
:1041580055F0546A536A526A4D505210566E4E507A
:104168005310576E4F505410586E50505510596E8A
:104178004A5056105A6E4B5057105B6E000E58102E
:104188005C6E000E59105D6E8AC0D9FF8BC0DAFFD5
:10419800DF505A105E6E5B505F6E5C50606E5D5013
:1041A800616E5E50846F5F50856F6050866F0F0E32
:1041B8006114876F15D044C0D9FF45C0DAFFDF50BE
:1041C8004A6E4B6A4B5001E014D64A50010A01E18D
:1041D8001ED6030A01E1E0D6010A01E13BD709D660
:1041E80084C044F085C045F086C046F087C047F0DB
:1041F800120018C0F6FF19C0F7FF000EF86E0F0E78
:10420800F76403D00800F55005D0F6CFE9FFF7CFE3
:10421800EAFFEF50466E184A192A465001E112008B
:10422800250E461804E0465087EC5AF0E2D7416A5A
:10423800426A18C0F6FF19C0F7FF000EF86E0F0E9D
:10424800F76403D00800F55005D0F6CFE9FFF7CFA3
:10425800EAFFEF50466E184A192A300E461818E140
:10426800426A010E416E18C0F6FF19C0F7FF000E32
:10427800F86E0F0EF76403D00800F55005D0F6CF9E
:10428800E9FFF7CFEAFFEF50466E184A192A06D021
:104298002D0E461803E1426A020EE4D7396A3A6ADB
:1042A80027D00A0E3902F3CF1BF0F4CF1CF03A02E4
:1042B800F3501C2646501B26000E1C22D00E1B2431
:1042C800396EFF0E1C203A6E18C0F6FF19C0F7FFB2
:1042D800000EF86E0F0EF76403D00800F55005D0F5
:1042E800F6CFE9FFF7CFEAFFEF50466E184A192AD2
:1042F8002F0E466403D0390E4664D3D76C0E461889
:1043080003E04C0E461815E1418418C0F6FF19C0A9
:10431800F7FF000EF86E0F0EF76403D00800F55093
:1043280005D0F6CFE9FFF7CFEAFFEF50466E184AFF
:10433800192A465001E1120046C045F0600E456456
:1043480072D0200E455E6FD01A50D96EDA6A020E0E
:10435800DF26DF5CD96EDA6ADECF35F0DECF36F0E5
:104368003B6A3C6A02D03B4A3C2A3B5035241B6ED0
:104378003C5036201C6E1BC0F6FF1CC0F7FF000E19
:10438800F86E0F0EF76403D00800F55005D0F6CF8D
:10439800E9FFF7CFEAFFEF50000904E0E4D7200E69
:1043A80087EC5AF041B20BD03B501B6E3C501C6E50
:1043B8003B4A3C2A39501B5C3A501C58F0E335C044
:1043C8000CF036C00DF0ABEC56F003D0200E87ECA5
:1043D8005AF03B501B6E3C501C6E3B4A3C2A3950ED
:1043E8001B5C3A501C5801E304D7F0D71A50D96E19
:1043F800DA6ADF50DF2ADF2AD96EDA6ADF5087EC03
:104408005AF0F7D6386A020E08D0386A080E05D076
:10441800386A0A0E02D0386A100E376E19D0465024
:1044280087EC5AF0E6D645501B6E1C6A1C50F7E123
:104438001B50420AE7E0010AD9E0070AE9E00B0A43
:10444800E4E01C0A81E0060AE3E00D0AE4E0E7D7AD
:1044580041B430D0440E451813E01A50D96EDA6AC8
:10446800DF50DF2ADF2AD96EDA6ADECF1BF0DDCF14
:104478001CF01BC02DF01CC02EF02F6A306A11D022
:104488001A50D96EDA6ADF50DF2ADF2AD96EDA6A63
:10449800DECF2DF0DDCF2EF0000E2EBEFF0E2F6EDC
:1044A800306E2DC03DF02EC03EF02FC03FF030C022
:1044B80040F010D01A50D96EDA6A040EDF26DF5C9D
:1044C800D96EDA6ADECF3DF0DECF3EF0DECF3FF0C8
:1044D800DECF40F0440E45180CE140AE0AD03D6CEA
:1044E8003E1ED8B03E2A3F1ED8B03F2A000E405686
:1044F8004186436A446A3DC00BF03EC00CF03FC0A1
:104508000DF040C00EF037C00FF038C010F0116A3F
:10451800126A48EC55F00B50456E3DC00BF03EC09A
:104528000CF03FC00DF040C00EF037C00FF038C09F
:1045380010F0116A126ABCEC53F00BC03DF00CC0CD
:104548003EF00DC03FF00EC040F0090E45640BD0A0
:10455800780E461803E0326A070E02D0326A270E38
:10456800316E3150452643501D0FD96EDA6A4550D9
:10457800300FDF6E434A442A3D503E103F10401032
:1045880005E0445003E1100E435CB5E341A608D0B2
:1045980043501D0FD96EDA6A2D0EDF6E434A442A46
:1045A80043C03BF044C03CF041B003D0346A200E15
:1045B80002D0346A300E336E33C045F003D0455014
:1045C80087EC5AF041B20BD03B501B6E3C501C6E2E
:1045D8003B4A3C2A39501B5C3A501C58F0E34306CE
:1045E800D8A0440643501D0FD96EDA6ADF5087EC15
:1045F8005AF04350441004E0F2D7200E87EC5AF0EA
:104608003B501B6E3C501C6E3B4A3C2A39501B5C8D
:104618003A501C5801E3EDD5F0D72A6E1BC041F083
:104628001CC042F02A5001E0040C010E3F6E74B029
:10463800030CE9D150EC5AF0000901E1FDD13F6AC1
:10464800FBD1146A156A166A176A090EBDEC58F090
:10465800000901E0F1D12B0E0B6E0C6A0E6A100EE8
:104668000D6E00EC56F0000901E1E6D12B44E84656
:10467800030BE8064DE132C01DF03F0E1D161DC0AC
:104688001EF01F6A206A216A1FC021F01EC020F098
:104698001F6A1E6A3350236E226A3450246E256ABC
:1046A800225024262350252224501E24266E2550CD
:1046B8001F20276E000E2020286E000E2120296E54
:1046C80026283B6E000E27203C6E000E28203D6EEB
:1046D800000E29203E6E3BC01DF03CC01EF03DC0C0
:1046E8001FF03EC020F00A0ED8901D361E361F3629
:1046F8002036E82EF9D71BC0D9FF1CC0DAFF1DC031
:10470800DEFF1EC0DEFF1FC0DEFF20C0DEFF97D722
:104718001D6A35AE01D01D2A010E1D1630C01EF0CF
:104728000F0E1E163450030B020DF3501E241D24C9
:10473800020F406E3150030B1D6E1E6A0A0ED89090
:104748001D361E36E82EFBD732501F6E206AD890D1
:104758001F362036D8901F3620363344E846030BE0
:10476800216E226A1F502126205022221D50212608
:104778001E502222212A000E222221C03BF022C0F4
:104788003CF03D6A3E6A40C01DF0F70E1D263BC056
:104798001EF03CC01FF03DC020F03EC021F01D2A95
:1047A80005D0D8901E361F36203621361D2EF9D753
:1047B80034D06EA43FD0146A156A166A176A8D0E33
:1047C800BDEC58F0000901E037D1A3EC5AF02B0EEC
:1047D8000B6E0C6A0E6A100E0D6E00EC56F0000996
:1047E80001E12AD1300E406E03D0A3EC5AF0400606
:1047F8004050FBE135C01DF01D3A0F0E1D16100E7E
:104808001E6E1F6A206A216A1D2A05D0D8901E369E
:104818001F36203621361D2EF9D71BC0D9FF1CC0E4
:10482800DAFF1EC0DEFF1FC0DEFF20C0DEFF21C092
:10483800DEFF05D7146A156A166A176A090EBDECF9
:1048480058F0000901E0F8D02B0E0B6E0C6A0E6AC6
:10485800100E0D6E00EC56F0000901E1EDD06EA2CD
:1048680032D038C01DF0060E1E6ED8901D321E2E96
:10487800FCD7FF0E1D2635503F0B1F6E206AD890BF
:104888001F3620363644010B1F26000E20221F2A11
:1048980020221D2A03D0D8901F3620361D2EFBD784
:1048A8001F50216E2050226E236A246A1BC0D9FF34
:1048B8001CC0DAFF21C0DEFF22C0DEFF23C0DEFFFE
:1048C80024C0DEFFBCD63650030B1D6E1E6AD8907E
:1048D8001D361E36D8901D361E36D8901D361E360B
:1048E8003638E842070B1D26000E1E221D2A1E22FE
:1048F8003540E8423F0B1F0B1F6E206A1F2A000E2F
:1049080020221D501F02F3CF21F0F4CF22F0200205
:10491800F35022261E501F02F35022262150236EE8
:104928002250246E256A266A1BC0D9FF1CC0DAFFF4
:1049380023C0DEFF24C0DEFF25C0DEFF26C0DEFF69
:104948007ED641C0D9FF42C0DAFF6EC0DFFF77D6FE
:10495800146A156A166A176A090EBDEC58F0000940
:104968006BE141C00BF042C00CF00E6A100E0D6EE8
:1049780000EC56F0000901E062D65ED0146A156AB0
:10498800166A176A0A0EBDEC58F0000955E141C0D5
:104998000BF042C00CF00E6A100E0D6E00EC56F0D3
:1049A800E9D7146A156A166A176A3A0EBDEC58F008
:1049B800000942E1040E406E0AD0A3EC5AF041C04F
:1049C800D9FF42C0DAFFDF6E414A422A4006405012
:1049D80001E135D6F2D7146A156A166A176A8D0E80
:1049E800BDEC58F0000928E1A3EC5AF041C00BF0E7
:1049F80042C00CF00E6A400E0D6E00EC56F0BAD7AD
:104A0800040E3F6E19D01A501D6E1E6A1E50F8E132
:104A18001D5001E10FD6010A01E113D6020A01E196
:104A2800C8D6090A8EE0010A93E0070AA7E0010A3E
:104A3800B8E0030AD0E0E4D7BBEC5AF03F501200CC
:104A480055C058F056C059F001017C6B7D6BF6D10A
:104A580054C046F0580E476E57C048F04750D96EBC
:104A6800DA6ADECFF6FFDDCFF7FFF86A000EF86EE0
:104A78000800F550250AD8A4C3D14750D96EDA6A80
:104A8800DE2A000EDD2201017E6B7F6B826B836B59
:104A9800806981694750D96EDA6ADECFF6FFDDCFCB
:104AA800F7FFF86A000EF86E0800F550780AD8B4D7
:104AB8000FD04750D96EDA6ADECFF6FFDDCFF7FFA9
:104AC800F86A000EF86E0800F550580AD8A46ED19E
:104AD8004750D96EDA6ADECFF6FFDDCFF7FFF86A06
:104AE800000EF86E0800F5CF53F04750D96EDA6A19
:104AF800DE2A000EDD224850D96EDA6ADF50DF2A3E
:104B0800DF2AD96EDA6ADECF49F0DDCF4AF049C034
:104B18004BF04AC04CF04D6A4E6A4F6A506A516A6F
:104B2800526A46C024F04BC025F04CC026F04DC058
:104B380027F04EC028F04FC029F050C02AF051C0CD
:104B48002BF052C02CF053C02DF081BF01D08293BE
:104B580081BF05D0815107E18005D8B004D0376AFC
:104B6800010E366E04D080C136F081C137F07EC1A7
:104B780040F07FC141F082A904D0FE0E4026FF0E0E
:104B8800412225C038F026C039F027C03AF028C0A5
:104B98003BF029C03CF02AC03DF02BC03EF02CC0B1
:104BA8003FF0436A1F0E426E02019F6B6DD04206B2
:104BB800D8A043060F0E3814446E456A45BE08D087
:104BC800455004E10A0E445CD8A002D0570E01D02B
:104BD800300E4426000E4522BF0E2E6E2F682D5033
:104BE800306E316A2E5030262F503122315005E177
:104BF8001A0E305C02E2010E01D0000E326E336AEA
:104C080032503310D8B425D09F0E2E6E2F68200E48
:104C18004410306E000E4510316E2E5030262F5045
:104C28003122315005E11A0E305C02E2010E01D04A
:104C3800000E346E356A34503510D8B40AD044C0EA
:104C480011F045C012F04BEC57F011C044F012C0FF
:104C580045F0800E4224D96E020E4320DA6E44C01D
:104C6800DFFF3606D8A037064006D8A04106040E56
:104C78002E6ED8903F323E323D323C323B323A3291
:104C8800393238322E2EF5D743BE21D0435004E1B5
:104C9800020E425CD8A01BD0385039103A103B1095
:104CA8003C103D103E103F10D8A481D737BE05D028
:104CB800375002E13604D8B07AD741BE08D0415007
:104CC80003E14004D8A003D0010182B370D70101E9
:104CD80082A916D04206D8A04306800E4224D96E77
:104CE800020E4320DA6E2DC0DFFF4206D8A043062D
:104CF800800E4224D96E020E4320DA6E300EDF6E2B
:104D080024C01AF0800E42241B6E020E43201C6E33
:104D180040C01DF041C01EF082A108D01BC014F095
:104D28001CC015F01AC016F03EEC59F01EBE05D096
:104D38001DC022F01EC023F002D0226A236A206A16
:104D4800216A0AD0000E0D6E200E0C6E1AC00EF0ED
:104D58007AEC52F0204A212A2250205C2150800A05
:104D68001F6E2350800A1F58D8A0ECD7010182B1CA
:104D780008D01BC014F01CC015F01AC016F03EEC89
:104D880059F01BC00BF01CC00CF0AFEC57F02250D0
:104D98000B241A6E23500C201B6E1AC024F01BC063
:104DA80025F024C046F025C047F043D04750D96EBF
:104DB800DA6ADECFF6FFDDCFF7FFF86A000EF86E8D
:104DC8000800F550250AD8A412D04750D96EDA6ADF
:104DD800DE2A000EDD22000E0D6E250E0C6E46C07A
:104DE8000EF07AEC52F0476A010E466E22D0475018
:104DF800D96EDA6ADE2A000EDD22466A476A19D0C1
:104E08004750D96EDA6ADECFF6FFDDCFF7FFF86AD2
:104E1800000EF86E0800F5500C6E0D6A46C00EF0D4
:104E28007AEC52F04750D96EDA6ADE2A000EDD229B
:104E3800DAD7465001017C2747507D2358C0F6FF3A
:104E480059C0F7FF0800F55001E002D67CC154F0C4
:104E58007DC155F012004D6E495002E0F7EC53F059
:104E68004C6A485001E184D14D9E040E4D1803E070
:104E7800140E4D1807E101018E6B8F6B496A070EFE
:104E8800486E070C3F0E4D1807E16F6A01018E6BE3
:104E98008F6B486A496A12005F0E4D1807E1706A05
:104EA80001018E6B8F6B486A496A12003F0E4D6490
:104EB80006D05F0E4D6003D0400E4D18F0E1400E55
:104EC8004D1809E1010E706E6F6A01018E6B8F6BD0
:104ED800486A496A1200200E4D1801E049D1010EB6
:104EE8006F6EF3D7600E4D1809E1705007E00101AD
:104EF8009E51080ED8B4030E4C6E73D0600E4D1838
:104F080009E16F5007E001019E5102E0090E14D03B
:104F1800050E12D0680E4D1809E16F5007E01A0E01
:104F280001018F6F900E17D189807CD1680E4D18C2
:104F380005E1705003E0020E4C6E53D06A0E4D1816
:104F480007E16F5005E01A0E01018F6FF40E03D1CF
:104F58006C0E4D1807E16F5005E01A0E01018F6FB6
:104F68002C0EF9D0700E4D1808E1705006E0040EB2
:104F78004C6E01018E6B8F6BD7D7700E4D1801E008
:104F880051D16F5001E14ED11B0E01018F6F620E9E
:104F9800E2D08980020E4D1805E11A0E01018F6FCB
:104FA800920E8E6F050E4D1805E11A0E01018F6FD6
:104FB800AE0E8E6F070E4D1805E11A0E01018F6FA8
:104FC800B80E8E6F080E4D1805E11A0E01018F6F8D
:104FD800CC0E8E6F030E4D1802E04D2806E14C6A88
:104FE800899001018E6B8F6B1DD1160E4D1801E053
:104FF80019D11A0E01018F6FA40E9ED0050E4D18FF
:1050080001E010D11A0E01018F6FF50E95D04DC039
:1050180073F01A0E01018F6F9B0E8ED01A0E0101CC
:105028008F6F9C0E89D07350070D500EF324D96EE4
:10503800010EF420DA6E4DC0DFFF1A0E01018F6FEA
:105048009D0E7AD07350070D510EF324D96E010EC0
:10505800F420DA6E4DC0DFFF1A0E01018F6F9E0E2D
:105068006BD07350070D520EF324D96E010EF42045
:10507800DA6E4DC0DFFF01018E6B8F6B010E2AD0F7
:105088001A0E01018F6FB90E66D01A0E01018F6FCB
:10509800BA0E52D01A0E01018F6FBB0E8E6FAC0E76
:1050A8000001806FFE0E816F7DEC5AF001019F6B4D
:1050B8008E6B8F6B48D001018E6B8F6BAC0E00012D
:1050C800806FFE0E816F7DEC5AF03DD001018E6B32
:1050D8008F6B060E4C6EA6D04DC073F001018E6B1F
:1050E8008F6B4C6A30D001019E6B1A0E8F6FF70ED2
:1050F8008E6F29D01A0E01018F6FF70E1DD089907F
:10510800270E01018F6F0F0E17D0180E4D1801E0F2
:1051180089D01A0E01018F6F2D0E0ED01A0E0101C3
:105128008F6F2E0E09D01A0E01018F6F2F0E04D02B
:105138001A0E01018F6F300E8E6F74D001018E6BC5
:105148008F6B0A0E4C6E89906DD0040E4C6E270E34
:1051580001018F6F0F0E8E6FE7D68980010104D091
:105168008990010E01019E6F8E6B8F6B4C6A5AD02D
:105178008EC14AF08FC14BF04B5007E01A0A09E084
:10518800010A48E03C0A4CE04DD04A5001E1AAD659
:1051980049D04A502C0AB9E0010AC0E0030AC3E02A
:1051A800010AC6E01F0ACAE0A00A01E1F2D6020A13
:1051B80001E12DD7090A01E131D7070A01E133D707
:1051C800010A01E13FD7030A01E14BD73A0A01E19D
:1051D8007DD70A0AC5E0160A01E152D7010A01E1A2
:1051E80054D7030A01E156D7010A01E164D7790AC5
:1051F80001E1A1D60E0A01E16FD7380A01E1FED616
:10520800010A01E170D7030A01E174D7010A01E13B
:1052180076D708D04A50580A98E03A0A9EE002D059
:105228004A500F0A4CC048F0496A120020EE04F0B8
:10523800A351D926A451DA22DECFA7F0DDCFA8F0FA
:10524800A729B06F000EA821B16FB011D8B4040C13
:1052580020EE0EF0A351D926A451DA22DE50DE103A
:10526800DE10DE1001E1040CB0C0A7F00F0EA71786
:1052780001E094D120EE0EF0A351D926A451DA22F0
:10528800DE2A000EDE22DE22DE2220EE0AF0A35104
:10529800D926A451DA22DE50DE10DE10DE1011E12C
:1052A800A3C0D9FFA4C0DAFF10EE08F0DE50E12653
:1052B800DD50E222E650B05DE650B15901E26ED110
:1052C800040CB0C0A7F0B1C0A8F0040EA96FD89024
:1052D800A833A733A92FFBD7AA69AB69A3C0D9FF05
:1052E800A4C0DAFF10EE02F0DE50E126DD50E22223
:1052F800E750AC6FAD6BAA51AC27AB51AD23A751AA
:10530800AC17A851AD17AC51AD1101E047D1A3C0FE
:10531800D9FFA4C0DAFFDECF44F0DDCF45F020EEA0
:105328000AF0A351D926A451DA22DECF46F0DECF07
:1053380047F0DECF48F0DECF49F0E7EC1EF044C07E
:10534800B2F045C0B3F046C0B4F047C0B5F00001B4
:10535800B551B411B31104E1020EB25D01E2020CC1
:10536800B22907E1B32905E1B42903E1B52901E12F
:10537800010CA3C0D9FFA4C0DAFF10EE12F0DE5072
:10538800E126DD50E222E650B25DE650B359E65020
:10539800B459E650B55901E2D2D0A551A61101E1A0
:1053A800040CA3C0D9FFA4C0DAFFDECF8CF0DDCF98
:1053B8008DF020EE0AF0A351D926A451DA22DECFCF
:1053C8008EF0DECF8FF0DECF90F0DECF91F0E2EC02
:1053D80032F08CC0B2F08DC0B3F08EC0B4F08FC084
:1053E800B5F0B251B311B411B51101E1070CB20512
:1053F800B311B411B51101E1020CB22907E1B329C7
:1054080005E1B42903E1B52901E1010CA3C0D9FFE5
:10541800A4C0DAFFDECF24F0DDCF25F07AEC47F028
:10542800000901E0010CA3C0D9FFA4C0DAFFDECF58
:10543800A7F0DDCFA8F02E0E0001A7250B6E000EF9
:10544800A8210C6E0E6A0D6A020E106E0F6AC2EC6D
:1054580059F0A3C0D9FFA4C0DAFFDECF0BF0DDCF2F
:105468000CF0B2C00DF0B3C00EF0B4C00FF0B5C070
:1054780010F071EC4AF0A3C0D9FFA4C0DAFF10EE17
:105488002AF0DE50E126DD50E2220BC0E6FF0CC018
:10549800E6FF0DC0E6FF0EC0E6FF0001AE6BAF6B86
:1054A8002BD0A3C0D9FFA4C0DAFF10EE04F0DE5061
:1054B800E126DD50E222010EE76EA3C0D9FFA4C0A9
:1054C800DAFFDECF24F0DDCF25F07AEC47F00009D3
:1054D80001E0010CA3C0D9FFA4C0DAFF10EE2AF046
:1054E800DE50E126DD50E222E62A000EE622E62220
:1054F800E6220001AE4BAF2BA3C0D9FFA4C0DAFF50
:1055080010EE02F0DE50E126DD50E222E750A76FF0
:10551800A86BA751AE5DA851AF59C3E3A3C0D9FF8B
:10552800A4C0DAFF10EE2AF0DE50E126DD50E222B8
:10553800AE51E65EAF51E65A000EE65AE65A20EE44
:105548000AF0A351D926A451DA22B2C0DEFFB3C0B3
:10555800DEFFB4C0DEFFB5C0DEFFA3C0D9FFA4C024
:10556800DAFFDECF0BF0DDCF0CF0B2C00DF0B3C028
:105578000EF0B4C00FF0B5C010F071EC4AF00001A5
:1055880020EE0EF0A351D926A451DA220BC0DEFF7B
:105598000CC0DEFF0DC0DEFF0EC0DEFF20EE04F003
:1055A800A351D926A451DA22B0C0DEFFB1C0DDFF75
:1055B8000F0EB015A76FA86B050ED890A737A837A0
:1055C800E82EFBD7A3C0D9FFA4C0DAFFDECFA9F02D
:1055D800DDCFAAF0A751A927A851AA232E0EA927E3
:1055E800000EAA2320EE12F0A351D926A451DA22E4
:1055F800A9C0DEFFAAC0DDFF000C000E626E020E1D
:10560800636E740E646E0A0E656E020E676E666ACD
:10561800DD0E686E696A16EC15F06C6E7A0E000184
:10562800806FFD0E816FDDC082F0DEC083F07DECFF
:105638005AF00001DF6BE06BDB6BDC6BE16BE26B5C
:10564800E151BD0FD96EDA6ADF6AE151CC0FD96E2C
:10565800DA6A000EDF6EE14BE22BE2BFF1D7E251CE
:1056680003E10F0EE15DECE3E36BE46B2DD1740E07
:10567800E325D96E0A0EE421DA6E0D0EDE1801E07C
:10568800E8D0000E806F040E816FDE0E826FFE0E72
:10569800836FBD0E846F856BCC0E866F876B7DEC38
:1056A8005AF08E0E0B6EFF0E0C6EBD0E0D6E5CEC7E
:1056B80051F00B500C1007E1CC0E126E7AEC4BF047
:1056C80012500101FE6F880E0B6EFF0E0C6EBD0EA0
:1056D8000D6E5CEC51F00B500C1007E1CC0E126E05
:1056E8007AEC4BF012500101A06F660E0B6EFF0EA4
:1056F8000C6EBD0E0D6E5CEC51F00B500C1007E1FA
:10570800CC0E126E7AEC4BF012500101976FD30E4B
:105718000B6EFF0E0C6EBD0E0D6E5CEC51F00B5057
:105728000C1006E1CC0E126E7AEC4BF01250726E31
:105738000001E56BE66BAE0E5A6E5B6A6D0E5C6E31
:10574800FF0E5D6EE5C05EF0E6C05FF0A1EC58F0BC
:10575800AE0E0B6E0C6ABD0E0D6E5CEC51F00B506C
:105768000C1018E10F0E0001E503F3CFACF0F4CFF5
:10577800ADF0E603F350AD27740EAC250B6E0C0E9E
:10578800AD210C6ECC0E0D6E0E6A106A0F0E0F6EE8
:105798002CEC56F00001E54BE62BE6BFCCD7E651E2
:1057A80003E1100EE55DC7E3E66B010EE56FAE0E93
:1057B8005A6E5B6A740E5C6EFF0E5D6EE5C05EF03D
:1057C800E6C05FF0A1EC58F0AE0E0B6E0C6ABD0E91
:1057D8000D6E5CEC51F00B500C1018E10F0E00012F
:1057E800E503F3CFACF0F4CFADF0E603F350AD270B
:1057F800640EAC250B6E0D0EAD210C6ECC0E0D6E2D
:105808000E6A106A0F0E0F6E2CEC56F00001E54B75
:10581800E62BE6BFCCD7E65103E1040EE55DC7E30E
:10582800E16BE26BE151BD0FD96EDA6ADF6AE151D3
:10583800CC0FD96EDA6A000EDF6EE14BE22BE2BFC5
:10584800F1D7E25103E10F0EE15DECE3DB6BDC6BBA
:1058580015D0740EE325D96E0A0EE421DA6E0A0E0D
:10586800DE1830E0740EE325D96E0A0EE421DA6EF4
:10587800200EDE1806E1DC6B010EDB6FDF6BE06BE0
:1058880021D0DB51DC1109E0740EE325D96E0A0E34
:10589800E421DA6EDF51CC0F08D0740EE325D96EFF
:1058A8000A0EE421DA6EDF51BD0FE16EE26ADFCF46
:1058B800E7FFE0BF05D0E05105E10F0EDF5D02E232
:1058C800DF4BE02BE34BE42BDD51E35DDE51E45984
:1058D80001E2CDD66A0E806FFD0E816F97C182F00E
:1058E800836B7DEC5AF0D70E0001806FFD0E816F3F
:1058F800FEC182F0836B7DEC5AF0C80E0001806F08
:10590800FD0E816FA0C182F0836B7DEC5AF000011F
:10591800E56BE66BF50E806FFC0E816FE5C082F0DB
:10592800E6C083F00F0EE503F3CFACF0F4CFADF093
:10593800E603F350AD27740EAC25846F0C0EAD2131
:10594800856F7DEC5AF00001E54BE62BE6BFE2D708
:10595800E65103E1100EE55DDDE3E46B010EE36F54
:10596800060E806FFD0E816FE3C082F0E4C083F005
:105978000F0EE303F3CFACF0F4CFADF0E403F35034
:10598800AD27640EAC25846F0D0EAD21856F7DECBF
:105998005AF00001E34BE42BE4BFE2D7E45103E102
:1059A800040EE35DDDE3490E806FFC0E816F7DEF31
:1059B8005AF00001C16B010EC06F300E806FF50EFA
:1059C800816FCFCF82F0836BCECF84F0856B73501D
:1059D800070D500EF324D96E010EF420DA6EDF5055
:1059E800866F876B7350070D510EF324D96E010E25
:1059F800F420DA6EDF50886F896B7350070D520EF2
:105A0800F324D96E010EF420DA6EDF508A6F8B6BA7
:105A18007350070D510EF324D96E010EF420DA6E7F
:105A2800DF50AC6FACC0ADF0AE6BAF6BB06B040EBB
:105A3800D890AD37AE37AF37B037E82EF9D77350B7
:105A4800070D500EF324D96E010EF420DA6EDF50E4
:105A5800B16FB1C0B2F0B36BB46BB56B050ED89033
:105A6800B237B337B437B537E82EF9D7AD51B225C9
:105A7800B66FAE51B321B76FAF51B421B86FB05103
:105A8800B521B96F7350070D520EF324D96E010E6C
:105A9800F420DA6EDF50B6258C6F000EB7218D6FBB
:105AA800000EB8218E6F000EB9218F6F7DEC5AF071
:105AB80089800001BA6BBB6BBC6BBD6BF7D07350B0
:105AC800200D000EF324626E020EF420636E740E35
:105AD800646E0A0E656E010E676E666AC80E686EA1
:105AE800696A16EC15F0870E0001806FF80E816F59
:105AF800C8C082F0C9C083F07DEC5AF0725066E0ED
:105B08007350070D530EF324D96E010EF420DA6E8C
:105B180078C1B1F079C1B2F07AC1B3F00001B06BCD
:105B2800000EB025B46F010EB121B56F000EB22181
:105B3800B66F000EB321B76FDE50B41947E1DE50DF
:105B4800B51944E1DE50B61941E1DE50B7193EE11E
:105B580014EC55F00FC0C4F010C0C5F011C0C6F069
:105B680012C0C7F0000EE8CF74FA2AEE75F0C7C06D
:105B7800DFFFE8CF76FA2AEE77F0C6C0DFFFE8CF7E
:105B880078FA2AEE79F0C5C0DFFFE8CF7AFA2AEE74
:105B98007BF0C4C0DFFF7D0E0001806FF60E816FC1
:105BA8002AEE75F0DF50826F836B2AEE77F0DF50B4
:105BB800846F856B2AEE79F0DF50866F876B2AEE4B
:105BC8007BF0DF50886F896B7DEC5AF00101FC9304
:105BD800C8C048F0C9C049F08EEC3DF048C0C2F0DA
:105BE80049C0C3F00001C251BA27C351BB23000EFC
:105BF800BC23BD2381AC5FD0C851C21903E1C95190
:105C0800C3190BE0B90E806FFE0E816FC2C082F01F
:105C1800C3C083F07DEC5AF04ED01BEC5AF0B6ECC2
:105C28005AF00B500C1011E0310E0001806FFE0E7F
:105C3800816FB6EC5AF00BC082F00CC083F07DEC9B
:105C48005AF0010E01019F6F36D00001BF6B050E9F
:105C5800BE6F1CD0680E0001AC6FE40EE82EFED7B4
:105C6800AC2FFCD700F0B6EC5AF00B500C100EE03D
:105C78000001C06BC16B8A0E806FFD0E816FBEC0C4
:105C880082F0BFC083F07DEC5AF008D00001BE0757
:105C9800D8A0BF07BE29DEE1BF29DCE1B6EC5AF087
:105CA8000B500C1003E00001C06BC16B0001C05128
:105CB800C11101E004D77D0E0001806FFA0E816FDB
:105CC800CFCF82F0836BCECF84F0856BBAC086F0DD
:105CD800BBC087F0BCC088F0BDC089F07DEC5AF02D
:105CE80001019F6B8990120043C024F044C025F045
:105CF8007AEC47F04D6E4D5001E08ED143C0D9FF8C
:105D080044C0DAFF030EDE1801E076D120EE05F07C
:105D18004350D9264450DA22DE0401E06DD12E0E1C
:105D280043240B6E000E44200C6E0E6A0D6A020EA0
:105D3800106E0F6AC2EC59F022EE2CF04350D926AF
:105D48004450DA22550EDF6E22EE2DF04350D9264C
:105D58004450DA22AA0EDF6E20EE2EF04350D926E8
:105D68004450DA22520EDF6E20EE2FF04350D9262F
:105D78004450DA22520EDF6E20EE30F04350D9261E
:105D88004450DA22610EDF6E20EE31F04350D926FE
:105D98004450DA22410EDF6E22EE12F04350D9262B
:105DA8004450DA22720EDF6E22EE13F04350D926E9
:105DB8004450DA22720EDF6E22EE14F04350D926D8
:105DC8004450DA22410EDF6E22EE15F04350D926F8
:105DD8004450DA22610EDF6E20EE0EF04350D926D1
:105DE8004450DA2212EE16F04350E1264450E222E3
:105DF800DFCFE7FF22EE17F04350D9264450DA22CE
:105E080010EE0EF04350E1264450E222E6CF45F072
:105E1800E5CF46F046C045F0466A4550DF6E22EEB3
:105E280018F04350D9264450DA2210EE0EF04350B1
:105E3800E1264450E222E6CF45F0E6CF46F0E6CF31
:105E480047F0E6CF48F0110E05D0D89048324732D7
:105E580046324532E82EF9D74550DF6E22EE19F06A
:105E68004350D9264450DA2210EE0EF04350E12672
:105E78004450E222E6CF45F0E6CF46F0E6CF47F0C1
:105E8800E6CF48F0190E05D0D8904832473246324E
:105E98004532E82EF9D74550DF6E20EE0AF0435020
:105EA800D9264450DA2212EE1AF04350E126445023
:105EB800E222DFCFE7FF22EE1BF04350D926445001
:105EC800DA2210EE0AF04350E1264450E222E6CFEF
:105ED80045F0E5CF46F046C045F0466A4550DF6ECE
:105EE80022EE1CF04350D9264450DA2210EE0AF074
:105EF8004350E1264450E222E6CF45F0E6CF46F093
:105F0800E6CF47F0E6CF48F0110E05D0D8904832DA
:105F1800473246324532E82EF9D74550DF6E22EE39
:105F28001DF04350D9264450DA2210EE0AF04350AF
:105F3800E1264450E222E6CF45F0E6CF46F0E6CF30
:105F480047F0E6CF48F0190E05D0D89048324732CE
:105F580046324532E82EF9D74550DF6E20EE1AF06A
:105F68004350D9264450DA22DECF45F0DECF46F042
:105F7800DECF47F0DECF48F04528496E000E4620B8
:105F88004A6E000E47204B6E000E48204C6E20EEE5
:105F98002AF04350D9264450DA2249C0DEFF4AC0CD
:105FA800DEFF4BC0DEFF4CC0DEFF2E0E43241A6E10
:105FB800000E44201B6E20EE2AF04350D926445090
:105FC800DA22DECF1CF0DECF1DF0DECF1EF0DECFF2
:105FD8001FF0216A010E206E20EE01F04350D926F1
:105FE8004450DA22DF5075EC4CF020EE05F04350B7
:105FF800D9264450DA22DF6A1A6A1B6A1C6A20EE24
:1060080001F04350D9264450DA22DF5011EC23F036
:10601800000902E0010E4D6E4D50120089806B6A36
:10602800E90E0001806FF60E816FCFCF82F0836B8F
:10603800CECF84F0856B7350140D070EF324D96E00
:10604800010EF420DA6EDECF86F0DECF87F0DECFE9
:1060580088F0DECF89F07350140D070EF324D96E43
:10606800010EF420DA6EDECF8AF0DECF8BF0DECFC1
:106078008CF0DECF8DF07DEC5AF0B2EC41F0CAC066
:10608800B3F1CBC0B4F10101B351B41105E0B3C110
:10609800EAF0B4C1EBF01200716AAE6BAF6BB06B93
:1060A800B16BAD6B010EAC6FB76B0DD1B56BB66B49
:1060B8001CD0B6EC5AF00B500C1013E0B70E0B6E58
:1060C800010E0C6E35EC52F00101AB6F000E71241D
:1060D800D96EDA6A030EDA22ABC1DFFF712AB54B3B
:1060E800B62B0101B7AB81AC04D0B6BFE2D7B60579
:1060F800E0E3B5C1ECF0B6C1EDF0000E0001EDBF74
:10610800FF0EEE6FEF6FEC510101AE270001ED516C
:106118000101AF230001EE510101B0230001EF514D
:106128000101B1237350140D0F0EF324D96E010E23
:10613800F420DA6EDE50AE5DDE50AF59DE50B05955
:10614800DE50B15902E3AC6BAD6BB7AB02D0AC6BB0
:10615800AD6B81BC02D0AC6BAD6B71500EE0E20E42
:106168000001806FFA0E816FB3C182F0B4C183F071
:1061780071C084F0856B7DEC5AF00101B6BF02D086
:10618800B60519E2000E71240B6E0C6A030E0C2280
:10619800FF0E7124D96EDA6A020EDA22DF500D6E14
:1061A8000E6A715000080F6E000ED8A0E82A010888
:1061B800106EB3EC48F072505BE07350140D070E8C
:1061C800F324D96E010EF420DA6E78C1F1F079C1AA
:1061D800F2F07AC1F3F00001F06B000EF025F46FD5
:1061E800010EF121F56F000EF221F66F000EF3217A
:1061F800F76FDE50F4193CE1DE50F51939E1DE5055
:10620800F61936E1DE50F71933E101C3BBF103C3D8
:10621800BAF105C3B9F107C3B8F1B8C10EF0B9C1F5
:106228000FF0BAC110F0BBC111F0D5EC56F0010E59
:106238000001806FF50E816FCFCF82F0836BCECFD8
:1062480084F0856B2AEE74F0DF50866F876B2AEE38
:1062580075F0DF50886F896B2AEE76F0DF508A6F11
:106268008B6B2AEE77F0DF508C6F8D6B7DEC5AF0DC
:106278006BEC54F0E1510101B26FB25124E0120EFF
:106288000001806FFB0E816FB2C182F0836B7DECE1
:106298005AF0010E6B6E7350140D130EF324D96E61
:1062A800010EF420DA6E7350140D130EF324E16E10
:1062B800010EF420E26EE7500409DF6E6BC0EAF0CD
:1062C8000001EB6B1200AC51AD1101E0EFD6E60E08
:1062D8000001806FF50E816FCFCF82F0836BCECF38
:1062E80084F0856BAEC186F0AFC187F0B0C188F08D
:1062F800B1C189F07DEC5AF082A402D0010E6B6E18
:1063080089900001EA6BEB6B12001550D96EDA6ABE
:10631800DECF22F0DDCF23F002D0224A232A22C08A
:10632800F6FF23C0F7FF000EF86E0F0EF76403D0D8
:106338000800F55005D0F6CFE9FFF7CFEAFFEF5098
:106348002F0AEBE022C0F6FF23C0F7FF000EF86E1D
:106358000F0EF76403D00800F55005D0F6CFE9FF1B
:10636800F7CFEAFFEF505C0AD8E020EE14F01350A4
:10637800D9261450DA22DECF24F0DDCF25F024C050
:106388000BF025C00CF00E6A200E0D6E106A0B0E75
:106398000F6EC2EC59F01E6A1EC026F0276A26C08E
:1063A8001CF027C01DF0206A080E1F6E1C50222406
:1063B800166E1D502320176E16C0F6FF17C0F7FF84
:1063C800000EF86E0F0EF76403D00800F55005D0E4
:1063D800F6CFE9FFF7CFEAFFEF50286E1C4A1D2AD7
:1063E800200E2864A7D02F0E281801E1A3D05C0E38
:1063F800281801E19FD02E0E281805E01F50265CB2
:106408002050275814E3080E1F182010D8A4060C93
:106418002E0E281801E0060C276A080E266E206A40
:106428000B0E1F6ED8901E36D8901E36BFD77F0E23
:10643800286402D0030E1E12800E286403D09F0E1B
:10644800286406D0DF0E28644CD0FD0E286049D0A1
:106458001C502224166E1D502320176E16C0F6FFFE
:1064680017C0F7FF000EF86E0F0EF76403D0080090
:10647800F55005D0F6CFE9FFF7CFEAFFEF50216ED0
:106488001C4A1D2A3F0E216403D07E0E216406D0CB
:106498007F0E2164060CFD0E2160060C1668176835
:1064A8001FC018F020C019F01650182617501922CE
:1064B8001850265C1950275801E3060C265024244E
:1064C800D96E27502520DA6E28C0DFFF264A272AF2
:1064D80026502424D96E27502520DA6E21C0DFFFEC
:1064E80026D0220E0B6EFE0E0C6E28C00DF00E6A22
:1064F80085EC58F00B500C1001E0060C400E286497
:1065080005D05B0E286002D01E8209D0600E286478
:1065180006D07B0E286003D01E80200E285E2650F1
:106528002424D96E27502520DA6E28C0DFFF264A9A
:10653800272A3CD71C502224166E1D502320176E84
:106548001550D96EDA6A16C0DEFF17C0DDFF200EBF
:10655800286403D01A6A1B6A03D01B6A040E1A6ED9
:106568001AC028F02650271001E1060C24C0D9FFD4
:1065780025C0DAFFE50EDE1806E124C0D9FF25C0E4
:10658800DAFF050EDF6E080E1F18201004E1D89000
:106598001E36D8901E361E50030BE80601E12888E7
:1065A8001E500C0B040A01E1288620EE0BF0245043
:1065B800D9262550DA2228C0DFFF000C8E518F1112
:1065C8009011911128E120EE0AF08C51D9268D51B5
:1065D800DA22DECF97F0DECF98F0DECF99F0DECF6B
:1065E8009AF09751981199119A110FE020EE12F034
:1065F8008C51D9268D51DA22DE50975DDE5098599C
:10660800DE509959DE509A5952E3010E976F986BF4
:10661800996B9A6B4CD08CC044F08DC045F08EC0FD
:1066280046F08FC047F090C048F091C049F0E7ECC1
:106638001EF044C09FF045C0A0F046C0A1F047C07E
:10664800A2F00001A251A111A01109E1020E9F5D63
:1066580006E2010E8C6F8D6B8E6B8F6B000C9F2981
:106668000FE1A0290DE1A1290BE1A22909E19FC0B1
:106678008CF0A0C08DF0A1C08EF0A2C08FF01200E7
:1066880020EE12F08C51D9268D51DA22DE509F5D12
:10669800DE50A059DE50A159DE50A259E8E38EC061
:1066A80097F08FC098F090C099F091C09AF097C079
:1066B8009BF098C09CF099C09DF09AC09EF09B2BCF
:1066C800000E9C239D239E2320EE12F08C51D92688
:1066D8008D51DA22DE509B5DDE509C59DE509D596B
:1066E800DE509E5911E3020E9B6F9C6B9D6B9E6B57
:1066F8009A519911981108E1020E975D05E28C6B89
:106708008D6B8E6B8F6B12008CC044F08DC045F082
:106718009BC046F09CC047F09DC048F09EC049F021
:10672800E7EC1EF044C09FF045C0A0F046C0A1F0C1
:1067380047C0A2F000019F51A011A111A2111AE0B7
:106748009F2906E1A02904E1A12902E1A2298FE0FD
:106758009F05A011A111A2118AE097519B19AFE1E1
:1067680098519C19ACE199519D19A9E19A519E192A
:10677800C6E0A5D78CC044F08DC045F09BC046F05C
:106788009CC047F09DC048F09EC049F04A684B68DD
:106798004C680F0E4D6E2EEC1AF0966F96511CE158
:1067A8008E518F119011911117E08CC044F08DC05B
:1067B80045F08EC046F08FC047F090C048F091C0B9
:1067C80049F09BC04AF09CC04BF09DC04CF09EC065
:1067D8004DF02EEC1AF0966F965130E120EE0AF04B
:1067E8008C51D9268D51DA229BC0DEFF9CC0DEFF7A
:1067F8009DC0DEFF9EC0DEFF20EE0EF08C51D92634
:106808008D51DA22DE2806E1DE2804E1DE2802E1E5
:10681800DE2821E020EE0EF08C51D9268D51DA22A7
:10682800DE06000EDE5ADE5ADE5A20EE05F08C51E6
:10683800D9268D51DA22000EDB800DD0960507E0AF
:10684800010E9B6F000E9C6B9D6B9E6B04D09B6929
:106858009C699D699E699BC08CF09CC08DF09DC011
:106868008EF09EC08FF0120020EE04F06250D92600
:106878006350DA2264C0DEFF65C0DDFF20EE06F05B
:106888006250D9266350DA22DECF99F0DECF9AF033
:10689800DECF9BF0DECF9CF0000199059A119B1189
:1068A8009C11D8B4020C62C0D9FF63C0DAFF10EEA5
:1068B80012F0DE50E126DD50E222E650995DE65006
:1068C8009A59E6509B59E6509C5901E3020C99519C
:1068D8009A119B119C1121E162C0D9FF63C0DAFFB4
:1068E800DECF8CF0DDCF8DF08CC0D9FF8DC0DAFF04
:1068F800030EDE1812E162C0D9FF63C0DAFF10EEA2
:1069080022F0DE50E126DD50E222E6CF99F0E6CF14
:106918009AF0E6CF9BF0E6CF9CF099519A119B1123
:106928009C1123E162C0D9FF63C0DAFF10EE08F0C2
:10693800DE50E126DD50E222E650645CE650655800
:1069480001E3020C62C0D9FF63C0DAFF10EE22F047
:10695800DE50E126DD50E222E6CF95F0E6CF96F054
:10696800E6CF97F0E6CF98F074D062C0D9FF63C045
:10697800DAFF10EE02F0DE50E126DD50E222E750A9
:10698800100DF3CF93F0F4CF94F044D062C0D9FF48
:1069980063C0DAFFDECF44F0DDCF45F099C046F0A2
:1069A8009AC047F09BC048F09CC049F0E7EC1EF045
:1069B80044C099F045C09AF046C09BF047C09CF08F
:1069C8000001992907E19A2905E19B2903E19C29FE
:1069D80001E1010C9C519B119A1104E1020E995D91
:1069E800D8A0020C62C0D9FF63C0DAFF10EE12F023
:1069F800DE50E126DD50E222E650995DE6509A59D4
:106A0800E6509B59E6509C5901E3020C9351645E91
:106A18009451655A9351645C94516558B7E262C0C9
:106A2800D9FF63C0DAFFDECF0BF0DDCF0CF099C0E1
:106A38000DF09AC00EF09BC00FF09CC010F071ECE6
:106A48004AF00BC095F00CC096F00DC097F00EC040
:106A580098F020EE0AF06250D9266350DA2299C0E5
:106A6800DEFF9AC0DEFF9BC0DEFF9CC0DEFF000198
:106A7800955196119711981101E1020C64C08CF0A0
:106A880065C08DF0040E8E6FD8908D338C338E2FA9
:106A9800FBD78C5195258F6F8D519621906F000EE5
:106AA8009721916F000E9821926F20EE0EF06250A0
:106AB800D9266350DA228FC0DEFF90C0DEFF91C076
:106AC800DEFF92C0DEFF0F0E64148C6F8D6B050E17
:106AD800D8908C378D37E82EFBD762C0D9FF63C0BA
:106AE800DAFFDECF8EF0DDCF8FF08C518E278D51FF
:106AF8008F232E0E8E27000E8F2320EE12F0625069
:106B0800D9266350DA228EC0DEFF8FC0DDFF000C6D
:106B1800000E0001F66F0A0EF56F000EF46F050EF9
:106B2800F36F28D1F66B140EF56F1CD1600E0C6E46
:106B3800FC0E0D6EABEC56F082B204D00001F66B81
:106B48001E0EF56F150E0001F26F4B0EF16FBE0EA3
:106B5800E82EFED7F12FFCD7F22FFAD700F002D19A
:106B6800C60E0C6EFE0E0D6EABEC56F0460E000116
:106B7800D26F080ED36F4B0ED46FFC0ED56FD66B49
:106B880011EC51F06C6E6C50FEEC56F06C50DAE182
:106B98000001F66B230ED5D7E60E0C6EFD0E0D6EBA
:106BA800ABEC56F0000E0001D26F020ED36F010E4F
:106BB800D46FFF0ED56F010ED66FCBEC17F06C6E4D
:106BC8006C50FEEC56F06C5009E101EC2BF0000E15
:106BD8005B6E020E5C6EF4EC58F06C6E6C50FEEC62
:106BE80056F0000E0001F66F280EF56F010197515F
:106BF8000CE1FD6B740E5A6E0C0E5B6E850E5C6EAE
:106C0800FE0E5D6EA1EC58F00DD08C0E0001806F69
:106C1800F80E816F97C182F0836BFDC184F0856B9C
:106C28007DEC5AF0F50E0001806FFD0E816F0101B9
:106C3800FD510F0D740EF3240001826F0C0EF42029
:106C4800836F7DEC5AF07ED7710E806FFB0E816FDB
:106C58000101FD510F0D740EF3240001826F0C0E1B
:106C6800F420836F7DEC5AF0000E0001D26F020E03
:106C7800D36F0101FD510F0D740EF3240001D46F81
:106C88000C0EF420D56F030ED66FCBEC17F06C6E9C
:106C98006C5004E10001F66B3C0EF56F040E6C18A5
:106CA80001E050D70001F66B320E4BD7D10E806F42
:106CB800FC0E816F0101FD510F0D740EF3240001CC
:106CC800826F0C0EF420836F7DEC5AF0000E0001E9
:106CD800D26F020ED36F0101FD510F0D740EF32414
:106CE8000001D46F0C0EF420D56F070ED66FCBECD5
:106CF80017F06C6E6C5001E025D70001F66B3C0E66
:106D080020D7870E806FFC0E816F0101FD510F0D9A
:106D1800740EF3240001826F0C0EF420836F7DEC57
:106D28005AF00001F06B010EEF6F010CF5C0F1F0A5
:106D3800F6C0F2F0F25116E1F1510A0A01E1F2D679
:106D48001E0A01E1F3D60A0A01E10AD73D0A01E168
:106D580023D70B0A01E178D7050A04E01F0AA6E049
:106D68000E0ACFE0140E0001F519F61103E0F3073F
:106D7800D8A0F407F4BF04D0F451D8E1F305D6E263
:106D8800EF6BF06B1200740E0101B76F0A0EB86F4B
:106D9800EAC00BF0EBC00CF0AFEC57F00B50010160
:106DA800AB6FCA0E0001A36FA46BA56BA66BA76B94
:106DB800A86B2CEC12F00101B46FB4510DE0B00EC9
:106DC8000001806FFA0E816F7DEC5AF00001CA6BEA
:106DD800CB6BCC6BCD6B1200CA0E626E636AB7C107
:106DE80064F0B8C165F0010E676E666AB20E686E2F
:106DF800010E696E16EC15F00101B46FB45108E08C
:106E0800B60E0001806FFB0E816F7DEC5AF0DED765
:106E1800B7C1D9FFB8C1DAFF800EDE1808E0170E37
:106E28000001806FFD0E816F7DEC5AF0CFD720EE08
:106E38000AF0B751D926B851DA22DF500001ED6FB8
:106E4800EC6B010120EE0BF0B751D926B851DA22CC
:106E5800DF500001EC250101B06F000E0001ED21AB
:106E68000101B16F9F0E0001806FFB0E816FB0C1F1
:106E780082F0B1C183F07DEC5AF0CA0E0001A36F15
:106E8800A46B0101B0510001ED6FEC6BECC0A5F0F3
:106E9800EDC0A6F0A76BA86B2CEC12F00101B46F43
:106EA800B45194E1CA0E626E636AB7C164F0B8C1A6
:106EB80065F0010E676E666AB20E686E010E696E45
:106EC80016EC15F00101B46FB45180E1B56BB66BE7
:106ED800EAC00BF0EBC00CF0B5C1ECF0B6C1EDF0B8
:106EE800050ED8900001EC37ED37E82EFAD7EC51B3
:106EF8000101B7250D6E0001ED510101B8210E6E9B
:106F0800ABC10FF0106AA7EC51F00B500C105DE10B
:106F1800B5C1ECF0B6C1EDF0050ED8900001EC3724
:106F2800ED37E82EFAD7B7C1EEF0B8C1EFF0EC5163
:106F3800EE27ED51EF230E0EEE25D96E000EEF2150
:106F4800DA6EDF50F16FF06BB5C1F2F0B6C1F3F055
:106F5800050ED890F237F337E82EFBD7B7C1F4F017
:106F6800B8C1F5F0F251F427F351F5230F0EF425CB
:106F7800D96E000EF521DA6EDF50F66FF76BF0511F
:106F8800F627F151F723F6C0ACF1F7C0ADF10101D6
:106F9800000EADBFFF0EAE6FAF6F040E0001806F25
:106FA800FE0E816FACC182F0ADC183F0AEC184F03A
:106FB800AFC185F07DEC5AF0ACC1CAF0ADC1CBF0E1
:106FC800AEC1CCF0AFC1CDF01200B54BB62BB6BFF9
:106FD8007FD7B65105E10F0EB55D01E3F7D678D737
:106FE800F5D6BA0E0001806FF50E816FCFCF82F013
:106FF800836BCECF84F0856B7350070D500EF3244E
:10700800D96E010EF420DA6EDF50866F876B7350ED
:10701800070D510EF324D96E010EF420DA6EDF50FD
:10702800886F896B7350070D520EF324D96E010EC9
:10703800F420DA6EDF508A6F8B6B7350070D510E98
:10704800F324D96E010EF420DA6EDF50E16FE1C04F
:10705800E2F0E36BE46BE56B040ED890E237E337BC
:10706800E437E537E82EF9D77350070D500EF324AF
:10707800D96E010EF420DA6EDF50E66FE6C0E7F055
:10708800E86BE96BEA6B050ED890E737E837E93724
:10709800EA37E82EF9D7E251E725EB6FE351E8210B
:1070A800EC6FE451E921ED6FE551EA21EE6F735081
:1070B800070D520EF324D96E010EF420DA6EDF505C
:1070C800EB258C6F000EEC218D6F000EED218E6F7D
:1070D800000EEE218F6F7DEC5AF08980DEEC54F0C3
:1070E80048C0F0F049C0F1F00001F1BF0AD0040E29
:1070F800F15D07E3000EF025F26FFC0EF121F36F4E
:1071080004D0F0C0F2F0F1C0F3F0725054E07350C4
:10711800070D530EF324D96E010EF420DA6E78C1F0
:10712800E6F079C1E7F07AC1E8F0E56B000EE525F5
:10713800E96F010EE621EA6F000EE721EB6F000E02
:10714800E821EC6FDE50E91936E1DE50EA1933E147
:10715800DE50EB1930E1DE50EC192DE101C3F7F0F8
:1071680003C3F6F005C3F5F007C3F4F0F4C00EF05E
:10717800F5C00FF0F6C010F0F7C011F0D5EC56F0DE
:107188000C0E0001806FF60E816F2AEE74F0DF504E
:10719800826F836B2AEE75F0DF50846F856B2AEE61
:1071A80076F0DF50866F876B2AEE77F0DF50886FB6
:1071B800896B7DEC5AF082B415D07350200D000E07
:1071C800F3240001A36F020EF420A46F000EA56F34
:1071D800030EA66F010EA86FA76BF20EA96FBEEC87
:1071E8000EF0EF6F0001EF5109E09A0E806FFD0E6F
:1071F800816FEFC082F0836B7DEC5AF0C90E0001FD
:10720800806FFA0E816FF2C082F0F3C083F07DECDC
:107218005AF06BEC3BF09F6B8990280E0001806F51
:10722800FD0E816FCFCF82F0836BCECF84F0856B5C
:107238007DEF5AF07350070D520EF324D96E010EEC
:10724800F420DA6EDF500001CA6FCAC0CBF0CC6BF5
:10725800CD6BCE6BCDC0CEF0CCC0CDF0CBC0CCF0DA
:10726800CB6B7350070D510EF324D96E010EF42029
:10727800DA6EDF50CF6FCFC0D0F0D16BD26BD36B4B
:107288000C0ED890D037D137D237D337E82EF9D76C
:107298007350070D500EF324D96E010EF420DA6EE8
:1072A800DF50D46FD4C0D5F0D66BD76BD86B0D0E2A
:1072B800D890D537D637D737D837E82EF9D7D05121
:1072C800D525D96FD151D621DA6FD251D721DB6FAD
:1072D800D351D821DC6FCB51D925DE6FCC51DA21BF
:1072E800DF6FCD51DB21E06FCE51DC21E16FC80E9D
:1072F800806FF80E816F73C082F0836B7350070D37
:10730800500EF324D96E010EF420DA6EDF50846F2C
:10731800856B7350070D510EF324D96E010EF420BE
:10732800DA6EDF50866F876B7350070D520EF324A9
:10733800D96E010EF420DA6EDF50886F896B7350B6
:10734800070D510EF324D96E010EF420DA6EDF50CA
:10735800CA6FCAC0CBF0CC6BCD6BCE6B040ED89085
:10736800CB37CC37CD37CE37E82EF9D77350070D4A
:10737800500EF324D96E010EF420DA6EDF50CF6F71
:10738800CFC0D0F0D16BD26BD36B050ED890D0376D
:10739800D137D237D337E82EF9D7CB51D025D46F90
:1073A800CC51D121D56FCD51D221D66FCE51D32119
:1073B800D76F7350070D520EF324D96E010EF420C7
:1073C800DA6EDF50D4258A6F000ED5218B6F000E40
:1073D800D6218C6F000ED7218D6F7DEC5AF0CD0E23
:1073E8000001806FFB0E816FDEC082F0DFC083F08A
:1073F800E0C084F0E1C085F0DEC086F0DFC087F031
:10740800E0C088F0E1C089F07DEC5AF07350200D9F
:10741800000EF3240001A36F020EF420A46FDEC057
:10742800A5F0DFC0A6F0E0C0A7F0E1C0A8F02CEC02
:1074380012F0DD6FDD5111E0420E806FFB0E816F9F
:10744800DEC082F0DFC083F0E0C084F0E1C085F0E8
:10745800DDC086F0876B7DEC5AF07350070D530E34
:10746800F324D96E010EF420DA6EDEC0DEFFDFC031
:10747800DEFFE0C0DEFFE1C0DEFF01019F6B899007
:1074880012000001AD6FA95102E0AFEC42F000011B
:10749800AC6BA85101E101D1040EAD1903E0140E43
:1074A800AD1909E10101926B846B856B0001A96B31
:1074B800070EA86F070C3F0EAD1907E1FD6B010120
:1074C800926B0001A86BA96B12005F0EAD1907E162
:1074D8000101936B926B0001A86BA96B12003F0E20
:1074E800AD6506D05F0EAD6103D0400EAD19F0E179
:1074F800400EAD1908E1010E0101936F926B000176
:10750800A86BA96B1200200EAD190CE1010EFD6FDE
:107518000101926B820E0001806FFF0E816F7DEC7E
:107528005AF0EDD7650EAD1909E1FD5107E00101EB
:10753800846B856B010E926F8980E1D76E0EAD1951
:1075480003E1020E0101926F700E0001AD1907E10F
:107558000101935104E0846B856B030E926F700EEA
:107568000001AD1908E1FD5106E089800101846B35
:10757800856B040E0ED0720EAD1901E08ED0FD5150
:1075880001E18BD089801C0E0101856F2A0E846F62
:10759800050E926FB4D7AD5111EC0BF00001AC6F32
:1075A80091D0240E806FFC0E816FADC082F0836B8A
:1075B8007DEC5AF089800001AD5101EC53F00001D7
:1075C800AC6F0101926B7ED089806E0E806FF80ED1
:1075D800816FCFCF82F0836BCECF84F0856B6BC089
:1075E80086F0876B7DEC5AF0740E0B6E0A0E0C6EEB
:1075F8000E6A0D6A010E106E0F6AB3EC48F00101B5
:10760800FC832AEE74F06BC0DFFF496A010E486EF6
:107618008EEC3DF0FC93080ED2D78990AC6B100E1F
:10762800806FF80E816FCFCF82F0836BCECF84F05E
:10763800856BADC086F0876B7DEC5AF043D0080EA1
:10764800AD1918E16F0E806FF70E816FCFCF82F002
:10765800836BCECF84F0856BADC086F0876B7DECF5
:107668005AF089900001AC6B6B6A0101926B846BD4
:10767800856B28D0090EAD1925E1750E806FF90EBE
:10768800816FCFCF82F0836BCECF84F0856BADC096
:1076980086F0876B7DEC5AF0E4D701019251000126
:1076A800AA6FAB6BAB510EE1AA510CE0010A01E1E4
:1076B80072D7030A01E175D7010A86E0070AADE02F
:1076C800010ABDE0ACC0A8F00001A96B120073501C
:1076D800070D520EF324D96E010EF420DA6EDF2A5C
:1076E8007350070D520EF324D96E010EF420DA6E92
:1076F8000F0EDF642FD07350070D520EF324D96E8E
:10770800010EF420DA6EDF6A7350070D510EF32470
:10771800D96E010EF420DA6EDF2A7350070D510E70
:10772800F324D96E010EF420DA6E010EDF6412D054
:107738007350070D510EF324D96E010EF420DA6E42
:10774800DF6A7350070D500EF324D96E010EF42032
:10775800DA6EDF2A7350070D520EF324D96E010E2C
:10776800F420DA6EDF500001CA6FCAC0CBF0CC6BD0
:10777800CD6BCE6BCDC0CEF0CCC0CDF0CBC0CCF0B5
:10778800CB6B7350070D510EF324D96E010EF42004
:10779800DA6EDF50CF6FCFC0D0F0D16BD26BD36B26
:1077A8000C0ED890D037D137D237D337E82EF9D747
:1077B8007350070D500EF324D96E010EF420DA6EC3
:1077C800DF50D46FD4C0D5F0D66BD76BD86B0D0E05
:1077D800D890D537D637D737D837E82EF9D7D051FC
:1077E800D525D96FD151D621DA6FD251D721DB6F88
:1077F800D351D821DC6FCB51D925DD6FCC51DA219B
:10780800DE6FCD51DB21DF6FCE51DC21E06F73508D
:10781800070D530EF324D96E010EF420DA6EDDC085
:10782800DEFFDEC0DEFFDFC0DEFFE0C0DEFF630E8E
:10783800806FFA0E816F73C082F0836B7350070DEF
:10784800500EF324D96E010EF420DA6EDF50846FE7
:10785800856B7350070D510EF324D96E010EF42079
:10786800DA6EDF50866F876B7350070D520EF32464
:10787800D96E010EF420DA6EDF50886F896B7DECCB
:107888005AF07350200D000EF3240001A36F020E6E
:10789800F420A46F7350070D530EF324D96E010E14
:1078A800F420DA6EDECFA5F0DECFA6F0DECFA7F0AB
:1078B800DECFA8F02CEC12F06A6E6A5019E0420E86
:1078C800806FFB0E816F7350070D530EF324D96E32
:1078D800010EF420DA6EDECF82F0DECF83F0DECF49
:1078E80084F0DECF85F06AC086F0876B7DEC5AF0B5
:1078F80001019F6B12000001F16B320E806FF60ED2
:10790800816F7350070D500EF324D96E010EF420C9
:10791800DA6EDF50826F836B7350070D510EF324BC
:10792800D96E010EF420DA6EDF50846F856B7350C8
:10793800070D520EF324D96E010EF420DA6EDF50D3
:10794800866F876B7350070D510EF324D96E010EA5
:10795800F420DA6EDF50E16FE1C0E2F0E36BE46B34
:10796800E56B040ED890E237E337E437E537E82EC5
:10797800F9D77350070D500EF324D96E010EF42079
:10798800DA6EDF50E66FE6C0E7F0E86BE96BEA6BAA
:10799800050ED890E737E837E937EA37E82EF9D700
:1079A800E251E725EB6FE351E821EC6FE451E9215F
:1079B800ED6FE551EA21EE6F7350070D520EF32477
:1079C800D96E010EF420DA6EDF50EB25886F000EB9
:1079D800EC21896F000EED218A6F000EEE218B6F6E
:1079E8007DEC5AF0898090D0DEEC54F048C0EFF07E
:1079F80049C0F0F00001F0BF06D0040EF05D03E3CB
:107A0800010EF16F03D0F4C0F2F0F36B82B414D01E
:107A18007350200D000EF324A36F020EF420A46F00
:107A2800000EA56F030EA66F010EA86FA76BF20ECE
:107A3800A96FBEEC0EF0F46FF45109E09A0E806F56
:107A4800FD0E816FF4C082F0836B7DEC5AF07250AA
:107A58004DE07350070D530EF324D96E010EF42038
:107A6800DA6E78C1E6F079C1E7F07AC1E8F0000192
:107A7800E56B000EE525E96F010EE621EA6F000EC1
:107A8800E721EB6F000EE821EC6FDE50E9192EE1DB
:107A9800DE50EA192BE1DE50EB1928E1DE50EC1933
:107AA80025E101C3F8F003C3F7F005C3F6F007C3F7
:107AB800F5F0F5C00EF0F6C00FF0F7C010F0F8C002
:107AC80011F0D5EC56F00C0E0001806FF60E816FA8
:107AD80000C382F0836B01C384F0856B02C386F018
:107AE800876B03C388F0896B7DEC5AF0C60E0001E2
:107AF800806FF90E816FF2C082F0F3C083F07DECE5
:107B08005AF06BEC3BF09F6B0001F15101E16CD72F
:107B18008990120001019C6B866B876B938693801A
:107B280093829384938895688A908A928A948A9893
:107B3800010E9B6F898E89B40ED0F1A707D0580E1D
:107B48000001806FF60E816F7DEC5AF001019B6B8E
:107B5800486A496A1200F2981A0EE82EFED700D039
:107B6800D3D081A881BA14D09F0E0001806FFE0E79
:107B7800816F010E80A0000E826F836B010E89A0B9
:107B8800000E846F856B9CC186F0876B7DEC5AF084
:107B980081B809D095689380130E0001806FFE0E9E
:107BA800816F7DEC5AF081B80BD0130E0001806F05
:107BB800FE0E816F7DEC5AF0630E01019C6FAAD016
:107BC800100E0101746F270E756F766B776B86D078
:107BD80081B281A410D07407000E755B765B775B69
:107BE800742906E1752904E1762902E17729D8A4E8
:107BF8008BD0620E69D0010E67D081A885D0020EA5
:107C080063D04A684B6848C04CF049C04DF04A50B0
:107C18004C264B504D2286514C1805E187514D1882
:107C280002E1FCB3939A740E8625D96E0A0E872159
:107C3800DA6EDF1C8C6E864B872B956A030E1ED07E
:107C4800100E746F270E756F766B776B5DD081B2EF
:107C58000DD07407000E755B765B775B742908E1BD
:107C6800752906E1762904E1772902E1040E9C6F63
:107C780081A24AD0040E28D09390050E9C6FE0D7BD
:107C8800938481B40DD07407000E755B765B775BC7
:107C9800742908E1752906E1762904E1772902E1CA
:107CA800060E9C6F81A430D0060E0ED0938A938066
:107CB80095684850865D8751800A4A6E4950800A07
:107CC8004A5899E3630E01019C6F1ED0A00E000173
:107CD800806FFF0E816F7DEC5AF0F4D79C514A6E8D
:107CE8004B6A4B5011E14A5001E172D7010A85E015
:107CF800030A87E0010AABE0070ABEE0010AC0E018
:107D0800030AD4E0640AE2E0630E01019C1902E070
:107D180081BC27D7F292F2889B6B938093829384DD
:107D28009388938A9568899E86C148F087C149F0EF
:107D3800120020EE04F04450D9264550DA22DF6ABA
:107D480020EE2AF04450D9264550DA22DE68DE6853
:107D5800DE68DD6844C039F045C03AF046C03BF003
:107D680047C03CF048C03DF049C03EF0C3EC50F07D
:107D7800000901E0030C22EE2DF04450D9264550AD
:107D8800DA22DF504B6E4A6A22EE2CF04450D92694
:107D98004550DA22DF504A12550E4A1803E1AA0E5E
:107DA8004B1801E0020C20EE65F04450D9264550EE
:107DB800DA22DF504B6E4A6A20EE66F04450D9262C
:107DC8004550DA22DF504C6E4CC04DF04E6A4F6A77
:107DD800506A4EC050F04DC04FF04E6A4D6A20EECA
:107DE80067F04450D9264550DA22DF50516E51C011
:107DF80052F0536A546A556A52C055F0546A536A2D
:107E0800526A4D505210566E4E505310576E4F5086
:107E18005410586E50505510596E4A5056105A6E9C
:107E28004B5057105B6E000E58105C6E000E5910C8
:107E38005D6E20EE64F04450D9264550DA22DF50BA
:107E48005A105E6E5B505F6E5C50606E5D50616E86
:107E58005E50626E5F50636E6050646E656A460E77
:107E6800621808E1410E631805E1540E64186510A4
:107E780001E1000C20EE81F04450D9264550DA2269
:107E8800DF504B6E4A6A20EE82F04450D9264550A6
:107E9800DA22DF504C6E4CC04DF04E6A4F6A506A81
:107EA8004EC050F04DC04FF04E6A4D6A20EE83F040
:107EB8004450D9264550DA22DF50516E51C052F055
:107EC800536A546A556A52C055F0546A536A526AE2
:107ED8004D505210566E4E505310576E4F5054100E
:107EE800586E50505510596E4A5056105A6E4B5095
:107EF80057105B6E000E58105C6E000E59105D6EC8
:107F080020EE80F04450D9264550DA22DF505A102E
:107F18005E6E5B505F6E5C50606E5D50616E5E5071
:107F2800626E5F50636E6050646E656A460E6218DA
:107F380008E1410E631805E1540E6418651001E16B
:107F4800000C010C4EC00CF04FC00DF0EEEC51F0DF
:107F5800546E545001E0FDD020EE04F04E50D92666
:107F68004F50DA22DFAAF5D04EC0D9FF4FC0DAFF52
:107F7800DECF39F0DDCF3AF020EE1AF04E50D92698
:107F88004F50DA22DECF3BF0DECF3CF0DECF3DF0C3
:107F9800DECF3EF0C3EC50F0546E545001E0D9D01F
:107FA80020EE1EF04E50D9264F50DA22DECF59F07F
:107FB800DDCF5AF020EE0BF05950D9265A50DA226C
:107FC800000EDB8A20EE0AF04E50D9264F50DA22F6
:107FD80010EE1CF05950E1265A50E222DFCFE7FF9D
:107FE80020EE1DF05950D9265A50DA2210EE0AF028
:107FF8004E50E1264F50E222E6CF50F0E5CF51F047
:1080080051C050F0516A5050DF6E20EE1EF05950AA
:10801800D9265A50DA2210EE0AF04E50E1264F5077
:10802800E222E6CF50F0E6CF51F0E6CF52F0E6CFAD
:1080380053F0110E05D0D89053325232513250328B
:10804800E82EF9D75050DF6E20EE1FF05950D92690
:108058005A50DA2210EE0AF04E50E1264F50E22232
:10806800E6CF50F0E6CF51F0E6CF52F0E6CF53F02E
:10807800190E05D0D8905332523251325032E82E70
:10808800F9D75050DF6E59C00BF05AC00CF020EEF3
:108098000EF04E50D9264F50DA22DECF0DF0DECF4B
:1080A8000EF0DECF0FF0DECF10F08EEC57F0556AF1
:1080B800566A210E576E460E586E20EE16F059502D
:1080C800D9265A50DA22DF6A20EE17F05950D926FD
:1080D8005A50DA2256C0DFFF20EE18F05950D92640
:1080E8005A50DA2257C0DFFF20EE19F05950D9262E
:1080F8005A50DA2258C0DFFF20EE12F05950D92624
:108108005A50DA22DF6A20EE13F05950D9265A5015
:10811800DA22DF6A20EE04F04E50D9264F50DA22D8
:10812800DF0EDF164EC0D9FF4FC0DAFF10EE04F0A5
:10813800DE50E126DD50E222010EE76E4EC0D9FF87
:108148004FC0DAFFDECF43F0DDCF44F078EC2EF0FD
:10815800546E545012000B0E0001806FF70E816FA1
:10816800CFCF82F0836BCECF84F0856B73C086F05F
:10817800876B7DEC5AF00101FC83740E0B6E0A0EBE
:108188000C6E0E6A0D6A010E106E0F6AB3EC48F0A1
:108198002AEE74F073C0DFFFFF0EE8CF75FA735054
:1081A800140D130EF324D96E010EF420DA6EDFA439
:1081B80003D0010EE8CF78FA7350140D130EF32490
:1081C800D96E010EF420DA6EDFA003D0020EE8CFDC
:1081D8007AFA7350140D130EF324D96E010EF4209D
:1081E800DA6EDFA203D0020EE8CF7AFA7350140DCC
:1081F800130EF324D96E010EF420DA6EDFA603D035
:10820800800EE8CF79FA82A403D0080EE8CF7AFA74
:10821800506A516AB00E0001806FF70E816FCFCFA0
:1082280082F0836BCECF84F0856B50C086F051C04E
:1082380087F0760E5024D96E0A0E5120DA6EDF5080
:10824800886F896B7DEC5AF06C0E5024D96E010E44
:108258005120DA6EDF1C4F6E760E5024D96E0A0E4E
:108268005120DA6E760E5024E16E0A0E5120E26E2D
:10827800E7504F14DF6E5F0E0001806FFF0E816FB5
:10828800760E5024D96E0A0E5120DA6EDF50826FB6
:10829800836B7DEC5AF0504A512A51BEBBD75150DE
:1082A80003E1070E505CB6E37350140D130EF3246C
:1082B800D96E010EF420DA6EDF506B6E7350140D18
:1082C800010EF324D96E010EF420DA6EDF504E6EE3
:1082D8004EC07FFA7350140D020EF324D96E010EAE
:1082E800F420DA6EDF504E6E4EC080FA7350140DD3
:1082F800030EF324D96E010EF420DA6EDF504E6EB1
:108308004EC081FA7350140D040EF324D96E010E79
:10831800F420DA6EDF504E6E4EC082FA7350140DA0
:10832800050EF324D96E010EF420DA6EDF504E6E7E
:108338004EC083FA7350140D060EF324D96E010E45
:10834800F420DA6EDF504E6E4EC084FA496A140E7D
:10835800486E8EEC3DF0FC93899012007350140D1A
:10836800070EF324D96E010EF420DA6EDECFDDF0AD
:10837800DECFDEF0DECFDFF0DECFE0F08D0E0001E5
:10838800806FF50E816FCFCF82F0836BCECF84F0F4
:10839800856BDDC086F0DEC087F0DFC088F0E0C006
:1083A80089F0DDC08AF0DEC08BF0DFC08CF0E0C061
:1083B8008DF07DEC5AF07350140D070EF324D96E2E
:1083C800010EF420DA6E7350140D0B0EF324E16ED7
:1083D800010EF420E26EDE50E65CDE50E658DE5018
:1083E800E658DE50E6581CE2BF0E0001806FFC0E16
:1083F800816F7DEC5AF0010E6B6E7350140D130EE5
:10840800F324D96E010EF420DA6E7350140D130E96
:10841800F324E16E010EF420E26EE7500409DF6EEA
:108428007350140D0F0EF324D96E010EF420DA6E7A
:10843800DECFCCF0DECFCDF0DECFCEF0DECFCFF08A
:108448007350140D070EF324D96E010EF420DA6E62
:10845800DECFD0F0DECFD1F0DECFD2F0DECFD3F05A
:108468000001CC51D025D46FCD51D121D56FCE513B
:10847800D221D66FCF51D321D76F7350140D0B0E65
:10848800F324D96E010EF420DA6ED451DE5CD55196
:10849800DE58D651DE58D751DE581BE2AD0E806F3C
:1084A800FC0E816F7DEC5AF0010E6B6E7350140D4B
:1084B800130EF324D96E010EF420DA6E7350140DE6
:1084C800130EF324E16E010EF420E26EE750040966
:1084D800DF6E6B6A7350200D000EF3240001A36F4A
:1084E800020EF420A46FDDC0A5F0DEC0A6F0DFC048
:1084F800A7F0E0C0A8F02CEC12F0DC6FDC5126E00D
:10850800420E806FFB0E816FDDC082F0DEC083F00B
:10851800DFC084F0E0C085F0DCC086F0876B7DECBE
:108528005AF0010E6B6E7350140D130EF324D96EAE
:10853800010EF420DA6E7350140D130EF324E16E5D
:10854800010EF420E26EE7500409DF6E6BC0CAF03A
:108558000001CB6B1200736A736A030E736401D057
:10856800EAD0735004E10001A66BA76B04D00001A8
:10857800A76B010EA66F7350140D130EF324D96E5A
:10858800010EF420DA6EDF6A7350140D000EF32426
:10859800D96E010EF420DA6EDF6A7350140D070EDF
:1085A800F324D96E010EF420DA6EDE6ADE6ADE6A22
:1085B800DD6A0D0EA603F3CF48F0F4CF49F0A70308
:1085C800F3504926D10E4824D96E020E4920DA6E9E
:1085D800DF504A6E4AC04BF04C6A4D6A4E6A4DC035
:1085E8004EF04CC04DF04BC04CF04B6A0D0EA6033C
:1085F800F3CF4FF0F4CF50F0A703F3505026D00E2E
:108608004F24D96E020E5020DA6EDF50516E51C0E1
:1086180052F0536A546A556A53C055F052C054F028
:10862800536A526A0D0EA603F3CF56F0F4CF57F0F3
:10863800A703F3505726CF0E5624D96E020E5720A3
:10864800DA6EDF50586E58C059F05A6A5B6A5C6A35
:1086580059C05CF05B6A5A6A596A0D0EA603F3CFDB
:108668005DF0F4CF5EF0A703F3505E26CE0E5D24D6
:10867800D96E020E5E20DA6EDF5059245F6E000E4E
:108688005A20606E000E5B20616E000E5C20626EE8
:1086980052505F24636E53506020646E54506120C2
:1086A800656E55506220666E4B506324676E4C5061
:1086B8006420686E4D506520696E4E5066206A6E63
:1086C8007350140D0B0EF324D96E010EF420DA6EDC
:1086D80067C0DEFF68C0DEFF69C0DEFF6AC0DEFF7C
:1086E800900E806FF70E816F73C082F0836B7350AA
:1086F800140D0B0EF324D96E010EF420DA6EDECFC2
:1087080084F0DECF85F0DECF86F0DECF87F07350C1
:10871800140D0B0EF324D96E010EF420DA6EDECFA1
:1087280088F0DECF89F0DECF8AF0DECF8BF07DECEB
:108738005AF0732A12D70101936B0001FD6B0101F6
:10874800926B846B856B020E6B6E8990020C81A60E
:1087580004D0350E486EFC0E03D0B50E486EFF0EE1
:10876800496E81AA04D0350E4A6EFC0E03D0B00EB5
:108778004A6EFF0E4B6E81A804D0350E4C6EFC0E6F
:1087880003D0BA0E4C6EFF0E4D6E81AE04D0350E7E
:108798004E6EFC0E03D0BF0E4E6EFF0E4F6E81ACB8
:1087A80004D0350E506EFC0E03D0AB0E506EFF0E8B
:1087B800516E81A404D0350E526EFC0E03D0C90E42
:1087C800526EFF0E536E81A204D0350E546EFC0E0D
:1087D80003D0CE0E546EFF0E556E81A004D0350E18
:1087E800566EFC0E03D0C40E566EFF0E576E83AE47
:1087F80004D0350E586EFC0E03D0F80E586EFF0EDE
:10880800596E83AC04D0350E5A6EFC0E03D0F50EAB
:108818005A6EFF0E5B6E83AA04D0350E5C6EFC0E9A
:1088280003D0F20E5C6EFF0E5D6E83A804D0350E89
:108838005E6EFC0E03D0EF0E5E6EFF0E5F6E83A6BB
:1088480004D0350E606EFC0E03D0EC0E606EFF0E89
:10885800616E83A404D0350E626EFC0E03D0E90E5F
:10886800626EFF0E636E83A204D0350E646EFC0E3A
:1088780003D0E60E646EFF0E656E83A004D0350E3D
:10888800666EFC0E03D0E30E666EFF0E676E1A0E60
:108898000001806FF40E816F831C826F836B81CF20
:1088A80084F0856B66C086F067C087F064C088F086
:1088B80065C089F062C08AF063C08BF060C08CF03C
:1088C80061C08DF05EC08EF05FC08FF05CC090F02C
:1088D8005DC091F05AC092F05BC093F058C094F01C
:1088E80059C095F056C096F057C097F054C098F00C
:1088F80055C099F052C09AF053C09BF050C09CF0FC
:1089080051C09DF04EC09EF04FC09FF04CC0A0F0EB
:108918004DC0A1F04AC0A2F04BC0A3F048C0A4F0DB
:1089280049C0A5F07DEF5AF0A20E0001806FF60E47
:10893800816F7350070D500EF324D96E010EF42089
:10894800DA6EDF50826F836B7350070D510EF3247C
:10895800D96E010EF420DA6EDF50846F856B735088
:10896800070D520EF324D96E010EF420DA6EDF5093
:10897800866F876B7350070D510EF324D96E010E65
:10898800F420DA6EDF50AC6FACC0ADF0AE6BAF6BFD
:10899800B06B040ED890AD37AE37AF37B037E82E8E
:1089A800F9D77350070D500EF324D96E010EF42039
:1089B800DA6EDF50B16FB1C0B2F0B36BB46BB56BA8
:1089C800050ED890B237B337B437B537E82EF9D794
:1089D800AD51B225B66FAE51B321B76FAF51B421C7
:1089E800B86FB051B521B96F7350070D520EF3240B
:1089F800D96E010EF420DA6EDF50B625886F000EAE
:108A0800B721896F000EB8218A6F000EB9218B6FCC
:108A18007DEC5AF089800001BC6BBD6BBE6BBF6BEF
:108A28007350200D000EF324626E020EF420636E64
:108A3800740E646E0A0E656E010E676E666AC10E6C
:108A4800686E696A16EC15F00001C06F200E806F21
:108A5800F90E816FC0C082F0836BC1C084F0C2C0C0
:108A680085F07DEC5AF00101FC93C1C048F0C2C00A
:108A780049F08EEC3DF048C0BAF049C0BBF00001A7
:108A8800BA51BC27BB51BD23000EBE23BF23E30E42
:108A9800806FFC0E816FBCC082F0BDC083F0BEC089
:108AA80084F0BFC085F07DEC5AF001019F6B89907E
:108AB80012001B6E1B5001E0010C74A202D074500E
:108AC8001200000E36EC5AF00A0E266E03D0A3EC04
:108AD8005AF026062650FBE1236A000E146A156A2E
:108AE800166A176ABDEC58F0E80601E097D0AA0E9E
:108AF800146E010E156E166A176A080EBDEC58F052
:108B0800E80651E1266A26501C0FD96EDA6AA3ECF2
:108B18005AF0DF6E262A030E2664F5D71E047EE17E
:108B2800AA0E1F187BE1030E256EE80E246E15D0E1
:108B3800146A156A166A400E176EA90EBDEC58F035
:108B480000090EE00B0E1A6E620EE82EFED71A2EE2
:108B5800FCD700D02406D8A0250624502510E8E12B
:108B6800245025105BE0146A156A166A176A3A0ED3
:108B7800BDEC58F0000952E1266A26501C0FD96E48
:108B8800DA6AA3EC5AF0DF6E262A030E2664F5D7BC
:108B98001CBC03D0216A040E02D0216A0C0E206E80
:108BA80020C023F03BD0146A156A166A176AA90E0A
:108BB800BDEC58F01A6E020E1A6003D0236EA90E8F
:108BC80002D0010E236E226E030E256EE80E246E6F
:108BD80014D0146A156A166A176A2250BDEC58F048
:108BE80000090EE00B0E1A6E620EE82EFED71A2E42
:108BF800FCD700D02406D8A0250624502510E9E18A
:108C0800245025100AE0146A020E156E166A176AB7
:108C1800100EBDEC58F0000901E0236A23C06EF085
:108C2800BBEC5AF0235001E14AD7749048D7BEC034
:108C3800F6FFBFC0F7FF000EF86E0F0EF76403D003
:108C48000800F55005D0F6CFE9FFF7CFEAFFEF505F
:108C58002F0A13E0BEC0F6FFBFC0F7FF000EF86E84
:108C68000F0EF76403D00800F55005D0F6CFE9FFE2
:108C7800F7CFEAFFEF505C0A03E10001BE4BBF2BC0
:108C8800000120EE06F0BC51D926BD51DA22DE6A79
:108C9800DE6ADE6ADD6ABEC0F6FFBFC0F7FF000EFF
:108CA800F86E0F0EF76403D00800F55005D0F6CF24
:108CB800E9FFF7CFEAFFEF506A6E200E6A6012D024
:108CC800BCC062F0BDC063F0656A646A38EC34F019
:108CD800C36F20EE12F0BC51D926BD51DA22DE6AEC
:108CE800DD6A5DD0BCC013F0BDC014F0BE0E156EB9
:108CF80089EC31F00001C36FC35151E1BCC0B6F03B
:108D0800BDC0B7F099EC4EF0C36F20EE14F0BC5123
:108D1800D926BD51DA2210EE0BF0DE50E126DD50E7
:108D2800E222E750C26FC35108E0040EC31937E1CD
:108D3800C2B535D0050EC36F32D0C2B530D020EEE3
:108D480012F0BC51D926BD51DA22DECFC0F0DDCFFA
:108D5800C1F020EE0BF0C051D926C151DA22DFA8AC
:108D6800E9D7BCC0D9FFBDC0DAFFDECF0BF0DDCF3D
:108D78000CF0C0C00DF0C1C00EF0CCEC4FF00001FB
:108D880020EE06F0BC51D926BD51DA220BC0DEFF19
:108D98000CC0DEFF0DC0DEFF0EC0DEFFA3D7C3513F
:108DA80012000600D9CF05F0DACF06F0F2A01CD0E9
:108DB80081BC02D08994899281A802D089A20FD05F
:108DC8009380939424EE44F0010EDBBE07D0000E8E
:108DD800DE5C020EDE5802E3939201D0938281B8E2
:108DE80089B201D09384F290F2B281B079D081B87F
:108DF80089B29392831C086E811C076E44C409F0E3
:108E080045C40AF00ABE03D0020E0A5C2BE2094AE6
:108E18000A2A09C044F40AC045F442C409F043C40C
:108E28000AF0460E0924D96E040E0A20DA6E08C02C
:108E3800DFFF460E0924D96E060E0A20DA6E07C037
:108E4800DFFF094A0A2A0168010E026E09C003F011
:108E58000AC004F0015003160250041603C042F47D
:108E680004C043F481B889B29384938481A0FED767
:108E780081A802D089A202D0939401D0938424EED1
:108E880044F0010EDBBE05D0000EDE5C020EDE589B
:108E980003E201019B5102E0939201D0938207A85B
:108EA8001ED00BD0898202D0898405D0899417D02E
:108EB80089A215D08994899212D00850016E026A4D
:108EC80002500DE10150040AF3E0100AF1E0340AFF
:108ED800E9E01F0AF0E07F0AE7E01F0AE7E0F29204
:108EE80006C0DAFF05C0D9FF75921100326A20EE7C
:108EF80004F02450D9262550DA22DF5001E197D01A
:108F080020EE2AF02450D9262550DA22DECF35F07B
:108F1800DECF36F0DECF37F0DECF38F02E0E242449
:108F28001A6E000E25201B6E35C01CF036C01DF0D1
:108F380037C01EF038C01FF0216A010E206E20EEE7
:108F480001F02450D9262550DA22DF5075EC4CF078
:108F5800000903E0010E326E6AD020EE04F02450BE
:108F6800D9262550DA22DF6A20EE16F02450D926B9
:108F78002550DA2210EE1EF02450E1262550E22278
:108F8800E6CF2AF0E6CF2BF0E6CF2CF0E6CF2DF097
:108F98002A50355C2E6E2B5036582F6E2C50375871
:108FA800306E2D503858316EDE502E5CDE502F5802
:108FB800DE503058DE5031583AE220EE03F02450AB
:108FC800D9262550DA22DF50336E346A345003E153
:108FD800020E335C2CE320EE16F02450D9262550DF
:108FE800DA22DE503526DE503622DE503722DD50BA
:108FF80038222E0E24241A6E000E25201B6E35C032
:109008001CF036C01DF037C01EF038C01FF0216AB2
:10901800010E206E20EE01F02450D9262550DA22C8
:10902800DF5075EC4CF03306D8A03406CFD7325059
:1090380012002F6C696664617461302E62696E205B
:10904800002F6C696664617461312E62696E20005C
:109058002F6C696664617461322E62696E20002F1C
:109068006C696664617461332E62696E20002F6CCE
:10907800696664617461342E62696E20002F6C69C0
:109088006664617461352E62696E20002F6C6966B2
:1090980064617461362E62696E20002F6C696664A3
:1090A800617461372E62696E20002F6C6966646195
:1090B8007461382E62696E20002F6C696664617471
:1090C80061392E62696E20002F6C69666461746173
:1090D800612E62696E20002F6C696664617461623A
:1090E8002E62696E20002F6C696664617461632E5C
:1090F80062696E20002F6C696664617461642E6217
:10910800696E20002F6C696664617461652E6269FE
:109118006E20002F6C696664617461662E62696EE8
:109128002000000000000000000000000000000017
:109138000000000000000000000000000000000027
:109148000000000000000000000000000000000017
:1091580000000000000000000000000000000BC03C
:1091680015F00CC016F00F50101001E1120015C0D8
:10917800D9FF16C0DAFF0DC0DFFF0F501524116E9E
:1091880010501620126EFF0E1124D96EFF0E1220F9
:10919800DA6E0DC0DFFF105004E1030E0F5C01E230
:1091A800120020EE01F01550D9261650DA220DC013
:1091B800DFFF20EE02F01550D9261650DA220DC036
:1091C800DFFF0F501524116E10501620126EFE0E80
:1091D8001124D96EFF0E1220DA6E0DC0DFFF0F507A
:1091E8001524116E10501620126EFD0E1124D96E22
:1091F800FF0E1220DA6E0DC0DFFF105004E1070EDB
:109208000F5C01E2120020EE03F01550D92616502B
:10921800DA220DC0DFFF0F501524116E10501620F2
:10922800126EFC0E1124D96EFF0E1220DA6E0DC0DC
:10923800DFFF105004E1090E0F5C01E2120015C0B7
:1092480011F016C012F0111E121E114A122A030E36
:109258001114136E146A1350152614501622135045
:109268000F5E1450105AFC0E0F160BD015C0D9FF04
:1092780016C0DAFF0DC0DFFF0F06D8A01006154A8A
:10928800162A0F501010F2E11200000191519011AE
:109298008F1103E1020E8E5D0FE320EE12F08C5168
:1092A800D9268D51DA22DE508E5DDE508F59DE5080
:1092B8009059DE50915902E3020E2CD0966B6AD079
:1092C8008CC044F08DC045F08EC046F08FC047F08A
:1092D80090C048F091C049F0E7EC1EF044C097F008
:1092E80045C098F046C099F047C09AF000019751E0
:1092F800981199119A115DE09705981199119A1191
:10930800DBE0972909E1982907E1992905E19A29DC
:1093180003E1010E966F4DD08CC044F08DC045F02E
:109328008EC046F08FC047F090C048F091C049F019
:109338004A6A4B6A4C6A4D6A2EEC1AF0966F96513F
:1093480038E120EE0EF08C51D9268D51DA22DE2834
:1093580006E1DE2804E1DE2802E1DE2813E020EE43
:109368000EF08C51D9268D51DA22DE2A000EDE222B
:10937800DE22DE2220EE05F08C51D9268D51DA222C
:10938800000EDB8097C08EF098C08FF099C090F0E7
:109398009AC091F020EE12F08C51D9268D51DA2224
:1093A800DE508E5DDE508F59DE509059DE50915957
:1093B80087E396511200136814680B50D96EDA6A65
:1093C800DE50DE1001E181D00B50D96EDA6ADECFB3
:1093D80017F0DDCF18F002D0174A182A17C0F6FF89
:1093E80018C0F7FF000EF86E0F0EF76403D00800E0
:1093F800F55005D0F6CFE9FFF7CFEAFFEF500D6E35
:10940800200E0D6413D017C0F6FF18C0F7FF000E2A
:10941800F86E0F0EF76403D00800F55005D0F6CFAC
:10942800E9FFF7CFEAFFEF503A0AD6E117C0F6FF97
:1094380018C0F7FF000EF86E0F0EF76403D008008F
:10944800F55005D0F6CFE9FFF7CFEAFFEF503A0A1B
:1094580041E10B50D96EDA6ADECF11F0DDCF12F0A0
:1094680011C0F6FF12C0F7FF000EF86E0F0EF7647A
:1094780003D00800F55005D0F6CFE9FFF7CFEAFF93
:10948800EF500D6ED00E0D24156E166AFF0E1622C3
:10949800114A122A165019E10A0E155C16E21750E5
:1094A800111813E11850121810E1155016100DE19B
:1094B80015C013F016C014F0174A182A0B50D96EAD
:1094C800DA6A17C0DEFF18C0DDFF13C00BF014C046
:1094D8000CF01200136A146AF8D7020E0D5E000E23
:1094E8000E5A0F5A105A20EE12F00B50D9260C5073
:1094F800DA22FE0EDE24116EFF0EDE20126EFF0E43
:10950800DE20136EFF0EDE20146E11500D5C12501B
:109518000E5813500F581450105805E30B6A0C6A74
:109528000D6A0E6A120020EE26F00B50D9260C5058
:10953800DA22DECF11F0DECF12F0DECF13F0DECF6D
:1095480014F020EE02F00B50D9260C50DA22DF502E
:10955800156E15C016F0176A186A196A16500D02AA
:10956800F3CF1AF0F4CF1BF01C6A1D6A0E02F350F9
:109578001B26F4501C22000E1D2217500D02F3501A
:109588001B26F4501C22000E1D2216500F02F35009
:109598001C26F4501D2217500E02F3501C26F450BE
:1095A8001D2218500D02F3501C26F4501D22105095
:1095B8001602F3501D2617500F02F3501D2618509F
:1095C8000E02F3501D2619500D02F3501D2611509E
:1095D8001A240B6E12501B200C6E13501C200D6E9B
:1095E80014501D200E6E1200FDC14AF070D0FBEC25
:1095F80059F04A6EFD1978E0150E496E4B0E486E0B
:10960800BE0EE82EFED7482EFCD7492EFAD700D03A
:109618006BD0D3EC55F04B6E4B5066E04BB06D2AD7
:109628004BB26D060F0E6D16000E0B6EC00E27ECBA
:1096380057F0EAEC59F0000E0B6EC00E27EC57F00D
:109648006D500F0D740EF3240F6E0C0EF420106E77
:1096580043EC53F00D0E496E2D0E486ED80EE82ED1
:10966800FED7482EFCD7492EFAD74BA43DD00C6A1A
:109678000B6A6DC00DF068EC58F09A0E0001806F0F
:10968800FC0E816F6DC082F0836B7DEC5AF06DC06B
:109698004AF0000E0B6E800E27EC57F0EAEC59F0FA
:1096A800000E0B6E800E27EC57F06D500F0D740EE8
:1096B800F3240F6E0C0EF420106E43EC53F0000EE2
:1096C8000B6EC00E27EC57F0EAEC59F00DD00101F3
:1096D8009751486E496A495007E14850010A87E0A6
:1096E800030A85E0010A95E04A5012001F6A206AC1
:1096F800186A196A01D0122A010E1E6E1250D96E0C
:10970800DA6A200EDE1813E0F70E146E1568125090
:10971800D96EDA6ADF50166E176A1450162615507D
:109728001722175003E1050E165C01E31E6A1EC0DE
:109738001AF01B6A1A501B1006E0DDD7196A010ED1
:10974800186E122A25D01250D96EDA6ADF50146EBC
:10975800156A15501DE114502B0AF3E0060AEEE0D5
:1097680017D00A0E1F02F3CF14F0F4CF15F0200221
:10977800F35015261250D96EDA6ADF50145E000EC7
:10978800155A300E14241F6E000E1520206ED9D7DE
:10979800D00E146E15681250D96EDA6ADF50166E44
:1097A800176A1450162615501722175005E10A0E8D
:1097B800165C02E2010E01D0000E1C6E1D6A1C50E0
:1097C8001D10CFE1185019100DE11FC014F020C072
:1097D80015F0141E151E144A152A14C012F015C0CF
:1097E80013F012001FC012F020C013F012009F6B7C
:1097F8008980000E0B6E030E0C6E0E6AF60E0D6E4F
:10980800010E106E0F6AB3EC48F06A0E0001806F0B
:10981800FE0E816F7DEC5AF00001E76BE86B2E0EAF
:1098280087EC5AF082B415D07350200D000EF32443
:109838000001A36F020EF420A46F000EA56F030EA3
:10984800A66F010EA86FA76BE30EA96FBEEC0EF012
:10985800E56F0001E55109E07B0E806FFF0E816F17
:10986800E5C082F0836B7DEF5AF0B6EC5AF00B50EE
:109878000C1027E0E60E0B6E0C6A35EC52F0000176
:10988800E26FE651100B486E000E496EE2512FEC64
:1098980027F048C0E9F049C0EAF0040E0001E919D0
:1098A800EA1102E14BEC58F0020E0001E919EA1145
:1098B80002E179EC55F00001E905EA1102E11EEC3C
:1098C80039F00001E74BE82BE85103E1C80EE75DEA
:1098D800A6E3210E806FFF0E816F7DEC5AF0899010
:1098E8001200236E2350D8A4040C2050211001E14B
:1098F800040C74B0030C74B4020C6EB608D0090ED4
:10990800D8901C361D361E361F36E82EF9D720048F
:1099180021101AE11CC014F01DC015F01EC016F06D
:109928001FC017F0180EBDEC58F0000945E11AC029
:109938000DF01BC00EF0FE0E0F6E81EC56F0000904
:109948003BE0206A216A38D06EC022F0060E22164B
:1099580009E020C014F021C015F0166A176A970EA6
:10996800BDEC58F01CC014F01DC015F01EC016F058
:109978001FC017F0190EBDEC58F000091DE11AC000
:109988000DF01BC00EF0FC0E0F6E81EC56F00009B6
:1099980008E0020E1B262006D8A021062050211020
:1099A800EEE10D6A0E6AFD0E0F6E81EC56F00009AD
:1099B80003E1216A010E206EBBEC5AF02050211001
:1099C800D8A4010C000C3A0EF66E900EF76E000E3D
:1099D800F86E0CEE74F011EE2CF00900F5CFEEFFE6
:1099E800E550E150FAE1E250F8E1A00EF66EAF0E54
:1099F800F76E000EF86E02EEA0F010EE40F00900CF
:109A0800F5CFEEFFE550E150FAE1600EF66EB50EC7
:109A1800F76E000EF86E01EEF1F010EE0BF0090093
:109A2800F5CFEEFFE550E150FAE1940EF66EB50E73
:109A3800F76E000EF86E0900F5CF74F004EE40F0F2
:109A480018EE34F0EE6AE550E150FCE1E250FAE13C
:109A580004EE00F0400EEE6AE806FDE103EE00F0C9
:109A680011EE00F0EE6AE550E150FCE1E250FAE157
:109A780002EE00F0A00EEE6AE806FDE101EE00F04D
:109A8800AB0EEE6AE806FDE10001FD6B00EE6BF03F
:109A9800090EEE6AE806FDE175907592000EF86E03
:109AA800000149EF07F00F0EC16E969496929690BA
:109AB800929A090E106E1E0E0F6EE40EE82EFED757
:109AC8000F2EFCD7102EFAD700D0090E106E1E0EDE
:109AD8000F6EE40EE82EFED70F2EFCD7102EFAD705
:109AE80000D0D00E0F6ECA0EE82EFED70F2EFCD770
:109AF800000E0B6E300E27EC57F0150E0F6EC60ECB
:109B0800E82EFED70F2EFCD700D0000E0B6E300EBD
:109B180027EC57F0000E0B6E300E27EC57F0000EB6
:109B28000B6E390E27EC57F0000E0B6E140E27EC57
:109B380057F0000E0B6E560E27EC57F0000E0B6E0A
:109B48006D0E27EC57F0000E0B6E700E27EC57F0D9
:109B5800000E0B6E0C0E27EC57F0000E0B6E060E67
:109B680027EC57F0000E0B6E010E27EC57F0680E2D
:109B78000F6EE40EE82EFED70F2EFCD700D0120091
:109B8800030E0001806FF90E816FCFCF82F0836BD7
:109B9800CECF84F0856B73C086F0876B7DEC5AF06E
:109BA8000101FC83735028E1740E0B6E0A0E0C6ED3
:109BB800F20E0D6E010E0E6E106A050E0F6E6DEC34
:109BC80057F0790E0B6E0A0E0C6EA00E0D6E020E7B
:109BD8000E6E106A130E0F6E6DEC57F08C0E0B6E36
:109BE8000A0E0C6EC60E0D6E020E0E6E106A0D0E6B
:109BF8000F6E6DEC57F027D0740E0B6E0A0E0C6EBC
:109C0800F70E0D6E010E0E6E106A050E0F6E6DECDE
:109C180057F0790E0B6E0A0E0C6EB30E0D6E020E17
:109C28000E6E106A130E0F6E6DEC57F08C0E0B6EE5
:109C38000A0E0C6ED30E0D6E020E0E6E106A0D0E0D
:109C48000F6E6DEC57F0496A250E486E8EEC3DF0AC
:109C5800FC93899012007350140D070EF324D96EEB
:109C6800010EF420DA6E000EDE24CA6F010EDE202B
:109C7800CB6F000EDE20CC6F000EDE20CD6F735050
:109C8800140D070EF324D96E010EF420DA6ECAC043
:109C9800DEFFCBC0DEFFCCC0DEFFCDC0DEFF7350E1
:109CA800140D070EF324D96E010EF420DA6EDECF00
:109CB800CFF0DDCFD0F09F0E806FF40E816FCFCF45
:109CC80082F0836BCECF84F0856BCFC086F0D0C096
:109CD80087F0CFC088F0D0C089F07DEC5AF073507F
:109CE800200D000EF3240001A36F020EF420A46FD0
:109CF800CFC0A5F0D0C0A6F0A76BA86B2CEC12F0D3
:109D0800CE6FCE5110E0420E806FFB0E816FCFC038
:109D180082F0D0C083F0CEC084F0856B7DEC5AF021
:109D2800010E6B6E010C6B6A1200B6C062F0B7C010
:109D380063F0656A646A38EC34F0BB6FBB5102E0CB
:109D4800BB511200B6C0D9FFB7C0DAFFDECF39F079
:109D5800DDCF3AF020EE0EF0B651D926B751DA220F
:109D6800DECF3BF0DECF3CF0DECF3DF0DECF3EF085
:109D7800C3EC50F00001BB6FBB51E2E120EE12F0E2
:109D8800B651D926B751DA22DECFB9F0DDCFBAF015
:109D9800B9C0D9FFBAC0DAFFDF50B86FB85103E1D4
:109DA800040EBB6FCDD720EE0BF0B951D926BA51AE
:109DB800DA22DFB616D0B9C00BF0BAC00CF020EE2C
:109DC80014F0B651D926B751DA22DECF0DF0DDCF27
:109DD8000EF0106A0B0E0F6EA6EC55F00B500C101F
:109DE800AFE0B6C0A3F0B7C0A4F0A66BA56B1AECA1
:109DF80029F00001BB6FBB51A3E1A4D7B6C062F044
:109E0800B7C063F0656A646A38EC34F0BF6FBF515D
:109E180057E1BD6BBE6BB6C0D9FFB7C0DAFFDECF66
:109E280039F0DDCF3AF020EE0EF0B651D926B75111
:109E3800DA22DECF3BF0DECF3CF0DECF3DF0DECFE6
:109E48003EF0C3EC50F00001BF6FBF5139E120EE86
:109E580012F0B651D926B751DA22DECFBAF0DDCFEB
:109E6800BBF0BAC0D9FFBBC0DAFFE50EDE1810E0C0
:109E780020EE12F0B651D926B751DA22DECFBAF069
:109E8800DDCFBBF0BAC0D9FFBBC0DAFFDF5009E1B4
:109E9800BD4BBE2BB851BD1906E1B951BE1910E032
:109EA80002D0BD6BBE6BB6C0A3F0B7C0A4F0A66B62
:109EB800010EA56F1AEC29F00001BF6FBF51ABE08E
:109EC800040EBF1902E1070EBF6FBF511200C0C0D8
:109ED800B6F0C1C0B7F0B96B010EB86F02EC4FF025
:109EE8006A6E6A5053E1C0C0D9FFC1C0DAFFDECF45
:109EF80039F0DDCF3AF020EE0EF0C051D926C1512D
:109F0800DA22DECF3BF0DECF3CF0DECF3DF0DECF15
:109F18003EF0C3EC50F06A6E6A5038E1000120EE62
:109F280012F0C051D926C151DA22DECF0BF0DDCFB5
:109F38000CF00E6A0D6A106A200E0F6EC2EC59F012
:109F4800000120EE12F0C051D926C151DA22DECF2D
:109F58000BF0DDCF0CF020EE14F0C051D926C15122
:109F6800DA22DECF0DF0DDCF0EF0106A0B0E0F6E89
:109F7800F0EC57F0C0C0D9FFC1C0DAFF10EE04F012
:109F8800DE50E126DD50E222010EE76E6A50120033
:109F98001A0E0D240F6E000E0E20106E0F28D96EAB
:109FA800000E1020DA6EDF50126E116A1A0E0D24A0
:109FB800D96E000E0E20DA6EDF50111211C017F0A4
:109FC80012C018F0196A1A6A0BC0D9FF0CC0DAFF60
:109FD800030EDE1829E1140E0D240F6E000E0E205C
:109FE800106E0F28D96E000E1020DA6EDF50126E38
:109FF800116A140E0D24D96E000E0E20DA6EDF5091
:10A008001110136E1250146E156A166A14C016F0E9
:10A0180013C015F0146A136A13501712145018124B
:10A028001550191216501A1217C00BF018C00CF060
:10A0380019C00DF01AC00EF01200226E2250D8A4DA
:10A04800040C2050211001E1040C74B0030C6EB60E
:10A0580008D0090ED8901C361D361E361F36E82E3D
:10A06800F9D7215006E1020E205C03E2246A110EA2
:10A0780002D0246A120E236E23C025F01CC014F0EF
:10A088001DC015F01EC016F01FC017F02550BDECFE
:10A0980058F000091DE11AC00BF01BC00CF0020EAD
:10A0A8000E6E0D6A00EC56F0000908E0020E1B2641
:10A0B8002006D8A0210620502110EDE1120E251807
:10A0C80007E1146A156A166A176A0C0EBDEC58F097
:10A0D800BBEC5AF020502110D8A4010C000C898048
:10A0E800000E0B6E030E0C6E0E6AF60E0D6E010E50
:10A0F800106E0F6AB3EC48F06A0E0001806FFE0E16
:10A10800816F7DEC5AF00001C96BCA6B2E0E87EC8B
:10A118005AF082B415D07350200D000EF3240001BC
:10A12800A36F020EF420A46F000EA56F030EA66F96
:10A13800010EA86FA76BC60EA96FBEEC0EF0C86F14
:10A148000001C85109E07B0E806FFF0E816FC8C007
:10A1580082F0836B7DEF5AF0C94BCA2BCABFD6D7A2
:10A16800CA5103E1640EC95DD1E3210E806FFF0E71
:10A17800816F7DEC5AF0899089906B6A1200436A6E
:10A1880020EE2AF03950D9263A50DA223B50DE1810
:10A1980009E13C50DE1806E13D50DE1803E13E506F
:10A1A800DE1839E039C024F03AC025F07AEC47F0DF
:10A1B800436E435030E12E0E39241A6E000E3A20B9
:10A1C8001B6E3BC01CF03CC01DF03DC01EF03EC0E5
:10A1D8001FF0216A010E206E20EE01F03950D926B9
:10A1E8003A50DA22DF5021EC50F0000906E03B68D3
:10A1F8003C683D683E68010E436E20EE2AF03950F7
:10A20800D9263A50DA223BC0DEFF3CC0DEFF3DC013
:10A21800DEFF3EC0DEFF43501200D4C0DAF0D5C0E6
:10A22800DBF0DA0E0B6EDFEC49F00BC0DCF00CC093
:10A23800DDF00001DDBF0B0CD890DC35D96EDD35C3
:10A24800DA6E8C0ED926010EDA22DECFD8F0DDCFF9
:10A25800D9F0D851D91105E0D8C0D9FFD9C0DAFF53
:10A26800DF6AD251D31105E0D2C0D9FFD3C0DAFFDB
:10A27800DF6AD890DC35D96EDD35DA6E8C0ED926DA
:10A28800010EDA22D2C0DEFFD3C0DDFFD251D311D6
:10A29800D8B4000CD60501E0000CD20E666E676AD1
:10A2A800D40E686E696A09EC00F0D76FD7511200B6
:10A2B80003D00B4A0C2A0D2A0D50D96EDA6ADF50EA
:10A2C8000E6E0BC0F6FF0CC0F7FF000EF86E0F0EF7
:10A2D800F76403D00800F55005D0F6CFE9FFF7CFB3
:10A2E800EAFFEF500E1813E10BC0F6FF0CC0F7FFA2
:10A2F800000EF86E0F0EF76403D00800F55005D075
:10A30800F6CFE9FFF7CFEAFFEF500009D2E10BC023
:10A31800F6FF0CC0F7FF000EF86E0F0EF76403D0BF
:10A328000800F55005D0F6CFE9FFF7CFEAFFEF5068
:10A338000E6E0D50D96EDA6ADF500E5C0B6E0C6A29
:10A34800D8A00C0612000BC012F00CC013F00DC000
:10A3580014F00EC015F00F06D8A010060F280CE157
:10A3680010280AE10B6A0C6A1200124A132A144ACE
:10A37800152A0F06D8A0100612C0F6FF13C0F7FF63
:10A388000800F55015E014C0D9FF15C0DAFFDF50FA
:10A398000FE00F5010100CE014C0D9FF15C0DAFF01
:10A3A80012C0F6FF13C0F7FFDE500900F518DDE014
:10A3B80012C0F6FF13C0F7FF0800F5CF11F014C064
:10A3C800D9FF15C0DAFFDF50115C0B6E0C6AD8A0FC
:10A3D8000C0612000CC012F00DC013F0125013102E
:10A3E800D8B4090C12C0D9FF13C0DAFFDE50DE1052
:10A3F800D8B4090C12C0D9FF13C0DAFFDECF0EF0B3
:10A40800DDCF0FF00EC0D9FF0FC0DAFFDF50D8B490
:10A41800090C20EE02F01250D9261350DA2212C08D
:10A42800E1FF13C0E2FF00EE06F0E650E926E55032
:10A43800EA22DE50EE1813E1DE50EE18D8A4090C1B
:10A4480012C0D9FF13C0DAFF10EE01F0DE50E1268A
:10A45800DD50E222E750AAEC5AF00E6E0EB0090C5D
:10A46800000C24EE44F0DE50DE10FBE040C413F094
:10A4780041C414F0460E1324D96E040E1420DA6E6B
:10A48800DF50116E460E1324D96E060E1420DA6EB4
:10A49800DF50126E134A142A0D68010E0E6E13C097
:10A4A8000FF014C010F00D500F160E5010160FC0FC
:10A4B80040F410C041F4F29E24EE44F0DE06000E93
:10A4C800DD5AF28E0BC0D9FF0CC0DAFF12C0DFFFD5
:10A4D80024EE44F0010EDBBE05D0000EDE5C020E59
:10A4E800DE5802E289B29382115012000E5002E047
:10A4F8000E5003E10C5073EF5AF00E50D96EDA6A21
:10A50800040ED926DE50DE1014E00E50D96EDA6A39
:10A51800040ED9260E50E16EE26A020EE126DE50E4
:10A52800E65CE650800A136EDE50800A1358D8B0F5
:10A5380012000E50D96EDA6A020ED926DECF0FF05D
:10A54800DDCF10F00E50D96EDA6ADECF11F0DDCF14
:10A5580012F00F501124D96E10501220DA6E0CC070
:10A56800DFFF0E50D96EDA6A020ED926DE2A000EF7
:10A57800DD22000C0B500F02F3CF13F0F4CF14F0D0
:10A58800156A166A0B501002F3501426F45015225F
:10A59800000E16220C500F02F3501426F450152208
:10A5A800000E16220B501102F3501526F4501622F5
:10A5B8000C501002F3501526F45016220D500F02BD
:10A5C800F3501526F450162212500B02F35016269B
:10A5D8000C501102F35016260D501002F350162697
:10A5E8000E500F02F350162613C00BF014C00CF0D7
:10A5F80015C00DF016C00EF01200AA0E806FFD0EE9
:10A60800816F84C182F085C183F07DEC5AF011D04E
:10A61800030E0BD0050E4A6E0101846B856B2DD09D
:10A628000A0E03D0010E01D0020E4A6E26D04A6AE5
:10A6380024D084C148F085C149F0495009E0020A94
:10A648000DE00E0A0FE0010A11E02A0A13E0EFD725
:10A6580048500A0ADDE01E0ADDE0E9D74850BC0A86
:10A66800E3E0E5D748501C0ADBE0E1D74850AC0AE4
:10A67800D9E0DDD748500F0ADAE14A5012000B0E34
:10A68800116E620EE82EFED7112EFCD700D020D016
:10A698000B0E116E620EE82EFED7112EFCD700D0DD
:10A6A800010E0B6E0FC0F6FF10C0F7FF000EF86E1C
:10A6B8000F0EF76403D00800F55005D0F6CFE9FF78
:10A6C800F7CFEAFFEF5027EC57F00F4A102AD7D7F9
:10A6D8000FC0F6FF10C0F7FF000EF86E0F0EF764FC
:10A6E80003D00800F55005D0F6CFE9FFF7CFEAFF11
:10A6F800EF500009CDE11200FA0E0001806FFA0E4A
:10A70800816FCFCF82F0836BCECF84F0856B7DECE9
:10A718005AF0486A496A7350140D070EF324D96E2B
:10A72800010EF420DA6EDE6ADE6ADE6ADD6A7350D4
:10A73800140D130EF324D96E010EF420DA6EDF6ABD
:10A748007350140D0F0EF324D96E010EF420DA6E37
:10A75800DE6ADE6ADE6ADD6A484A492A49BEDBD714
:10A76800495003E1040E485CD6E389906B6A1200F5
:10A77800136A146A156A166A0F5010101110121015
:10A7880029E0010E176E06D0D8900F361036113614
:10A798001236172A12AEF8D7D89013361436153653
:10A7A80016360F500B5C10500C5811500D581250A3
:10A7B8000E5809E30F500B5E10500C5A11500D5AE9
:10A7C80012500E5A1380D8901232113210320F32B2
:10A7D800172EE2D713C00BF014C00CF015C00DF003
:10A7E80016C00EF01200706A6F6A01018E6B8F6BD3
:10A7F800020E9F6F89909E6B9D6B736A030E736444
:10A8080001D029D07350070D520EF324D96E010ED2
:10A81800F420DA6EDF6A7350070D510EF324D96EF7
:10A82800010EF420DA6EDF6A7350070D500EF32420
:10A83800D96E010EF420DA6EDF6A7350070D530EDD
:10A84800F324D96E010EF420DA6EDE6ADE6ADE6A5F
:10A85800DD6A732AD3D7736A12000C0E0001806F69
:10A86800FF0E816F7DEC5AF0736A030E736401D09A
:10A8780029D07350070D520EF324D96E010EF4201F
:10A88800DA6EDF6A7350070D510EF324D96E010E8C
:10A89800F420DA6EDF6A7350070D500EF324D96E78
:10A8A800010EF420DA6EDF6A7350070D530EF3249D
:10A8B800D96E010EF420DA6EDE6ADE6ADE6ADD6ABF
:10A8C800732AD3D7736A899001019F6B1200B2EC87
:10A8D80041F0CAC0E5F0CBC0E6F0E551E61105E06D
:10A8E800E5C0E1F0E6C0E2F0120082B414D0735083
:10A8F800200D000EF324A36F020EF420A46F000EA7
:10A90800A56F030EA66F010EA86FA76BE30EA96FC4
:10A91800BEEC0EF0E96FE9510EE09A0E806FFD0E65
:10A92800816FE9C082F0836B7DEC5AF0E9C0E1F0F9
:10A938000001E26B12002FEC4EF00001E16BE26BBC
:10A948001200136E0C0E131807E0BBEC5AF050EC13
:10A958005AF0000901E1FF0C135040099AEC5AF033
:10A9680010509AEC5AF00F509AEC5AF00E509AEC9C
:10A978005AF00D509AEC5AF0010E126E135002E183
:10A98800950E126E080E131802E1870E126E125001
:10A998009AEC5AF00C0E131802E1A3EC5AF00A0EC6
:10A9A800126EA3EC5AF0116E11AE02D0122EF9D726
:10A9B800115012005C0E0001806FFE0E816F7DEC5D
:10A9C8005AF04C6A4D6A716A4B6A21D0B6EC5AF05B
:10A9D8000B500C1011E04B0E0B6E0C6A35EC52F05C
:10A9E8004A6E000E7124D96EDA6A030EDA224AC062
:10A9F800DFFF712A4C4A4D2A4BAA07D0000E4C247F
:10AA0800486E040E4D20496E120081AC04D04DBE34
:10AA1800DDD74D04DBE34CC048F04DC049F01200CF
:10AA28002DEC58F0CC0E29EC5AF0660E29EC5AF0B1
:10AA38000CEC5AF0156E155005E10F6A106A116A90
:10AA4800126A1200136A146A1350150FD96EDA6A63
:10AA58000CEC5AF0DF6E134A142A14BEF5D71450C2
:10AA680003E1040E135CF0E318501710161003E10D
:10AA7800060E155CE2E315C00FF016C010F017C003
:10AA880011F018C012F012000F501010111012100F
:10AA980023E0010E136E06D0D8900F36103611360B
:10AAA8001236132A12AEF8D70F500B5C10500C5800
:10AAB80011500D5812500E5808E30F500B5E1050ED
:10AAC8000C5A11500D5A12500E5AD8901232113297
:10AAD80010320F32132EE8D70BC00BF00CC00CF05D
:10AAE8000DC00DF00EC00EF01200390E0001806F7F
:10AAF800FD0E816F7DEC5AF089800101FC832AEEFE
:10AB080074F09DC1DFFF000EE8CF75FA0D0EE8CF97
:10AB180076FA000EE8CF77FA82A403D0600EE8CF69
:10AB280077FA82A406D076CA4EF0200E4E124EC096
:10AB380076FA496A040E486E8EEC3DF0FC939D6BE4
:10AB4800899012000BC012F00CC013F00DC014F065
:10AB58000EC015F0166A176A0F06D8A010060F283F
:10AB680002E1102817E012C0D9FF13C0DAFF124A19
:10AB7800132ADF50116E14C0D9FF15C0DAFF144A2A
:10AB8800152ADF50115C166E176AD8A017061650E2
:10AB98001710E2E016C00BF017C00CF01200010EFF
:10ABA8000B6E0C6A92868D828D8400D000D000D006
:10ABB80000D08D9400D000D000D000D00D6A0E6A6D
:10ABC80080A602D00B500C12D8900B368D9000D076
:10ABD80000D000D000D08D8000D000D000D000D0B0
:10ABE8008D900D4A0E2A0EBEEBD70E5003E1030ED0
:10ABF8000D5CE6E30C501200070E106ED00E0F6EBF
:10AC08000CD0A3EC5AF0116E11280AE1A00E00D066
:10AC1800E82EFDD70F06D8A010060F501010F1E14E
:10AC2800FE0E111801E0000CA3EC5AF00BC0D9FF7E
:10AC38000CC0DAFFDF6E0B4A0C2A0D06D8A00E06F0
:10AC48000D500E10F1E1A3EC5AF0A3EC5AF0010CF0
:10AC58000BC011F00CC012F013D00F06D8A01006CC
:10AC68000DC0D9FF0EC0DAFF0D4A0E2A11C0E1FF50
:10AC780012C0E2FF114A122ADFCFE7FFE7500BE0CC
:10AC88000F50101008E0E9D711C0D9FF12C0DAFF41
:10AC9800DF6A114A122A0F06D8A010060F28F4E11D
:10ACA8001028F2E112008C6A8A6A9568936801019B
:10ACB8009B6B716A89928994886B896B09D0000EA5
:10ACC8008825D96E030E8921DA6EDF6A884B892BB5
:10ACD80089BFF5D78905F3E3886B896B09D0740EB2
:10ACE8008825D96E0A0E8921DA6EDF6A884B892B8E
:10ACF80089BFF5D78905F3E3120026EC59F000095E
:10AD080001E1000C0F509AEC5AF0FD0E0F181EE0EE
:10AD1800020E116E106A0DC0D9FF0EC0DAFFDF50A7
:10AD28009AEC5AF00D4A0E2A1006D8A011061050B7
:10AD38001110F1E1A3EC5AF0A3EC5AF0A3EC5AF08D
:10AD4800126E12501F0B050A01E0000C010C15D001
:10AD58000CC0F6FF0DC0F7FF000EF86E0F0EF7647B
:10AD680003D00800F55005D0F6CFE9FFF7CFEAFF8A
:10AD7800EF5087EC5AF00C4A0D2A0CC0F6FF0DC0B4
:10AD8800F7FF000EF86E0F0EF76403D00800F550B9
:10AD980005D0F6CFE9FFF7CFEAFFEF500009D8E179
:10ADA80012000EC012F00FC013F010C014F011C042
:10ADB80015F02DEC58F0CC0E29EC5AF0990E29EC30
:10ADC8005AF00C0E29EC5AF0166A176A1650120F30
:10ADD800D96EDA6ADF5029EC5AF0164A172A17BEDC
:10ADE800F5D7175002E02DEF58F0040E165CEEE38D
:10ADF8002DEF58F0496ED30E4A6EF30E4B6E486A2B
:10AE08000AD04AC0F6FF4BC0F7FF4A4A4B2A08004F
:10AE1800F550F7E1482A4950481807E04AC0F6FFBC
:10AE28004BC0F7FF0800F550ECE14E0E0001806FB3
:10AE3800FE0E816F49C082F0836B4AC084F04BC01C
:10AE480085F07DEF5AF00C6E8D9200D000D000D0C6
:10AE580000D00BB002D08D9401D08D84000E0E6E00
:10AE6800010E0D6E0CAE02D0898A01D0899AD89055
:10AE78000C368D908D808D900D4A0E2A0EBEF2D71D
:10AE88000E5003E1090E0D5CEDE38D8212009F0E5A
:10AE9800136E146811C015F012C016F01350152661
:10AEA80014501622165005E11A0E155C02E2010E26
:10AEB80001D0000E176E186A1750181005E05F0EC3
:10AEC8001114116E126A120011C011F012C012F0A2
:10AED80012000DC013F00EC014F00BC011F00CC01E
:10AEE80012F010D013C0D9FF14C0DAFFDF50156E6E
:10AEF800134A142A11C0D9FF12C0DAFF15C0DFFFA8
:10AF0800114A122A0F06D8A010060F28EBE11028C4
:10AF1800E9E1120020EE1AF00B50D9260C50DA2283
:10AF28000DC0DFFF20EE1BF00B50D9260C50DA22A3
:10AF38000EC0DFFF20EE14F00B50D9260C50DA2299
:10AF48000FC0DFFF20EE15F00B50D9260C50DA2287
:10AF58001050DF6E12000BC00DF00CC00EF002D0C6
:10AF68000B4A0C2A0BC0F6FF0CC0F7FF000EF86E58
:10AF78000F0EF76403D00800F55005D0F6CFE9FFAF
:10AF8800F7CFEAFFEF500009EBE10D500B5C0B6EB9
:10AF98000E500C580C6E12000007958101004000FD
:10AFA80001000300005001F4010100000795810130
:10AFB80000400001000300005001F40101000006F8
:10AFC8002305003E000000091127000006230500A4
:10AFD8003E000000091127000BC011F00CC012F050
:10AFE8000DC013F00EC014F00ED013C0D9FF14C05A
:10AFF800DAFF11C0E1FF12C0E2FFDFCFE7FF134A1B
:10B00800142A114A122A0F06D8A010060F28EDE1BB
:10B018001028EBE112000B6E0B500EE0BFEC5AF05B
:10B02800200EE82EFED7C2EC5AF0CC0E00D0E82E47
:10B03800FDD700D000D01200BFEC5AF0C00E00D0EF
:10B04800E82EFDD7C2EC5AF0350EE82EFED700F0F8
:10B058001200BFEC5AF00A0E0C6EF80EE82EFED75E
:10B068000C2EFCD700D0C2EC5AF0E00E00D0E82E2F
:10B07800FDD791EC5AF00D6E090E0C6E840EE82E79
:10B08800FED70C2EFCD7C2EC5AF00D501200460E1B
:10B098000001806FFF0E816F7DEC5AF0740E0B6E0D
:10B0A8000A0E0C6E0E6A0D6A010E106E0F6AB3EC72
:10B0B80048F02AEE74F09FC1DFFF496A010E486E1E
:10B0C8008EEC3DF09F6B1200000EF2BE010E0E6E6C
:10B0D8000C50030BAA6E0BC0A9FF0DC0A8FFA69EBB
:10B0E800A69CA684F29E550EA76EAA0EA76EA682EF
:10B0F800A6B2FED7A6940EB002D0F29E01D0F28E70
:10B10800120002D00B4A0C2A0BC0F6FF0CC0F7FF46
:10B118000800F55009E00BC0F6FF0CC0F7FF080067
:10B12800F5500D180E10EEE10BC0F6FF0CC0F7FF3E
:10B138000800F5500B6E0C6A12005E0E626E5AC063
:10B1480063F05BC064F0656A666A676A686A630E82
:10B15800546E5CC055F05DC056F0620E576E24EC1C
:10B1680025F065505A24D96E66505B20DA6EDF6A86
:10B17800000C186E18AE0ED0189E0D6A0E6A0F6A73
:10B18800106A370EA5EC54F0196E010E196402D03E
:10B198001950120014C00DF015C00EF016C00FF0B3
:10B1A80017C010F01850A5EF54F0010E116E200EC4
:10B1B8000B180C1011E0F70E0D6E0E680BC00FF097
:10B1C8000CC010F00D500F260E501022105003E145
:10B1D800050E0F5C01E3116A11C00BF00C6A120036
:10B1E8005BC04EF05CC04FF0A6EC3FF05D6E5D506A
:10B1F8000FE15BC00CF05CC00DF0EEEC51F05D6E41
:10B208005D5006E15BC0D9FF5CC0DAFFDE6ADD6A2B
:10B218005D5012009F0E0D6E0E68200E0B100F6E03
:10B22800000E0C10106E0D500F260E5010221050EC
:10B2380005E11A0E0F5C02E2010E01D0000E0B6E42
:10B248000C6A1200130E0C6E880E0B6E0BD0A3EC5A
:10B258005AF0FF0A0AE0A00E00D0E82EFDD70B0630
:10B26800D8A00C060B500C10F2E10B500C10D8A40F
:10B27800010C000C186A196A09D017C00CF00D6A85
:10B2880016C00EF07AEC52F0184A192A18501424F5
:10B29800D96E19501520DA6EDF50176E1750EDE190
:10B2A8001200740E0B6E0A0E0C6E0E6A0D6A010EF9
:10B2B800106E0F6AB3EC48F0010EE8CF74FA010182
:10B2C800FC83496A486E8EEC3DF0FC9312009F0E99
:10B2D8000D6E0E680BC00FF00CC010F00D500F264D
:10B2E8000E501022105005E11A0E0F5C02E2010EFA
:10B2F80001D0000E0B6E0C6A1200BF0E0D6E0E68A8
:10B308000BC00FF00CC010F00D500F260E5010227D
:10B31800105005E11A0E0F5C02E2010E01D0000E7A
:10B328000B6E0C6A1200D00E0D6E0E680BC00FF07B
:10B338000CC010F00D500F260E501022105005E1D1
:10B348000A0E0F5C02E2010E01D0000E0B6E0C6AB1
:10B358001200B886AC84B898440EAF6EB06AAC9848
:10B36800AB8EAB88AB9A9D989D9AD08E9F8AF28EB1
:10B37800AC90AB9CAC9AAC8A949112000BC011F0C3
:10B388000CC012F008D011C0D9FF12C0DAFF0DC0EE
:10B39800DFFF114A122A0F06D8A010060F28F3E182
:10B3A8001028F1E11200BFEC5AF0200EE82EFED76B
:10B3B800C2EC5AF0300EE82EFED791EC5AF00C6E23
:10B3C800B00E00D0E82EFDD70C501200106A100EF7
:10B3D8000F6E05D0010E0B6E200E27EC57F00F06EE
:10B3E800D8A010060F28F6E11028F4E112008450C6
:10B3F800070B0B6E928A80AA02D0080E0B26020E4B
:10B408000101971903E10B1C0F0B0B6E0B50120077
:10B418000D6A0E6AD8900D32D7EC59F0000901E098
:10B428000D8E0E2A070E0E64F5D70D501200000E71
:10B43800E8CF40F4E8CF41F4E8CF42F4E8CF43F452
:10B44800E8CF44F4E8CF45F4000C0C6E0D6A0C50BC
:10B45800010B0FEC58F0D8900C320D2A070E0D6432
:10B46800F6D7070C0B6E0B5007E0C66A010EC66EC6
:10B47800400EC76EC68A400CC66A020EF8D7C29044
:10B488000F0EC16E070EB46E4F0EC86E946A948884
:10B4980094829482826A1200C7EC5AF0A3EC5AF0A4
:10B4A80026EC59F0000901E0010CBBEC5AF0000C45
:10B4B8000C50030BAA6E0BC0A9FFA69EA69CA680E3
:10B4C80000F000F0A8501200EA0E0001806FFE0E96
:10B4D800816F7DEC5AF0899001019F6B12000B6E11
:10B4E80003D0C9EC5AF004009EA8FBD70BC0ADFFEF
:10B4F8001200820E476E80C018F081C019F0470E06
:10B508001A6EFDEF20F00B6E03D0C9EC5AF0040060
:10B518009EA8FBD70BC0ADFF1200928880A803D06D
:10B52800010E0B6E01D00B6A0B5012000B6E0BC094
:10B53800C9FFC7B0FED7C7A0FED7C9501200C96857
:10B54800C7B0FED7C7A0FED7C95012000B6E0B506C
:10B5580001E0010C74501200E7800103E80080014B
:03B5680003E800F5
:10B56C0044C40BF045C40CF01200C5EC5AF0A3EF28
:10B57C005AF08998929812008998928812008280C9
:09B58C001200829012001200016D
:10F3D200004F4B004449534B5F455252004E4F542D
:10F3E2005F5245414459004E4F5F46494C45004EDD
:10F3F2004F545F4F50454E4544004E4F545F454E6B
:10F4020041424C4544004E4F5F46494C455F53597B
:10F412005354454D000020000D0A20253258202566
:10F42200325820253273202532732025327320254D
:10F432003273202532732025327320253273202522
:10F44200327320253473202534732025347320250C
:10F4520034732025347320253473202534732025FA
:10F46200347320000D0A253032582530325820538B
:10F472005338303A53657420537461747573206D38
:10F4820061736B20255820255820255820255820A7
:10F49200255820255820255820255820000D0A25BA
:10F4A2003032582530325820535338303A20496E82
:10F4B2006372656D656E743A205365656B696E673C
:10F4C20020746F20256C752028256C582920000D8A
:10F4D2000A48504469736B204D6B204949202831FA
:10F4E200384634363230292025732025732025737F
:10F4F200205374617274696E672E2E2E0D0A000DF0
:10F502000A253032582530325820526563656976B3
:10F512006564205254432062797465732025325801
:10F5220020253258202532582025325820000D0A35
:10F53200253032582530325820414D3A556E627589
:10F54200666620726420632F682F733A2025642F29
:10F5520025642F256420733A256C6420000D0A254A
:10F56200303258253032582053656E64696E6720F8
:10F572005254432062797465732025325820253213
:10F5820058202532582025325820000D0A253032C5
:10F5920058253032582053533830783A5365656BCA
:10F5A2003A205365656B696E6720746F20256C7510
:10F5B2002028256C582920000D0A25303258253084
:10F5C200325820414D3A4275666620777220632F89
:10F5D200682F733A2025642F25642F256420733AFF
:10F5E200256C64000D0A25303258253032582053DC
:10F5F2005338303A4275666620777220256C642053
:10F60200627974657320727820000D0A5265636511
:10F6120069766564205254432062797465732025AB
:10F6220032582025325820253258202532582000C1
:10F632000D0A414D3A556E627566662077722063F7
:10F642002F682F733A2025642F25642F2564207399
:10F652003A256C6420000D0A547269656420746F47
:10F662002074616C6B207768696C7374206E6F74A0
:10F6720020616464726573736564000D0A53656E7C
:10F6820064696E6720525443206279746573202541
:10F692003258202532582025325820253258200051
:10F6A2000D0A414D3A4275666620726420632F68E6
:10F6B2002F733A2025642F25642F256420733A2561
:10F6C2006C6420000D0A2530325825303258203122
:10F6D2003A526561642072746E2025582C2025648C
:10F6E200207265616420000D0A25303258253032BF
:10F6F200582053533830783A577269746520256C14
:10F70200642028256C582920000D0A2530325825FE
:10F712003032582053533830783A537461747573C9
:10F722002C20756E697420256420000D0A25303264
:10F7320058253032582053533830783A5265616434
:10F7420020256C752028256C582920000D0A2530AB
:10F7520032582530325820535338303A536574208A
:10F762006164647265737320256C5820000D0A254C
:10F772003032582530325820535338303A436820BB
:10F78200696E6420436C65617220256420000D0A55
:10F792004D617820566563746F72206469736B20C3
:10F7A200256420256C642028256C582920000D0A28
:10F7B20025303258253032582053533830783A5356
:10F7C20074617475735B25645D20255820000D0AF1
:10F7D200253032582530325820535338303A536549
:10F7E200742072656C6561736520255820000D0ACE
:10F7F200253032582530325820535338303A536529
:10F8020074206C656E67746820256C5820000D0AA0
:10F81200253032582530325820535338303A416D12
:10F8220069676F20436C65617220256420000D0AB0
:10F83200253032582530325820535338303A5365E8
:10F842007420766F6C756D6520256420000D0A2585
:10F852003032582530325820535338303A466F727E
:10F862006D617420706172616D7320000D0A253024
:10F8720032582530325820535338303A527074205F
:10F88200515354415420256420000D0A44736B7374
:10F89200656C2069732025642C206E756D6265721B
:10F8A20020697320256420003C6964656E743E20E3
:10F8B2002558202558206E7266643A2564206E64AD
:10F8C20061633A2564000D0A414D3A5365656B3A0E
:10F8D2002025642025642025642025642C20733A89
:10F8E200256C64000D0A25303258253032582053D9
:10F8F2005338303A53657420756E6974202564203C
:10F90200000D0A25303258253032582053533830F2
:10F91200783A4465736372207520256420000D0ACD
:10F92200526561642072746E2025582C2025642053
:10F9320062797465732072656164000D25303258F6
:10F942002530325820566563746F7220256C64200E
:10F9520028256C582920000D0A25303258253032CE
:10F962005820535338303A556E6B6E6F776E2025A0
:10F972005820000D0A253032582530325820535372
:10F9820038303A43616E63656C20256420000D0AAD
:10F99200253032582530325820535338303A496E88
:10F9A2006974206469736B20000D0A253032582572
:10F9B20030325820535338303A5271207374617484
:10F9C200757320000D0A414D3A556E6275666620C8
:10F9D2007772202564206279746573207278000D35
:10F9E2000A253032582530325820535338303A44A1
:10F9F2006573637269626520000D0A2530325825ED
:10FA02003032582053533830783A466D74206F7034
:10FA1200747300466F756E6420616E2052544320E9
:10FA220066696C652061742025580D0A004C6F6F61
:10FA32006B696E6720666F7220616E20525443209C
:10FA420066696C650D0A000D0A5573696E6720645C
:10FA520069736B2067656F6D6574727920257320F9
:10FA6200000D0A414D3A20496E63723A2025642006
:10FA720025642025642025642C20000D0A253032BF
:10FA8200582530325820256C6420627974657320C1
:10FA920073656E7400253032582530325820256C3B
:10FAA200642062797465732073656E742000466900
:10FAB2006E6446696C65206661696C656420736575
:10FAC200617263680D0A000D0A414D3A427566661D
:10FAD2002077722025642062797465732072780021
:10FAE2000D0A475049422072633A2564202564205A
:10FAF20062797465730D0A000D0A2530325825307B
:10FB020032582053533830783A436C656172200082
:10FB12000D0A57726974655F736563746F7273203F
:10FB22006661696C202564000D0A4469736B207359
:10FB3200656C656374206E756D6265722025640064
:10FB42000D0A5365656B20746F20256C6420666115
:10FB5200696C6564202564000D0A25303258253011
:10FB6200325820535338303A577269746520000D69
:10FB72000A4F70656E696E67206578697374696E85
:10FB82006720257320000D0A476F7420256C7520AD
:10FB9200202D20726573657474696E670053656504
:10FBA2006B696E6720746F20736563746F722025B2
:10FBB200580D0A0046696E6446696C652066616983
:10FBC2006C656420726561640D0A000D0A536565F7
:10FBD2006B696E6720746F20256C642028256C5831
:10FBE20029000D0A25303258253032582053533817
:10FBF200303A5265616420000D0A253032582530B2
:10FC0200325820535338303A44534A20000D0A25C3
:10FC12003032582530325820535338303A4E4F50F4
:10FC220020000D0A5472616E2045786563202558C4
:10FC32002020202020004469736B206368616E6776
:10FC4200653A20256420200D0A000D0A4469736B71
:10FC5200205374617475733A2025582C20000D0AC4
:10FC620057616974696E6720666F7220636172649E
:10FC720020000D566563746F7220256C6420282560
:10FC82006C582920000D0A46696C6520257320698D
:10FC920073206F70656E20000D0A57726F746520B5
:10FCA2006469736B6E6F3A202564000D0A526561B8
:10FCB20064206265796F6E6420656E64000D0A537C
:10FCC20065656B206265796F6E6420656E64000DF8
:10FCD2000A4F70656E696E67206E65772025732006
:10FCE200000D0A20256C64206279746573207365A7
:10FCF2006E74000D0A46696C6520255820697320D0
:10FD0200257320000D0A4469736B202558206973FE
:10FD120020257320004E6F742061204C49462064D8
:10FD220069736B0D0A000D0A25303258253032589E
:10FD3200204578697420000D0A414D3A53656E647E
:10FD420020737461747573000D0A52656164696E83
:10FD520067205254430D0A000D0A416D69676F20F6
:10FD620039313231440D0A000D0A44736B73656CEC
:10FD720020697320256420000D0A526561642025E4
:10FD820064206279746573000D0A48737420627985
:10FD920074657332202564000D0A577269746520F8
:10FDA2006661696C202564000D0A5353383065780A
:10FDB200656320256420000D0A4F70656E696E67C9
:10FDC2002025732020000D0A44656275672069733F
:10FDD20020256420000D0A50726F746F2069732011
:10FDE200256420000D0A5265616420636F6E6669A6
:10FDF2006720000D0A46696C656E616D652025738A
:10FE02002000566563746F722069732025580D0AAD
:10FE1200002041544E206173736572746564200042
:10FE2200222A2B2C3A3B3C3D3E3F5B5D7C7F000D02
:10FE32000A487374206279746573202564000D0A80
:10FE420056616C75653A2025580D0A0072633D258E
:10FE5200752046525F25730D0A000D0A52656365CF
:10FE620069766532353620000D0A466F726D61740F
:10FE720074696E6720000D0A4E6F20636172642000
:10FE82002564002F6C6966646174612E62696E007C
:10FE92000D0A25732025582025580D0A007B505045
:10FEA20025642025642025647D002A2A2056657257
:10FEB200696679202A2A000D0A73627974657331A2
:10FEC200202564000D0A4D6F756E74696E672000FF
:10FED2004E6F762032392032303230000D0A4B3AE2
:10FEE200257320563A2573000D0A414D3A57616B2E
:10FEF200657570004C6F6164696E672E2E2E006806
:10FF0200706469736B2E636667000D0A414D3A4354
:10FF12006C656172005B535251206F66665D0046EC
:10FF22006D742065786974200031373A35343A307F
:10FF320036005B2532582025645D005B5352512008
:10FF42006F6E5D000D0A414D3A44534A00485044D9
:10FF520069736B20004E6F2063617264002D3E2036
:10FF62002558200044534B53454C004E414D4525E6
:10FF720058004449534B25580072633D25642000C4
:10FF82005B4D4C415D0044454255470050524F5431
:10FF92004F005265616479002025303258007B455C
:10FFA20052527D00302E3135004946432000454FE4
:10FFB20049200052454E200041544E2000535251D8
:10FFC200200044415620004E444143004E524644D4
:10FFD20000525443002025580025325800207C202E
:10FFE20000443000443100443200443300443400C1
:0DFFF200443500443600443700256300000C
:020000040020DA
:08000000FFFFFFFFFFFFFFFF00
:020000040030CA
:0E000000FF06191EFF8181FF0FC00FE00F40A9
:00000001FF
